:020000040800F2
:1000000000800020CDF8000851050108793C000867
:1000100053050108550501085705010800000000B7
:10002000000000000000000000000000E1360008B1
:10003000590501080000000071370008B5370008B5
:100040005B0501085D0501085F0501086105010800
:100050006305010865050108E5040108EB040108D2
:10006000F1040108F7040108FD040108670501080F
:10007000690501086B0501086D0501086F05010898
:100080007105010873050108750501087705010868
:10009000790501087B0501087D05010803050108B4
:1000A0007F05010881050108830501088505010810
:1000B00087050108890501088B0501088D050108E0
:1000C0008F050108910501089305010895050108B0
:1000D000970501082D0D0108BD11010899050108BA
:1000E00027050108D10501089B0501089D050108A8
:1000F0009F05010800000000000000000000000053
:1001000000000000000000005FF808F110B5054C89
:10011000237833B9044B13B10448AFF300800123B3
:10012000237010BD80040020000000003CE901089D
:1001300008B5034B1BB103490348AFF3008008BD6A
:1001400000000000840400203CE9010808B50348D1
:100150000BF020F9BDE8084011F060B87A9D010865
:1001600011F05CB810B50446C06910B101210AF065
:100170003DFA206910B101210AF038FA204610BD7D
:10018000F8B50025C0E901120570C0E90335C0E9E2
:100190000555C0E90755456206990446164600F123
:1001A0001C0704F047F938B9314607480BF0F2F85C
:1001B0002021064803F0E2FC069A3946204604F066
:1001C00003F92046F8BD00BF989D0108C39D0108B2
:1001D000F8B50025C0E901120570C0E90335C0E992
:1001E0000555C0E90755456206990446164600F1D3
:1001F0001C0704F071F838B9314607480BF0CAF80B
:100200002021064803F0BAFC069A3946204604F03D
:100210004DF82046F8BD00BF989D0108C39D010818
:100220002DE9F04100259DF81860C0E90112057024
:10023000C0E90335C0E90555C0E9075545623146B7
:100240000446174600F11C0803F05AFF38B9394636
:1002500007480BF09FF82021064803F08FFC324638
:100260004146204603F03AFF2046BDE8F08100BF3A
:10027000989D0108C39D0108F0B5AFB008F040FC9F
:100280000146044612A808F041FF05F02BF9054687
:1002900012A90BF025FE04F111036B6321345A4BB4
:1002A0002C6308AC594A00930321594B2046FFF7B1
:1002B00067FF2146284605F0BBF92046FFF752FFAD
:1002C0004FF41653534A00930221534B2046FFF735
:1002D0007FFF2146284605F0ABF92046FFF742FF95
:1002E0000823012600274D4A009302214C4B20464B
:1002F000FFF76EFF2146284605F09AF92046FFF7E2
:1003000031FF484B484A00930321484B2046FFF7F2
:1003100037FF2146284605F08BF92046FFF722FFDC
:10032000434B444A00930321434B2046FFF728FFE9
:100330002146284605F07CF92046FFF713FF3F4B86
:100340003F4A009303213F4B2046FFF719FF214608
:10035000284605F06DF92046FFF704FF3A4B3B4A6B
:10036000009303213A4B2046FFF70AFF2146284617
:1003700005F05EF92046FFF7F5FE364B364A00964B
:1003800002212046FFF724FF2146284605F050F9B8
:100390002046FFF7E7FE314B314A314600962046B2
:1003A000FFF73EFF2146284605F042F92046FFF7B9
:1003B000D9FE2C4B2C4A314600972046FFF730FFE0
:1003C0002146284605F034F92046FFF7CBFE2846A3
:1003D000264B274A274904F0F3FF0621264B274ADC
:1003E0000893274BCDE905120993264B07970A93EB
:1003F00005AB93E807008DE807000B9794E80F0022
:1004000005F00EFB2FB0F0BD379B0108309B0108B3
:100410001C9B0108499B01083B9B0108659B010847
:10042000509B01087DCA0108AD9B01086F9B010824
:10043000D99B0108DE9B0108B89B0108349C010888
:100440002D9C0108E49B0108A19C01089B9C0108CC
:10045000429C0108AE9C0108F09C0108F69C010832
:10046000279D01082C9D0108459D01086101000898
:10047000509D0108749D010851FE00080000080805
:10048000D9FD00084D01000807B5054B02A901F888
:10049000010D0122186809F015FF03B05DF804FB97
:1004A0009C04002007B50B4D0B4E0C4C2B6842F200
:1004B00010720DF10701186801F0BCFB0128F5D19D
:1004C0003378002BF2D09DF8071020460AF062FF27
:1004D000ECE700BFE448002004000020049E01086F
:1004E000A0F14103052B02D8373840B27047A0F184
:1004F0006103052B01D85738F7E73038C0B2092817
:10050000F3D94FF0FF3070472DE9F04F8BB005F075
:1005100003F8037833B15A480AF03CFF4D2159489B
:1005200003F02CFB002205200121CDE9032001F07E
:1005300003FA039018B91221534803F01FFB534BE1
:1005400003AA1A6001240023C822CDE900435049C0
:10055000504801F0BBFE4FF496700AF041F8054692
:10056000C8200AF03DF8074664200AF039F806462C
:10057000C8200AF035F80995474D4FF4967180462A
:1005800005A8286009F097FE00F0C6F9214609F099
:10059000E7FB00F0E3F9214607F06EFC3F480AF064
:1005A000F9FE3F4810F0B0FB00F0D8F907F078FFF3
:1005B000DFF80491DFF804A1C8223946286809F061
:1005C000B5FE002819DD4FF0FF32002407F1FF3B94
:1005D0001BF8011F01B3632C2AD80A291CD00D294E
:1005E0001AD02029F4D00929F2D00846FFF778FF65
:1005F000002806DA2B480AF0CDFE0A2002F0DAF9CC
:10060000DAE7531C1FBF40EA021030554FF0FF32AB
:10061000013408BF0246DBE7013203D022480AF06A
:10062000B9FEEAE7012C01D12048F8E7002CE4D01C
:100630001F480AF0AFFE214630460AF011FF484637
:100640000AF0A8FE00238AF8003000F087F9C823DA
:10065000E2B231460093434607F000FF044600F043
:100660007DF907F01DFF012312488AF800300AF0D7
:1006700091FE404621460AF0F3FE4846CFE700BF10
:10068000099E01082A9E01087F9E0108E448002077
:10069000C19E0108A50400089C040020CC9E01080E
:1006A00089040008209F0108479F0108739F0108E3
:1006B000869F0108929F0108CBAC0108040000202E
:1006C00070470000F8B54FF000470026184CD4E9F9
:1006D0000223BB4208BFB24227D005F0ADFC04F1B3
:1006E0000805D5E900451349621C45F10003097866
:1006F00006F0ABF9B94208BFB04204460D4614D02B
:1007000008F0FEF9036E60301B689847A04271EB59
:1007100005030ADB294620460AF0BCFD01460648CF
:100720000AF038FE054B1878F8BD054BFBE700BF13
:10073000080000200D0700203BA001080B48002006
:100740000848002010B50020002106F061FE044694
:1007500088B14179042905D080290FD00B480AF0CF
:1007600019FE01E000F070FE204607F099F908211B
:10077000204609F03BFF064B187810BD054B027967
:100780000168186804F04EFAEEE700BF79A001088E
:10079000084800201007002038B508F0B1F90546D8
:1007A00008F036FB034C6082284608F025FB2082C7
:1007B00038BD00BF0800002008B508480AF0EAFD6F
:1007C00008F09EF9036E60301B689847044BC3E93C
:1007D0000201FFF7E1FF034B187808BD69A001088B
:1007E000080000200848002038B5114C2368DB07BA
:1007F00008D404F091FE802201460E4803F074FFF5
:10080000012323600C4B0B4A1A60FFF7C5FF08F069
:1008100077F905461C2009F0C7FE044605F174016E
:1008200007F0E2FE054B1C60054B187838BD00BF91
:10083000A0040020AC06002010070020BC0400200B
:100840000848002008B508F05BF9BDE8084008F04A
:1008500091B9000038B5114B1878D8B9104CD4E9CB
:100860000023B3F1004F08BF002A14D008F048F964
:10087000036E60301B689847D4E90023821A61EB4D
:10088000030314461D460023064AA242AB41B4BFEF
:100890000120002038BD0120FCE700BF0C0700202C
:1008A000480000204351010008B50B4B1B685B68F2
:1008B0000BB1012008BD094B1B78002BF9D1FFF7C4
:1008C000C9FF0028F5D1064B186803685B68984794
:1008D000003018BF0120EDE710070020B004002011
:1008E000BC0400201FB56123CDE9013101A90392A9
:1008F00005F0BCFB05B05DF804FB07B58DF80410EE
:1009000001A98DF805208DF8063005F06FFC03B0C5
:100910005DF804FB08F0F4B838B50C4C2368DB072D
:1009200012D408F0EDF8054608F0EAF805F14801A0
:1009300000F15802064809F04DF90123054A06491D
:100940000348236014F0E3FF014838BDA8040020E9
:10095000C006002000000020C106000810B5074CAA
:100960002368DB0708D4FFF7D7FF00F11C01044818
:1009700007F040FA01232360014810BDAC040020B9
:10098000EC0600202DE9F04F91B008F0B9F80446CC
:1009900007F0A0FD204607F0B3FDFFF76DFCFA203D
:1009A00002F008F804F0B8FD054604F0ADF9284659
:1009B00006F0D8FD5F49284604F056FC5E4C5F49BE
:1009C0002060284604F050FC082803D0092801D0F4
:1009D000072869D10026A0605949284604F04DFC3B
:1009E00007460146574817F0C5FA002861D105238C
:1009F000E3605549284604F040FC07460146534849
:100A000017F0B8FA00286ED1452363600E234FF02B
:100A10000108237484F8118084F81280FFF79EFF88
:100A20008146454C04AF0FCC0FC7D4F800C004AFCB
:100A300009F10C040FCF0FC44549C4F800C0284683
:100A400004F01BFC04460146424817F093FA0028C4
:100A50005CD1C9F804004049284604F005FC431E57
:100A6000022B01465FD93D480AF094FC01263C491F
:100A7000284604F002FC3B4B10AA1860002309A989
:100A800042F8343D0AF06CFA0399002900F08A809C
:100A900035480AF07FFC35480AF07CFC40F2FD1135
:100AA000334803F06BF880E032480AF073FC01260B
:100AB00092E73946304817F05DFA08B90A2397E7FC
:100AC00039462E4817F056FA08B90F2390E73946F1
:100AD0002B4817F04FFA08B9142389E729480AF080
:100AE00059FC012685E73946274817F043FA08B92B
:100AF0004F238AE73946254817F03CFA08B94E23B8
:100B000083E723480AF046FC01267FE72146214877
:100B100017F030FA10B9C9F804809CE71E480AF0B3
:100B200039FC464697E71D4B18701D480AF032FC09
:100B30009DE700BF499B010830000020659B01082C
:100B4000AD9B0108C4A00108DE9B010802A10108B9
:100B5000309B0108379B0108F09C010858A101084F
:100B60002D9C0108B40400208EA10108A9A1010850
:100B7000BCA101089FA001087DCA0108C8A0010806
:100B8000C5CA0108CCA0010807A10108D99B01082A
:100B90000BA101082A9B010834A10108B804002018
:100BA00077A10108002E7FF476AF284600F042FDC1
:100BB00004F0B2FC684904F03DFB08B1FFF7A4FC67
:100BC00066480AF0E7FB07F09BFF654D06462B6879
:100BD000644C13F0010F04D105F02EFA01232060BC
:100BE0002B6006F16001206805F0F8F820685E4986
:100BF00005F0F6F85D4B25681A685D4909A805F00F
:100C0000D7F809A9284605F02DF95A4D5A4A2870F7
:100C10005A492068FFF766FE594A8DF8060059497F
:100C20002068FFF75FFE8DF80700206806F046F9A0
:100C3000554A814655492068FFF754FE544A834679
:100C400054492068FFF74EFE534B8246534A54499D
:100C5000206806F05BFE534A064653492068FFF7BA
:100C600041FE524A8DF8050051492068FFF73AFECF
:100C70002A7880464F49206806F062FA07464E4DB2
:100C800020689DF806302A7880F828309DF80610F4
:100C90009DF80730FFF731FE4B462A789DF8071084
:100CA0002068FFF72AFE454A5B46494620681278CD
:100CB000FFF723FEDFF8109133462A785946206863
:100CC000FFF71BFE33462A789DF805102068FFF7D2
:100CD00014FE9DF8053099F8002031462068FFF792
:100CE0000CFE43462A7831462068FFF706FE344A58
:100CF0005346414620681278FFF7FFFD3B462A78AD
:100D000041462068FFF7F9FD9DF8053099F800206D
:100D100039462068FFF7F1FD164A534639462068E8
:100D20001278FFF7EAFD5B462A7851462068FFF704
:100D3000E4FD206805F010FC22480AF02BFB01229C
:100D40004FF4FA71206805F0A1FB002001F0ACFB24
:100D500011B0BDE8F08F00BF0BA2010816A2010878
:100D6000A4040020BC06002045080008B4040020AC
:100D700033A201080D070020E9070008EEB80108BA
:100D8000510E000838A20108CD0D000843A2010849
:100D9000B90700084EA201081D100008A9080008A4
:100DA00055A201084507000862A20108C50600080F
:100DB0006BA20108C3B80108084800200C480020B5
:100DC0000B48002075A20108C148002010B51B4C3B
:100DD00020680368DB69984707F092FE036E603075
:100DE0001B689847164BC3E900010AF053FA014605
:100DF00014480AF0CFFAFFF78FFD012108F0B0FF89
:100E0000FFF7ACFD012107F037F8206800F038FA51
:100E1000FFF7A4FD002107F02FF8FFF77DFD00216B
:100E200008F09EFF206803685B68984710B90122AC
:100E3000054B1A70054B187810BD00BFBC0400208C
:100E4000080000208FA201080C070020084800209D
:100E500010B5FFF7A1FC11480AF09CFA104CFFF7FF
:100E60005BFD012108F07CFFFFF778FD012107F011
:100E700003F8206800F004FAFFF770FD002106F087
:100E8000FBFFFFF749FD002108F06AFF20680368B7
:100E9000DB699847034B187810BD00BFA3A2010877
:100EA000BC040020084800202DE9F04FB2F5827FF5
:100EB000C9B0074689469246049303D99421554800
:100EC00002F05CFE40F20513534528BF53464FF035
:100ED00000440593002300264FF00108CDE90234B9
:100EE0003B6838465B689847002800F08E803B6876
:100EF000059A1B6906A9384698470528044607D86D
:100F000045480AF047FA3B6838469B699847E7E747
:100F10000DF119009DF818500AF051FBCDE90001C0
:100F2000E1B28C1F042DE4B22ED80539C9B24B1D95
:100F3000DBB2B8F1000F42D0529A9A4515702DD30A
:100F4000062D26D8DDE90023484602910AF065FB0C
:100F500080460299AAEB08038B421DD3033D012D65
:100F600094BF0125002509EB0800284498BF09F823
:100F7000084022460DF11E0116F015F92544EDB288
:100F8000A8445FFA88F80BE0072D2146CFD123460D
:100F9000CFE74FF00008DDE70025F1E74FF000084C
:100FA0003B6838469B699847049B46449E422CD236
:100FB000DDE900344FF00008CDE9023490E7049AEF
:100FC0008B19934221D8529B1B78AB421DD1DDE98E
:100FD0000223DDE900BC634508BF5A4515D1049BD7
:100FE0009B1B9942DCD8033D012D98BF4FF00108AF
:100FF00009EB0600404498BF09F8064022460DF16F
:101000001E0116F0D0F8A044BBE7304649B0BDE859
:10101000F08F00BFBCA1010822A001082DE9F0411A
:101020004F4E88B004460D46DE22314604A809F032
:101030001EFA00234B4F8DF80E303B68D3F8048026
:10104000B8F1000F0FD048480AF0A4F90DF10F03D2
:101050002A463146386803F097FB9DF80F3026602A
:101060006371207119E0414E3778CFB140480AF0E2
:1010700091F9404A404913680968C91A8D4228BF4E
:101080000D464FF0050161713C4928BF86F800808C
:1010900019442B4421602571136008B0BDE8F0812C
:1010A000FFF7D8FB00283ED035480AF073F907F067
:1010B00027FD036E60301B689847324DC5E900017B
:1010C000012104A809F0FEF9394604A809F0FAF94B
:1010D000032104A809F0F6F92B4B197809B1012175
:1010E0001F702A4E04A809F0EDF9B6F9121004A8F1
:1010F00009F018FA318A04A809F02CFAD5E900237E
:1011000004A809F01BFA224B04A8197809F0DAF9AF
:1011100004A809F0E2F9054604A809F0E0F9012362
:10112000256063719DE71B480AF034F9134F0DF1F8
:101130000E03194800934FF482722B46394600681B
:10114000FFF7B2FE0C4B854218609DF80E30276009
:10115000637186D2074B25711D60012333709CE7B4
:10116000C8040020100700209D9F0108B004002043
:10117000C39F0108C4040020C0040020A60500206D
:10118000E79F0108480000200C070020080000200D
:10119000B804002004A00108BC040020F7B507F043
:1011A000AFFC0F25044640F6C13707F025FE1D4E63
:1011B000B8420CDC014630460AF0ECF84FF47A7085
:1011C0000EF0E8FD204607F017FE013DF0D1236840
:1011D00020469B689847FFF79FFB0146204607F093
:1011E000BFF9204607F076F9204607F09BFC002463
:1011F00001234FF496720C49CDE900340B48234685
:1012000001F064F80A480AF0C5F80A480AF0C2F882
:1012100001F036FA40F23D21074802F0AFFC2046CB
:1012200003B0F0BDDCA2010816A30108850900087F
:101230001FA3010832A30108BCA1010810B5044690
:101240002C2109F0D3F9204610BD0000FF22014BEC
:101250001A7070470D07002003463038C0B20928C5
:101260000DD9A3F14102052A02D8373BD8B2704705
:10127000A3F16102052A01D8573BF7E7FF20704729
:101280002DE9F04F684CD5B04FF49672814609A90C
:1012900005A809F0ECF823685A681B689A4205D142
:1012A00062480AF077F855B0BDE8F08FFFF756FBBB
:1012B000012106F0E1FD23685D4F5A68D3F80080F4
:1012C000DFF880B10292029B984500F0A7803B783E
:1012D00058F8044B012B03D1032105A809F0F2F8BB
:1012E0003B78022B72D1062105A809F0EBF8DBE967
:1012F000002305A809F022F921794E480AF04AF89E
:10130000217920680AF0ACF84B480AF043F8FFF75F
:1013100025FB054605A8266894F804A009F0E8F81E
:10132000039005A809F0E0F8C0B2039B524631468D
:101330000090284607F092F80646014605463F48C9
:101340000AF028F805A809F0D3F831460AF088F821
:1013500039480AF01FF83B78023B012B0BD8226872
:1013600005A80392257909F0C3F8052D8246039A52
:1013700030D80025EDB2294605A809F0BDF83B7824
:10138000012B11D12379032B43D90222216805A80F
:10139000114409F079F8237905A8052B8ABF236841
:1013A0000021597909F08EF8D9F8003005A89C6819
:1013B00009F095F809A902464846A04710B9204807
:1013C00009F0E8FF05A809F08CF87CE7032B8ED123
:1013D000072189E7022ECCD91046294606F0ECFCFD
:1013E000421ED2B2F92AC4D89AF901200546002A31
:1013F00005DA0246FF21504615F0F9FEBAE7C21C95
:101400009642B6D302460AF10301504615F0D6FEC5
:10141000B0E7002105A809F09DF8BCE7FFF79EFAA8
:10142000002106F029FD3EE71407002063A3010810
:10143000B80400208AA30108CBAC01089DA30108D1
:10144000ACA30108080000202DE9F04FD7B00446F6
:1014500004F062F8524903F0EDFE28B9514809F052
:1014600099FF57B0BDE8F08FFFF754FA036E603074
:101470001B6898474FF49672CDE902010BA907A8A3
:1014800008F0F5FF267927683146474809F082FFC2
:101490003146384609F0E4FF444809F07BFFFFF786
:1014A0003BFA012108F05CFCFFF758FA012106F035
:1014B000E3FC0025DFF80491DFF804A1B54207D270
:1014C0006C1C7D5DE4B2022D0DD8394809F062FF35
:1014D000FFF744FA002106F0CFFCFFF71DFA0021C8
:1014E00008F03EFCBDE7321BD2B2954204D9294632
:1014F000304809F04FFFEBE7042107A808F0E2FFAE
:10150000DDE9022307A809F019F8FFF727FA834657
:1015100007A808F0EDFF059007A808F0E5FF07EB26
:101520000408C0B2059B2A4600904146584606F082
:1015300095FF83460146204809F02CFF594607A82D
:1015400008F0DAFF032D09D0A11C0222394407A8B4
:1015500008F09AFF052D06D8002106E0002107A813
:1015600008F0F8FFF8E798F8051007A808F0AAFFB8
:10157000D9F8008007A8D8F80030D3F808B008F0F0
:10158000AEFF0BA902464046D84710B9504609F0B5
:1015900001FF2C4407A8E5B208F0A3FF8EE700BFC7
:1015A000279D010815A501086BA50108CBAC010812
:1015B0007BA50108B0A50108F6A50108BC04002020
:1015C00004A60108F8B504460E46D0E9002180685B
:1015D0008B1A9B100133091AB3EBA10F4FEA830753
:1015E0000CD83A4462606FF040432168626830680A
:1015F000521A03EBA20341F82300F8BD384609F064
:1016000065FF054618B96921094802F0B7FAD4E91F
:1016100000128A4203D0521A284615F0CFFD2068E6
:1016200009F03EFF25603D44C4E90155DBE700BFFA
:1016300038A601082DE9F04F0446C5B00C2008F08B
:10164000B3FF00254D4FC0E90055856038604C4917
:10165000204603F012FE4FF00108834681462C46D7
:10166000DFF840A119F8016BB8F1000F0BD12C2E57
:1016700000D066B9A9EB0B01424809F08BFE282186
:10168000504602F07BFA2C2E2FD0002E54D030463C
:10169000FFF7E2FDFF280346A9EB0B0209D10090FA
:1016A0003146394809F076FE4221504602F066FA8A
:1016B000009BFF2C08D13548009309F06BFE4621B2
:1016C000504602F05BFA009BB8F1000F04D01D01F8
:1016D000EDB24FF00008C5E71D43EDB2631C04AA4C
:1016E00015554FF00108DCB2BCE71CB32849204671
:1016F00008F078FF034640B90090264809F04AFEFA
:101700003021504602F03AFA009B04A918462246BE
:10171000019315F048FD3A680820009208F044FF54
:10172000019B009A03600471039003A91046FFF720
:1017300049FF1EB1002495E7002CD7D13B6816481D
:1017400059681B68154EC91A891009F023FE3B68B9
:10175000134FD3E9004844450CD054F8045B384695
:1017600009F018FE2868297909F07AFE304609F058
:1017700011FEF0E745B0BDE8F08F00BF1407002070
:101780009B9C0108D7A3010879A40108B1A4010812
:101790003EE6010864A40108D9A40108CBAC010805
:1017A0000DA5010813A4010810B5044601F0AAFF15
:1017B000A46B01F0C7FFB4FA84F0400910BD70B506
:1017C0001546026C0446866B42B905689DB980686F
:1017D00001F03AFBA5600136A66370BD6DB94068A3
:1017E00015F0E1FC6368226C1344A26863609342C5
:1017F00001D3236863600020EDE7C06815F0D3FCD7
:10180000236CE2685B4221681A448A42E2603EBF70
:10181000A2689B18E360022DEDD10EB1013EEAE70C
:101820003046D8E703461A6C10B4084662B1D9684E
:101830009C681144A142D96028BF196810BC28BF18
:10184000D960D96815F0AFBC10BC704770B50446BC
:1018500001F058FF94F8455004F124066DB2002DB4
:1018600014DCFF2384F8453001F06CFF01F04AFFDF
:1018700094F8445004F110066DB2002D12DCFF23E1
:1018800084F84430BDE8704001F05CBF636A002B0F
:10189000E7D0304601F0AAF908B101F029FA013D7C
:1018A0006DB2DCE72369002BE9D0304601F09EF9E8
:1018B00008B101F01DFA013D6DB2DEE738B50D4605
:1018C000044620B940F20311194802F057F901F01B
:1018D00019FFD4E90F314B432268D0185B1A134427
:1018E000A060E3600020FF23A063626084F84430BE
:1018F00084F8453095B9236963B104F1100001F013
:1019000075F938B14FF080520A4B1A60BFF34F8F10
:10191000BFF36F8F01F016FF012038BD04F11000F6
:1019200001F058FE04F1240001F054FEF2E700BF7C
:1019300078A6010804ED00E0F8B50D461746064606
:1019400020B94FF4BB710D4802F018F905FB06F001
:10195000503002F011F8044648B155B92060C4E98E
:101960000F6501212046FFF7A9FF84F84C7020463F
:10197000F8BD00F150030360F1E700BF78A601084D
:101980002DE9FF47884601921E46044620B940F2E1
:10199000F1214B4802F0F2F8B8F1000F06D1236CA8
:1019A00023B140F2F221464802F0E8F8022E07D1B6
:1019B000E36B012B04D040F2F321414802F0DEF842
:1019C00001F0E0F930B9019B23B140F2F6213C4827
:1019D00002F0D4F80027B946DFF8E8A001F092FE43
:1019E000A26BE36B9A4201D3022E19D132464146D3
:1019F0002046FFF7E4FE636A1BB104F1240001F006
:101A0000F5F838B14FF080522E4B1A60BFF34F8F6C
:101A1000BFF36F8F01F096FE012004B0BDE8F087A0
:101A2000019D1DB901F08EFE0020F6E717B902A84E
:101A300001F01CF901F086FE00F062FE01F062FE8A
:101A400094F84430FF2B08BF84F8449094F8453054
:101A5000FF2B08BF84F8459001F074FE01A902A88D
:101A600001F010F928BB01F04DFEA26BE36B9A4226
:101A70000ED101F067FE019904F1100001F07CF82D
:101A80002046FFF7E3FE00F0E1FE48B10127A5E79D
:101A900001F058FE2046FFF7D9FE00F0D7FEF5E72B
:101AA0004FF08053CAF80030BFF34F8FBFF36F8FF2
:101AB000ECE72046FFF7CAFE00F0C8FEB4E700BF1F
:101AC00078A6010804ED00E010B5024600210120CF
:101AD000FFF732FF044638B1002383600360C36020
:101AE0001A461946FFF74CFF204610BD2DE9F84372
:101AF000894690461F46044620B940F2C331274824
:101B000002F03CF8B9F1000F06D1236C23B14FF479
:101B10007171224802F032F8022F07D1E36B012BDA
:101B200004D040F2C5311D4802F028F801F0C4FE8F
:101B3000EFF311864FF0500383F31188BFF36F8FDB
:101B4000BFF34F8FA26BE36B9A4201D3022F22D1D6
:101B500094F845503A466DB249462046FFF72FFEAD
:101B60006B1C13D1636A0BB901200BE004F1240054
:101B700001F03CF80028F7D0B8F1000FF4D00120B4
:101B8000C8F8000086F31188BDE8F88301356DB20E
:101B900084F84550E8E70020F4E700BF78A6010884
:101BA00070B50D46044620B94FF48C61204801F011
:101BB000E5FF236C23B140F264411D4801F0DEFFD4
:101BC000236833B9A36823B140F26941184801F092
:101BD000D5FF01F071FEEFF311864FF0500383F350
:101BE0001188BFF36F8FBFF34F8FA26BE36B9342EC
:101BF0001CD994F8453001325BB2A2635A1C10D153
:101C0000636A0BB9012009E004F1240000F0EEFF43
:101C10000028F7D0002DF5D00120286086F3118828
:101C200070BD01335BB284F84530EBE70020F5E787
:101C300078A601082DE9F04385B00F4601920446CD
:101C400020B94FF4A061424801F098FF37B9236CE6
:101C500023B140F204513E4801F090FF01F092F8A8
:101C600030B9019B23B140F20951394801F086FF98
:101C70000026B046DFF8DC9001F044FDA56BD5B13D
:101C800039462046013DFFF7CDFDA563236963B1C9
:101C900004F1100000F0AAFF38B14FF080522D4B34
:101CA0001A60BFF34F8FBFF36F8F01F04BFD012020
:101CB00005B0BDE8F083019D1DB901F043FD002092
:101CC000F6E716B902A800F0D1FF01F03BFD00F0E5
:101CD00017FD01F017FD94F84430FF2B08BF84F87E
:101CE000448094F84530FF2B08BF84F8458001F00C
:101CF00029FD01A902A800F0C5FFF0B92046FFF7B1
:101D000053FDA0B1019904F1240000F035FF2046F5
:101D1000FFF79CFD00F09AFD38B94FF08053C9F8E9
:101D20000030BFF34F8FBFF36F8F0126A4E720462B
:101D3000FFF78CFD00F08AFDF7E72046FFF786FDF0
:101D400000F084FD2046FFF72FFD0028EDD0B6E718
:101D500078A6010804ED00E02DE9FF410446019159
:101D600020B940F29151524801F008FF236C23B191
:101D700040F295514E4801F001FF01F003F830B9EF
:101D8000019B23B140F29A51494801F0F7FE00252A
:101D90002F462E46DFF81C8101F0B4FCA36BE3B1A3
:101DA000013BA363236813B901F0EEF8A060236937
:101DB00063B104F1100000F019FF38B14FF0805208
:101DC0003C4B1A60BFF34F8FBFF36F8F01F0BAFC2B
:101DD0000125284604B0BDE8F081019B4BB925B12F
:101DE00040F2E151324801F0C9FE01F0ABFC0025A0
:101DF000EFE717B902A800F039FF01F0A3FC00F0EB
:101E00007FFC01F07FFC94F84430FF2B08BF84F87E
:101E1000446094F84530FF2B08BF84F8456001F01A
:101E200091FC01A902A800F02DFF40BB2046FFF75E
:101E3000BBFCF0B123683BB901F064FCA06800F082
:101E4000B1FF054601F07EFC019904F1240000F089
:101E500093FE2046FFF7FAFC00F0F8FC38B94FF08B
:101E60008053C8F80030BFF34F8FBFF36F8F012747
:101E700092E72046FFF7EAFC00F0E8FCF7E720468F
:101E8000FFF7E4FC00F0E2FC2046FFF78DFC0028A1
:101E9000EDD0002D9DD001F035FC616A19B1236BA6
:101EA0001968C1F10501A06801F01AF89DE700BFAB
:101EB00078A6010804ED00E02DE9F04385B00F4657
:101EC0000192044620B94FF4CD61424801F056FE1C
:101ED00037B9236C23B140F26C613E4801F04EFEED
:101EE00000F050FF30B9019B23B140F271613948D5
:101EF00001F044FE0026B046DFF8DC9001F002FC61
:101F0000A36BD3B139462046E568FFF78BFC636AC3
:101F1000E56063B104F1240000F068FE38B14FF0D1
:101F200080522D4B1A60BFF34F8FBFF36F8F01F0BC
:101F300009FC012005B0BDE8F083019D1DB901F049
:101F400001FC0020F6E716B902A800F08FFE01F0B0
:101F5000F9FB00F0D5FB01F0D5FB94F84430FF2BE2
:101F600008BF84F8448094F84530FF2B08BF84F8FC
:101F7000458001F0E7FB01A902A800F083FEF0B95B
:101F80002046FFF711FCA0B1019904F1240000F0F4
:101F9000F3FD2046FFF75AFC00F058FC38B94FF02B
:101FA0008053C9F80030BFF34F8FBFF36F8F012606
:101FB000A4E72046FFF74AFC00F048FCF7E720467C
:101FC000FFF744FC00F042FC2046FFF7EDFB002841
:101FD000EDD0B6E778A6010804ED00E02DE9F8435E
:101FE00089469046054620B940F2FB61204801F041
:101FF000C5FDB9F1000F06D12B6C23B140F2FC6195
:102000001B4801F0BBFD01F057FCEFF311874FF0C7
:10201000500383F31188BFF36F8FBFF34F8FAC6B07
:102020001CB395F84460494676B22846FFF7FAFBA0
:10203000013C731CAC6313D12B690BB901200BE07D
:1020400005F1100000F0D2FD0028F7D0B8F1000F24
:10205000F4D00120C8F8000087F31188BDE8F883A8
:10206000013676B285F84460E8E72046F4E700BF21
:1020700078A6010810B5044620B940F28A710548D7
:1020800001F07CFD01F03EFBA46B01F05BFB204600
:1020900010BD00BF78A6010838B5054620B940F24A
:1020A000A471064801F06AFD01F02CFBA86BEC6BF3
:1020B000241A01F047FB204638BD00BF78A601086E
:1020C000002330B5064A52F8335002EBC3041DB961
:1020D00042F83310606030BD0133052BF3D1FAE7CD
:1020E000A4500020002310B5074A02EBC3014C683E
:1020F000844204D1002042F83300486010BD01330F
:10210000052BF2D1FAE700BFA450002010B5044619
:1021100020B94FF4F861054801F030FD2046FFF783
:10212000E1FF2046BDE8104001F0B8BC78A60108E8
:1021300070B504460D46164601F0E4FA94F84430B2
:10214000FF2B04BF002384F8443094F84530FF2B64
:1021500004BF002384F8453001F0F4FAA36B2BB9D7
:102160003246294604F1240000F020FD2046BDE857
:102170007040FFF76BBB0000064A13681968064BF6
:1021800019B94FF0FF321A6070471268D268D268EE
:102190005268F8E71C070020CC07002010B5044661
:1021A00020B940F2F261084801F0E8FC6269074B8F
:1021B0009A4207D1A06A064B984203D0B0FA80F049
:1021C000400910BD0020FCE7C4A60108EC07002070
:1021D000D4070020F8B51B4B1B4E1C680546306821
:1021E0000F46043001F027FA334640B90120316828
:1021F000164EC96A3268884022EA000232606A1CC0
:1022000007D137B1196812480431BDE8F84001F030
:10221000EFB91A686419546007D30E4A1068196838
:10222000BDE8F840043101F0EFB90B4A10681968B5
:10223000043101F0E9F9094B1A68A24288BF1C6019
:10224000F8BD00BF14080020180700209C070020DC
:10225000EC070020200700201C070020CC070020EE
:1022600080B5DFF86480144F144C154E236863B9B1
:10227000144B1B68012BF8D94FF08053C8F800307D
:10228000BFF34F8FBFF36F8FEEE701F03BFAFB68B0
:10229000DD68281D01F0CFF93368013B3360236806
:1022A000013B236001F04EFA286B01F0F7FB284652
:1022B00001F0F4FBDAE700BF000800208C070020E3
:1022C000880700202407002004ED00E02DE9F84FE6
:1022D0004FEA820A804650460D4699460B9E01F011
:1022E0004BFB0746002800F0AB805C2001F044FB6C
:1022F0000446002800F0A180076325B94FF4587107
:10230000564801F03BFC5246A521206B14F06FFFAC
:10231000236BAAF1040A9A442AF0070A6B1E04F1FF
:1023200034020F3513F8011F02F8011B197809B1A7
:10233000AB42F7D10A9D4FF0000B042D28BF0425B6
:10234000271DE562C4E9135B384684F843B001F009
:102350004CF9C5F1050504F1180001F046F9C4F87F
:1023600054B02461A561646284F858B04A4641467D
:10237000504601F09FF9206006B1346001F0C2F9C7
:10238000374B384E1A68DFF8188101321A6032680C
:10239000002A58D134601B68012B25D1324801F046
:1023A00019F9324801F016F9314801F013F9DFF854
:1023B000F490304801F00EF92F4D304801F00AF941
:1023C000484601F007F9284601F004F92C4801F0CD
:1023D00001F92C4801F0FEF82B4801F0FBF82B4BDB
:1023E000C3F800902A4B1D6001252A4A2A49136828
:1023F000086801331360E26A636405FA02F3034379
:1024000014200B60184B394600FB023001F0F0F845
:1024100001F098F9D8F8003063B13368DA6AE36AFA
:102420009A4207D24FF080521C4B1A60BFF34F8F75
:10243000BFF36F8F2846BDE8F88F384601F02EFBBA
:102440004FF0FF35F6E7D8F80030002BCCD13368D9
:10245000DA6AE36A9A4298BF3460C5E7C4A6010805
:1024600088070020180700202407002038070020D4
:102470004C07002060070020B407002074070020EC
:10248000D407002000080020EC0700201C070020D3
:1024900020070020980700209C07002004ED00E0A2
:1024A000E8070020A007002070B50446284D01F081
:1024B00029F904B92C68261D304601F0BCF860B932
:1024C0001421E06A234B41435B5833B9012222496E
:1024D00082400B6823EA02030B60A36A1BB104F17C
:1024E000180001F0A8F81D4A1368013313602B6827
:1024F000A34220D131461A4801F07AF8194A1368EC
:102500000133136001F01EF9174B1B6893B12B6860
:10251000A3420FD1154B1B6823B140F2B6411448BA
:1025200001F02CFB4FF08052124B1A60BFF34F8F1B
:10253000BFF36F8F70BD104A206B1368013B1360AF
:1025400001F0ACFA204601F0A9FAFFF715FED9E731
:1025500018070020240700209C070020980700206F
:10256000000800208C070020E807002094070020C6
:10257000C4A6010804ED00E088070020F8B5054670
:1025800020B940F24C51174801F0F8FA164B1B687D
:10259000AB4220D001F0B6F8144B6C691F68144BA5
:1025A0001E6801F0CFF8BC4217D0B44215D0114BD1
:1025B0009C4208D1AB6A83B995F85830012B0CBF07
:1025C00002200320F8BD0C4B9C4208D0002C0CBF0D
:1025D00004200120F6E70020F4E70220F2E70420BF
:1025E000F0E700BFC4A60108180700201C07002060
:1025F00020070020EC0700200008002070B50446EA
:1026000020B940F21C71194801F0B8FA184D2B6836
:10261000A34229D044B301F075F82046FFF7BEFD70
:10262000F0B1261D304601F006F801231149E26A97
:1026300008689340034314200B600F4B314600FBA6
:10264000023000F0D5FF2B68E26ADB6A9A4207D3BA
:102650004FF08052094B1A60BFF34F8FBFF36F8F5B
:10266000BDE8704001F06EB870BD00BFC4A601089F
:10267000180700209C0700202407002004ED00E03C
:1026800013B50024174B009401935022234616499A
:102690001648FFF71BFE012818D100F013FE012891
:1026A00014D14FF0500383F31188BFF36F8FBFF342
:1026B0004F8F4FF0FF320E4B1A600E4B18600E4BCF
:1026C0001C6002B0BDE8104001F09CB8013007D199
:1026D00040F60401094802B0BDE8104001F04EBACE
:1026E00002B010BDC807002010A701086122000831
:1026F000CC070020E807002014080020C4A6010829
:10270000024A136801331360704700BF940700202A
:10271000014B1868704700BF1408002008B501F08D
:10272000CBF8014B186808BD140800202DE9F84FBC
:102730003A4B1B68002B6AD1394B1C6801341C6072
:102740009CB9384D2B681B6823B140F6622136488E
:1027500001F014FA354B2A68196829601A60344A66
:10276000136801331360FFF707FD324D4FF0000B84
:102770002B68314FA34211D93A68304BD16A1422E9
:102780004A439A58022A28BF4FF0010B2C4A12687C
:10279000002A0CBF58460120BDE8F88FDFF884A05E
:1027A000DFF8A490DAF8002012681AB94FF0FF326F
:1027B0002A60E1E7DAF80020D268D66871688C42B6
:1027C00001D22960D8E706F10408404600F033FF43
:1027D000B16A19B106F1180000F02DFF01224FF087
:1027E000140CF06AD9F8003002FA00F11943134BC7
:1027F000C9F800100CFB0030414600F0F9FE3868C3
:10280000F16AC26A914228BF4FF0010BCAE70D4A34
:102810004FF0000B136801331360B7E794070020F3
:10282000140800201C070020C4A60108200700206F
:10283000D0070020CC070020180700202407002024
:1028400018080020900700209C0700202DE9F8437D
:102850002E4C236823B940F668012D4801F08EF90B
:1028600000F050FF2368013B236024682CB1002452
:1028700000F068FF2046BDE8F883264B1B68002B5C
:10288000F5D0254D254EDFF8A8801FE0EB68012725
:10289000DC6804F1040904F1180000F0CCFE48469D
:1028A00000F0C9FE1420E26A316807FA02F30B4314
:1028B00000FB02804946336000F09AFE184BE26A42
:1028C0001B68DB6A9A4201D3164B1F602B68002BF2
:1028D000DCD10CB1FFF750FC134D2C6844B101273B
:1028E000104EFFF723FF00B13760013CF9D12C6097
:1028F0000C4B1B68002BBAD04FF080520B4B1A6068
:10290000BFF34F8FBFF36F8F0124B1E7940700200F
:10291000C4A6010888070020D40700209C070020D7
:1029200018070020180800209007002004ED00E0A0
:102930002407002038B50C46054620B940F2CA41AC
:10294000184801F01BF924B940F2CB41154801F0B9
:1029500015F9154B1B6823B140F2CC41114801F029
:102960000DF9FFF7CDFE114B2A68186814192CBF1A
:102970000121002182422C600CD961B9FFF766FF6A
:1029800038B94FF080520A4B1A60BFF34F8FBFF334
:102990006F8F38BD09B9A042F0D20021201AFFF78D
:1029A00019FCEBE7C4A601089407002014080020D6
:1029B00004ED00E010B5044640B94FF080520D4BD5
:1029C0001A60BFF34F8FBFF36F8F10BD0A4B1B68A8
:1029D00023B14FF4A461094801F0D0F8FFF790FE4D
:1029E00000212046FFF7F6FBFFF730FF0028E4D078
:1029F000EBE700BF04ED00E094070020C4A6010847
:102A0000224B70B51A68224B12B101221A6070BDB8
:102A1000204E1A6033681B6B1A68B2F1A53F0BD1C8
:102A20005A68B2F1A53F07D19A68B2F1A53F03D128
:102A3000DB68B3F1A53F04D030683168343101F070
:102A40006DF8154B1C68B4FA84F41423E4B2C4F195
:102A50001F046343114DEB5823B940F688311048E9
:102A600001F08CF8142202FB04F3E91848680833DB
:102A700040682B44984202FB045408BF43684860F6
:102A800008BF4B606368DB683360C0E794070020D1
:102A900018080020180700209C07002024070020A9
:102AA000C4A6010870B504462A4E00F02BFE04B9F6
:102AB0003468251D284600F0BEFD60B91421E06A87
:102AC000254B41435B5833B90122244982400B68AE
:102AD00023EA02030B60A36A1BB104F1180000F0A3
:102AE000AAFD29461E4800F083FD94F858301D4D7C
:102AF000012B04BF002384F8583000F023FE2A681D
:102B00002AB100F0FFFDFFF737FB00F01BFE336832
:102B1000A34211D12B6883B1134B1B6823B14FF42F
:102B2000D961124801F02AF84FF08052104B1A6018
:102B3000BFF34F8FBFF36F8F70BD094A11680D4A05
:102B40001268914201D13360F6E7BDE87040FFF7AB
:102B500057BF00BF18070020240700209C07002053
:102B6000EC070020E807002094070020C4A6010815
:102B700004ED00E08807002038B50D46044620B972
:102B800040F69F31074800F0F9FF074B20461968CF
:102B9000183100F039FD2846BDE838400121FFF723
:102BA00019BB00BFC4A601081807002070B50E4667
:102BB0001446054620B940F6CA310A4800F0DEFF47
:102BC000094B28461968183100F012FD002C2146E7
:102BD00008BF3046BDE8704018BF4FF0FF30FFF728
:102BE000F9BA00BFC4A601081807002038B5C368A9
:102BF000DC6824B940F6FA31154800F0BFFF04F153
:102C00001805284600F017FD124B1B68E3B9251D77
:102C1000284600F010FD01230F49E26A086893403E
:102C2000034314200B6029460C4B00FB023000F0DC
:102C3000DFFC0B4BE26A1B68DB6A9A4285BF01200E
:102C4000084B0020186038BD29460748EFE700BF51
:102C5000C4A60108940700209C0700202407002038
:102C60001807002018080020D4070020034B1B6819
:102C70000360034B1B684360704700BFD007002010
:102C80001408002070B50C46054620B940F6654191
:102C9000144800F073FF24B940F66641114800F073
:102CA0006DFF00F02FFD104B1A682368591C0FD0E0
:102CB0000E482E6800686968864201D091420ED99C
:102CC000521A934209D99B1A23602846FFF7CEFF78
:102CD000002400F037FD204670BD0023236001244E
:102CE000F7E700BFC4A6010814080020D0070020A1
:102CF0000122014B1A6070471808002070B50C467D
:102D00001646054608B91B4A156805F1340262608B
:102D1000EA6A052B22612A6B2560E2616A6CA26077
:102D2000EA6C62614FF00002A2611BD01149096890
:102D3000A9420BD12273D6B1296B0A46531A12F855
:102D4000010BA528FAD09B08238470BD032B2373A5
:102D5000F1D1FFF7D5FCAB6A0BB102232373FFF768
:102D600075FDE8E72846FFF709FC2073E3E72684B2
:102D7000EBE700BF18070020014B1868704700BF41
:102D800018070020054B1B6833B1054B1B68002B4F
:102D90000CBF02200020704701207047E807002088
:102DA000940700202DE9F0410446002836D0234A3C
:102DB000C36A11681746C96A8B4237D214268269E2
:102DC0001F4D002AA8BF3A6806FB0353A2BFD26A70
:102DD000C2F10502826142699A4221D100F10408E0
:102DE000404600F028FC174B48B9E06A4643AA5910
:102DF0002AB901211A68814022EA01021A603A6860
:102E00001968D26AE262012404FA02F008431860E9
:102E10001420414600FB025000F0EAFB204603E08C
:102E20003B68DB6AC3620120BDE8F0811368C06CB7
:102E3000DC6AA0422CBF00200120F5E71807002023
:102E4000240700209C070020F8B5044608B900209C
:102E5000F8BD1F4B1B68834204D040F67A711D48B1
:102E600000F08CFE236D23B940F67B71194800F009
:102E700085FE236DE16AE26C013B91422365E6D059
:102E8000002BE4D1251D284600F0D5FB124E134A35
:102E900050B91421E76A794373582BB9012013689C
:102EA000B84023EA00031360E36CC3F10501A1619C
:102EB000E3620124116804FA03F00843106014204F
:102EC000294600FB036000F093FB2046C0E700BFEB
:102ED00018070020C4A60108240700209C07002032
:102EE000F8B50D460446002845D0036D23B940F6D9
:102EF000C971214800F042FEE36C9D4238BF1D4677
:102F0000E36AAB4237D0236D012B34D11B4B1B68D6
:102F1000A34204D140F6E471174800F02FFE1426B6
:102F2000A269E36A002AE562A4BFC5F10505A561AF
:102F3000134D626906FB03539A421CD1271D384684
:102F400000F079FBE26A0F4C40B95643AB592BB9FC
:102F500001212368914023EA010323600123142007
:102F6000216893400B432360394600FB0250BDE8C3
:102F7000F84000F03DBBF8BDC4A6010818070020CA
:102F8000240700209C070020044B1A681AB1196816
:102F90000A6D01320A651868704700BF18070020E3
:102FA0002DE9F0411E4C1E4680460F46154600F0A6
:102FB000A9FB236893F85830022B14D00121236811
:102FC0005A6D22EA08025A65236883F8581056B1F0
:102FD0003046FFF7FFF84FF08052124B1A60BFF3F4
:102FE0004F8FBFF36F8F00F0ADFB00F08BFB15B17F
:102FF00023685B6D2B602368002293F85830022B06
:1030000009BF012500252368596D04BFB9435965DF
:10301000236883F8582000F095FB2846BDE8F0812E
:103020001807002004ED00E0F8B50E4617461D46CF
:10303000044620B941F219212B4800F09FFD00F011
:1030400061FB0DB1636D2B60022394F8585084F836
:103050005830EDB2042F16D8DFE807F00A03070551
:103060001100636D1E43666502E0636D01336365A5
:10307000012D11D0012400F065FB2046F8BD022D82
:10308000F1D10024F7E7636D0133F1D041F24A2119
:10309000154800F073FDEBE7261D304600F0CBFA33
:1030A0001420124AE36A11689D400D431560104ACE
:1030B000314600FB032000F09BFAA36A23B141F2E2
:1030C0005921094800F05AFD0A4BE26A1B68DB6A85
:1030D0009A42CFD94FF08052074B1A60BFF34F8FFF
:1030E000BFF36F8FC6E700BFC4A601089C0700208E
:1030F000240700201807002004ED00E02DE9F84324
:10310000DDF820800E4691461D46044620B941F266
:103110008C21354800F032FD00F0CEFBEFF3118733
:103120004FF0500383F31188BFF36F8FBFF34F8FBE
:103130000DB1636D2B60022394F8585084F8583019
:10314000EDB2B9F1040F16D8DFE809F00A0307055C
:103150001100636D1E43666502E0636D01336365B4
:10316000012D11D0012087F31188BDE8F883022DCD
:10317000F1D10020F7E7636D0133F1D041F2CF21A7
:10318000194800F0FBFCEBE7A36A23B141F2DA2116
:10319000154800F0F3FC154B1B6803BB251D2846A2
:1031A00000F049FA01231249E26A08689340034398
:1031B00014200B6029460F4B00FB023000F018FA78
:1031C0000D4BE26A1B68DB6A9A42CBD90123B8F146
:1031D000000F01D0C8F80030084A1360C2E704F1BC
:1031E00018010748EAE700BFC4A6010894070020B9
:1031F0009C07002024070020180700201808002042
:10320000D407002038B5054608B9084B1D680024CE
:1032100000F078FA95F85830022B04BF85F8584032
:10322000012400F08FFA204638BD00BF18070020A7
:10323000F8B50F4C00F066FA2568ADB90D4F0E4E8B
:10324000384600F0C7F9304600F0C4F90B4B2A4667
:103250001F600B4B0C210A201E60FEF76DFB2060E7
:1032600010B10849FEF72CFFBDE8F84000F06ABA3B
:103270005008002024080020380800201C080020E6
:103280002008002015A70108914208B5416000619F
:103290000AD8D21A83699A420DD2084B011D1868C8
:1032A00000F0B2F9002008BD9A4201D2994202D240
:1032B000011D034BF3E70120F5E700BF20080020C4
:1032C0001C08002007B5FFF7B3FF0C4B1B6843B980
:1032D0000B484FF4897100F051FC002003B05DF8F9
:1032E00004FB084BC82201930123074900930748B8
:1032F0000023FEF7EBFF0028EAD0EFE7500800209C
:103300001AA701085408002067A7010829340008FB
:103310002DE9F04180462C200D4617461E4600F050
:103320002BFB044688B125B94FF4B671084800F06C
:1033300025FCFFF77DFF069BC4F80080C4E9065713
:1033400026626362201D00F050F92046BDE8F0813E
:103350001AA701082DE9FF410D4690461F46064673
:1033600020B94FF4C3710F4800F008FC0E4C2068E0
:1033700078B1052DCDE9015803960DDCFFF702FD6C
:10338000002302280CBF0A9A1A4601A92068FEF7FA
:10339000F7FA04B0BDE8F08100233A4601A9FEF730
:1033A000A5FBF6E71AA70108500800202DE9F7430E
:1033B00000271A4DDFF86C802B681A6832B9184A5A
:1033C00011681360296003B0BDE8F083DB68DC6836
:1033D0001E6804F10409484600F02DF9636A20468E
:1033E0009847E369012BE7D1A36933449E4206D293
:1033F000636024614946286800F006F9DCE7002391
:103400000097324619462046FFF7A4FF0028D3D183
:1034100040F27231404600F0B1FBCDE71C080020BD
:10342000200800201AA701082DE9F04F4FF00108ED
:10343000624D89B0DFF898B1DBF80020136843B320
:103440000024D368D3F80090FFF75AF9FFF760F92A
:103450005B4B82461A681F4690425A4E1CD3186036
:10346000002C4CD0584B1B681A68B2FA82F25209F1
:10347000A9EB0A013068FEF75BFEFFF7E7F998B9A0
:103480004FF08052514B1A60BFF34F8FBFF36F8FD5
:103490000AE001249946D7E70393FFF787FF039BD0
:1034A000C3F800A0FFF7D2F9002205A93068FEF7A3
:1034B000C1FB0028BED0059B002BF5DB079C636990
:1034C00013B1201D00F0B7F8FFF722F93B688146E1
:1034D000984201D2FFF76AFF059BC7F80090092BBD
:1034E000E2D808FA03F313F4047A57D113F0C70FA4
:1034F00033D19B06D8D5204600F0D0FAD4E78145D9
:1035000029D8FFF7A3F9DBF80030DB68D3F80CB05B
:103510000BF1040000F08FF8DBF81C30012B15D103
:10352000DBF818104B46524649445846FFF7ACFEAC
:1035300060B1009423464A4621465846FFF70AFFE9
:1035400020B94FF4F471284600F018FBDBF8243062
:1035500058469847A8E722468AE7A169069B4A464B
:1035600019442046FFF790FE00289DD0636A20464C
:103570009847E369012B97D1A2690699CDF800A07D
:103580000A44534651462046FFF7E4FE00288BD1FB
:1035900040F20131284600F0F1FA85E7069BA3616D
:1035A00023B94FF44671284600F0E8FAA1694B466A
:1035B0004A4649442046FFF767FE75E71AA7010807
:1035C0004C080020500800202008002004ED00E0F6
:1035D0001C0800204FF0FF3200F108034360C0E9EF
:1035E00002230361002303607047002303617047D7
:1035F00043689A684B608A609A6851609960036872
:1036000008610133036070470A6830B5531C0AD162
:1036100003695A684A6091608B6059600368086169
:103620000133036030BD00F108035C6825689542F2
:10363000EFD82346F9E70369D0E901128A6082686E
:1036400051605968814208BF5A60002202611A68BD
:10365000013A1A601868704706480068006880F3ED
:10366000088862B661B6BFF34F8FBFF36F8F00DF7C
:1036700000BF000008ED00E0002307B501930B4BED
:103680001B68013303D0CA21094800F077FA4FF0D4
:10369000500383F31188BFF36F8FBFF34F8F019BEC
:1036A000002BFCD003B05DF804FB00BF50000020ED
:1036B0006FA701084FF0807340F8043C054B21F0E0
:1036C000010140F8081C40F80C3C40F8202C403820
:1036D000704700BF793600080000000000000000BD
:1036E000074B19680868B0E8F00F80F30988BFF34A
:1036F0006F8F4FF0000080F311884EF00D0E704771
:10370000180700204FF0500383F31188BFF36F8F29
:10371000BFF34F8F084A13680133012B136009D19F
:10372000064B1B6813F0FF0F04D040F275110448DC
:1037300000F024BA704700BF5000002004ED00E004
:103740006FA7010810B5074C236823B94FF4BE7169
:10375000054800F013FA2368013B23600BB983F39B
:10376000118810BD500000206FA701080000000064
:10377000EFF30980BFF36F8F0D4B1A6820E9F00F4C
:1037800010602DE908404FF0500080F31188FFF7DA
:1037900037F94FF0000080F31188BDE80840196840
:1037A0000868B0E8F00F80F30988BFF36F8F7047A7
:1037B0001807002008B54FF0500383F31188BFF3BA
:1037C0006F8FBFF34F8FFEF7B1FF18B14FF08052EC
:1037D000024B1A60002383F3118808BD04ED00E05A
:1037E0000022054B05491A600A6041F26701044A4C
:1037F000116007221A60704710E000E018E000E056
:1038000014E000E013B5264B264C1A78D2B2019290
:10381000FF221A701B78244ADBB28DF803309DF822
:10382000033003F0500313700723002223609DF838
:103830000310581E090629D402B123602368032B04
:1038400004D04FF49B71194800F098F92368144A8A
:103850001B0203F4E06323600024019BDBB21370BE
:10386000134B1A6842F470021A601A6842F07042F0
:103870001A60FFF7B5FF0F4B1C60FFF7EDFEFFF777
:10388000BFF8FFF7F9FE204602B010BD9DF80330E7
:1038900001225B00DBB28DF803300346C7E700BFAF
:1038A00000E400E05C080020580800206FA7010831
:1038B00020ED00E05000002008B5EFF305830F2B4A
:1038C0000AD90D4A9B5C0D4A12789A4204D940F2FB
:1038D000A5210B4800F052F90A4B0B4A1B681268ED
:1038E00003F4E063934206D9BDE8084040F2B521F5
:1038F000034800F043B908BDF0E300E05808002099
:103900006FA701080CED00E05C08002010B50F4B1C
:103910001A68824218D35C681919884201BF41684D
:10392000184609195960446801198A4207D10849A3
:1039300009688A421FBF516812680919416098429C
:10394000026018BF186010BD1346E1E77044002004
:103950006008002038B5064B064D1C68246804B981
:1039600038BD6307FAD07921284600F007F9F5E75A
:1039700070440020CFA701082DE9F8430746FEF761
:10398000BFFE3F493F4D0B680BBB3F4A3F4E5007C0
:103990001DBFD01D20F0070002F570534FF4705387
:1039A0001CBF02461B1A00201344083B23F00703E8
:1039B00070603260C3E90000981A0B60C2E9003001
:1039C000334B1860334B18604FF000432B602B686B
:1039D0001F4252D1002F41D007F1080462071CBFDB
:1039E00024F007040834002C47D02A4B1A68984664
:1039F000A24242D3254B1E687268A24202D23068AE
:103A0000002837D10968B14237D01F683168121BCE
:103A1000102A07F10807196010D906EB040919F0FC
:103A2000070F03D0D7211C4800F0A8F87368484658
:103A30001B1BC9F804307460FFF768FF14497268F3
:103A4000D8F8003008689B1A8342C8F8003038BFA5
:103A50000B602B681343736000233360FEF7F6FEA0
:103A60007B0704D040F217110B4800F087F8384666
:103A7000BDE8F88333460646BEE70027EEE700BF01
:103A80006008002064440020640800207044002086
:103A90006C44002068440020CFA7010838B50446D4
:103AA00070B3184D50F8041C2A68114204D140F23A
:103AB0002B11154800F062F854F8083C23B14FF47C
:103AC0009671114800F05AF854F8043C2A681342E1
:103AD00016D054F8081C99B923EA020344F8043CB0
:103AE000FEF70EFE094A54F8043C1168A4F10800E0
:103AF0000B441360FFF70AFFBDE83840FEF7A6BE8F
:103B000038BD00BF64440020CFA7010868440020EE
:103B1000014B1860704700BF0445002073B5124C7C
:103B2000064623780D46114A1BB913780BB172B6BD
:103B3000FEE70123002113700D48642213F057FBA8
:103B40002B4600960B4A6421094814F0BFF90A4B32
:103B50001B6803B198470125054E304607F05EFC0F
:103B600072B62570F9E700BFE444002078440020D5
:103B70007A44002040A8010804450020F7B5144C01
:103B8000064623780D46134A1BB913780BB172B65B
:103B9000FEE70123002113700F48642213F027FB76
:103BA0002B4600960D4A64210B4814F08FF90C4BFC
:103BB0001B6803B198470125074F0A4E384607F0A6
:103BC0002DFC304607F02AFC72B62570F6E700BFE0
:103BD000E5440020794400207A44002068A80108C8
:103BE0000445002077A801080368DFF888C080B585
:103BF000CCF80030164F4368164E3B608368164D74
:103C00003360C36815492B600369154A0B6043692B
:103C1000144C13608369C0692360134B1860DCF88F
:103C20000000386830682868096810481268002168
:103C3000226864221B6813F0DAFA23680C4A6421B4
:103C40000A4814F043F9094807F0E8FBFEE700BF13
:103C5000F4440020FC44002000450020F8440020EB
:103C6000E0440020E8440020EC4400207A44002096
:103C70002DA80108F0440020074B1B6803B19847AA
:103C80001EF0040F0CBFEFF30880EFF30980816989
:103C9000004A1047E93B00080445002010B101210B
:103CA00006F0A4BC704708B107F010BC70478068EC
:103CB0007047406870474368012B08D1D0E904324F
:103CC000934204D01878003018BF012070470020BC
:103CD00070474B6870B5042B04460E464FF0000346
:103CE00004D0C0E900338360204670BDD1E90425CB
:103CF000AD1AC0E9003383602846FFF7D4FFC4E95A
:103D000000000544A560D6E90453024629468B42CB
:103D100005D00AB10E78167001310132F7E75B1B4E
:103D200018446060E0E742680346022A06D1D3E9FE
:103D300004031B1A032B01D907F03FBC0020704776
:103D40004368032B06D1D0E904329A4208BF00230E
:103D5000184670470023FBE7037870B58168044676
:103D6000B3B1284A284807F015FB6368022B12D12B
:103D70002046FFF7D8FF0146244807F00BFBE16817
:103D80000B78002B3CD02248BDE8704007F002BB06
:103D9000204A2148E7E7032B05D12046FFF7D0FF53
:103DA00001461E48E9E7042B0ED100251C4ED4E93C
:103DB0000431C91A8D4205D2595D304607F0EAFA3E
:103DC0000135F4E71748D8E7012B08D12046FFF763
:103DD00072FF1549154B002818BF1946E1E7002569
:103DE0000F4ED4E904239B1A9D4205D2515D304603
:103DF00007F0D0FA0135F4E70D4807F0CBFABEE73B
:103E00000C48C1E7409C01081BA901082FA9010823
:103E100051A90108CCAC010825A90108E6AA0108AE
:103E2000049E010839A9010815A9010810A9010873
:103E30003FA90108CBAC0108B1F5705F2DE9F8434B
:103E400004460F4602D9174806F090FB06688368BF
:103E50009B1B994219D9D0F804900846FFF723FF1D
:103E600005460346A9EB0608B14505D00BB13278EB
:103E70001A7001360133F7E72068FFF70FFF05EBF3
:103E8000080325603D446360A56025683DB9284668
:103E9000C4E90155FFF702FF2846BDE8F883012079
:103EA000FBE700BF93A801082DE9F0410368561A0B
:103EB000904682680446D21A96420D4615D930467D
:103EC000FFF7F1FE07460346A84505D02A7803B15F
:103ED0001A7001350133F7E720683E44FFF7DEFE34
:103EE000C4E901662760BDE8F0814768481EFF1AF3
:103EF000BE420ED81A469D19A91A002904DD10F8F1
:103F0000011F02F8011BF7E7002EA8BF9B19636091
:103F1000E9E73D441F44FA1A002A04DD10F8012F96
:103F200003F8012BF7E763682E461846B04505D025
:103F3000327800B1027001360130F7E7A8EB0508CE
:103F40004344E4E708B509C81B1AC3F5705088421A
:103F500002D2104606F00AFB994238BF194658189B
:103F600005D2B0F5705F28BF4FF4705008BD4FF414
:103F70007050FBE72DE9F8430C46591C20461546C6
:103F80001F46FFF759FF064680B14FF00003EA19BC
:103F900029462046FFF788FFD4E901539D4208D007
:103FA0000DB100232B706368013363603046BDE8B8
:103FB000F8831B4A01212046FFF7C4FF2368074608
:103FC000A5EB0309FFF76FFE10EB090F1CBF0023E1
:103FD00000F80930236880461A460146954205D00C
:103FE00009B11078087001320131F7E7D31A0133B3
:103FF0004344104619466568954207D019B192F8B6
:1040000000C081F800C001320131F5E72D1A1D44CE
:1040100020684744FFF742FEC4E90085A760C5E772
:10402000CEA801081346426810B5032A06D1BDE8A0
:1040300010400A4600F11001FFF79CBF816802485A
:1040400007F0A8F9002010BD58A901082DE9F0419A
:1040500005460E4661B1D0E90132D21A8A4209D32F
:1040600000221E4403B11A700133B342FAD16B60CF
:10407000BDE8F081114AFFF765FF8046FFF713FEA8
:10408000D5E9001407460A460346944205D00BB111
:104090001078187001320133F7E70023641A3C44AA
:1040A000264404B123700134B442FAD12868FFF7E2
:1040B000F5FDC5E900744744AF60D9E73CAA0108A3
:1040C000D0E90032D21A914210B503D9891AFFF70C
:1040D000BDFF10BD3CBF5B184360FAE770B50C46EE
:1040E000012120461646FFF7A7FE054628B101210B
:1040F0002046FFF7E5FF23681E70284670BD0000CC
:10410000426808B5012A06D1BDE808400A4600F118
:104110001001FFF7E3BF8168024807F03BF9002078
:1041200008BD00BFCBA9010810B50C1A134605D075
:1041300001462246184613F041F80346181910BDEF
:104140002DE9F0410446A2EB01081646A368226857
:1041500008469B1A98450F4615D94046FFF7A3FD20
:1041600005460346BE4205D00BB13A781A700137B6
:104170000133F7E72068FFF791FD25604544C4E966
:104180000155BDE8F0816568AD1AA84504D83146EF
:10419000FFF7CAFF6060F4E70D442946FFF7C4FF4C
:1041A000636829461A468E4205D00AB10878107015
:1041B00001310132F7E7751B1D446560E1E700003E
:1041C00070B5D0E9043100F110060446C91A304632
:1041D000FFF732FE054640B1D4E90712914206D1FD
:1041E000A168064807F0D6F80025284670BD4FF0B4
:1041F00000033046FFF7A4FFF7E700BFE8A8010877
:104200002DE9F0418368A2EB0108174602680446D5
:104210009B1A98450E4615D94046FFF744FD0546C2
:104220000346B74205D0327803B11A700136013324
:10423000F7E72068FFF732FD25604544C4E90155E2
:10424000BDE8F0814568AD1AA84505D83946304625
:10425000FFF76AFF6060F3E70D4429463046FFF739
:1042600063FF636829461A468F4205D0087802B179
:10427000107001310132F7E77D1B1D446560DFE7F7
:1042800037B50D4601A8114607F0B5F904212846B7
:10429000FFF7D2FD044630B14FF0000302AA01A996
:1042A0002846FFF7ADFF204603B030BDFFF7E8BF5B
:1042B000426808B5022A06D1BDE808400A4600F166
:1042C0001001FFF7DDBF8168024807F063F80020A6
:1042D00008BD00BF03AA0108FFF7EABFF7B50E4605
:1042E00004461046154613F057FE00237268C4E9D1
:1042F0000033013AA360032A12D8DFE802F0022B50
:104300003B412D49284613F035FE20B12B49284664
:1043100013F030FE38B9012221463046FFF7DEFEA9
:10432000204603B0F0BD2649284613F023FE20B1F5
:104330002449284613F01EFE08B90022ECE70022AB
:1043400002A941F8042D284613F052FF021C18BFA1
:104350000122E1E702A941F8043D0022284613F0BA
:1043600047FF019B0246AB42DAD021463046FFF7B9
:1043700087FFD5E72A462146304600F025F8CFE7EB
:1043800010F00106CCD1470839462046FFF754FD0E
:104390000028C5D039462046FFF792FEB742BFD06D
:1043A000022105EB460007F0F0F80028B8DB23688F
:1043B00098550136F2E700BF10A90108A3A801082B
:1043C00015A90108A8A80108F0B5436885B0032B1A
:1043D0000D46164615D0014601A8FFF77FFFDDE91F
:1043E000011291420BD04FF000032846FFF7A8FEC0
:1043F00001240198FFF752FC204605B0F0BD0024CF
:10440000F7E7104613F0C8FD471C39462846FFF76A
:1044100013FD044618B9064806F0BCFFECE74FF060
:104420000003F21931462846FFF73EFDE4E700BFDE
:10443000AEA801080A4600F11001FFF7C5BFF8B5A4
:104440000D461946284616461F46FFF7F5FC04465A
:1044500030B14FF00003F21931462846FFF7D0FE85
:104460002046F8BD1346426810B5042A06D1BDE8BF
:1044700010400A4600F11001FFF7E1BF81680248D1
:1044800006F088FF002010BD92A901082DE9F04137
:104490000C4690461D46064640B139B108491846BB
:1044A00006F0A0F8074618B930602060BDE8F0813A
:1044B0002A46414612F077FE37602560F6E700BFD6
:1044C0003EE6010870B5054610460E46144613F048
:1044D00063FD2246034631462846BDE87040FFF79B
:1044E000D5BF000010B50C4631B1044900F0DCFC2A
:1044F000231A5842584110BD0846FCE7DEAB0108BC
:1045000010B500B121B9064806F044FF002010BDE7
:104510001AB9044AFFF7D6FFF8E70120F7E700BF12
:1045200056AA010863AA01082DE9F3410D46164673
:104530001F46FFF7E5FFB8B10E49222006F052F8FA
:104540000446A0B13046FFF7B2FB80463046FFF785
:10455000F7FB13F021FD3B46CDE90080064A2221FE
:10456000204613F0B3FC286002B0BDE8F08128605B
:10457000FAE700BF3EE601089DAA01082DE9F843CD
:104580000E46984616F8013B02F1FF39037046606B
:10459000C0F80890044615463D214A46304612F0C0
:1045A000E5FD074668BB4B46182B28BF1823C4F807
:1045B0003001A36204F10C05A26A3146284612F0CC
:1045C000F2FD0022A66AA3191A7337B1D4F830217C
:1045D000791C04F12C0012F0E6FD0022D4F83031F1
:1045E000234483F82C202EB12946404600F05CFC81
:1045F000C4F83401D4E901120A48BDE8F84306F0D2
:104600003FBF831B023DED1A182B1A46A8BF182284
:10461000B5F5807F28BF4FF48075A262C4F8305191
:10462000C8E700BFA5AA010830B504460D46084BEF
:104630009DB00093074A084B642103A813F046FC81
:1046400003AA29462046FFF73DFF1DB030BD00BF3D
:1046500097AA01088FAA010872AA01082DE9F04360
:104660001646642203F10C048FB0074688462046A4
:104670001849ADF8042013F07DFC70B9336B23B1F9
:10468000154A322101A813F021FC01AA41463846FF
:10469000FFF718FF0FB0BDE8F08320460F4913F075
:1046A00069FC0446A0B9736B002BEED00125DFF83E
:1046B0003490736B01A81B5DC5F1320128444A4652
:1046C000013413F003FC102C05F10205F1D1DCE7F5
:1046D000034ADBE7B1AA0108B6AA0108BAAA010891
:1046E000C2AA0108049E0108016000210273C0E90A
:1046F00001117047F8B5054617460E4639B332B377
:104700001D49182005F062FF044608B3C0E90067A0
:1047100000261A4B00F108074361C0E902660661F2
:104720008021384605F060FED4E90012384605F0D5
:1047300099FE1149082005F049FF90B16B68C0E966
:10474000004603B96860AB6803B15860A860F8BD63
:104750000B4806F01FFE01213046BDE8F84005F089
:1047600045BF084806F016FE0121206805F03EFF0F
:1047700018212046F1E700BF3EE6010880818283D0
:1047800061AB010866AB010870B54468054604B327
:10479000266806F1080005F02FFED6E903239A42A9
:1047A000C4B216D16B681BB96A210B48FFF7E6F952
:1047B0006868082143686B6005F018FF6B6803B9EF
:1047C000AB600121306805F011FF1821304605F07B
:1047D0000DFF204670BD00BFFEAA010810B50446BB
:1047E000006810B1012105F001FF204610BD7FB522
:1047F0000546FFF75CFA13F0CFFB0446861C2846FB
:10480000FFF757FA013803281DD8DFE800F0020649
:10481000080F0734601C04B070BD0D34FAE7284659
:10482000FFF78EFA13F0B8FB3418F3E701A8294616
:10483000FFF74FFADDE9014301A81B1B06EB430418
:10484000FFF7CCFFE6E70B34E4E700002DE9F04783
:1048500086B08146884614461D46FFF751FE68B172
:104860002046FFF7C4FF4049074605F0BBFE064659
:10487000C9F8000028B93D4806F08CFD06B0BDE837
:10488000F0872046FFF715FA0138032864D8DFE8DF
:1048900000F00214253D2046FFF709FA8146204624
:1048A000FFF709FA324B334A002814BF1846104666
:1048B000CDE900902B46304A0AE02046FFF7F7F991
:1048C00081462046FFF72FFA2B46CDE900902B4A70
:1048D0003946304613F0FAFA05463AE0612D204693
:1048E0000DD1FFF7E4F905462046FFF729FA2B46DC
:1048F000234A00903946304613F0E8FAECE7FFF718
:10490000D6F981462046FFF71BFAD1E72046FFF78C
:10491000CEF92B4600901B4A3946304613F0D6FAA2
:10492000DFF868902146054603A8FFF7D2F9DDE9D4
:10493000034AA2450AD0AF4214F8013B06D9791BBD
:1049400070194A4613F0C2FA0235F2E703A8FFF7DE
:1049500045FFC8F8005091E72046FFF7A8F92B461D
:104960000090094AC6E700BF3EE6010861AB0108B6
:1049700010A9010815A90108D1AA0108D9AA01089E
:10498000E2AA0108E9AA0108EFAA0108049E0108A9
:104990002DE9F0430E4607469046D1B04FF49C7285
:1049A000002102A81D46589C12F021FC31463B46CE
:1049B000424602A8FFF7E2FD3678642E5AD01CD892
:1049C0003F2E44D008D82E2E4BD09DF808106A48B0
:1049D00006F0E0FC694A48E0612E00F09380622E08
:1049E000F3D1674806F0D6FC664806F0D3FC4FF4D6
:1049F00093716548FFF7C2F830E0722E45D00CD8AD
:104A0000672EE2D105A9614806F0C4FC33464F9AEF
:104A100021462846FFF71AFF20E0732E50D0772E4C
:104A2000D3D15B4806F0B6FC0399002900F0A180C1
:104A3000584813F09FFA0446002840F09A805648E0
:104A400006F0A8FC2146384600F0B8FECCE75348F3
:104A500006F0A0FC21462846FFF7E6FD51B0BDE870
:104A6000F0834F4806F096FC4E4A21462846FFF751
:104A700029FDF3E703994C4806F08CFC02AB3A465B
:104A800021462846FFF7EAFDE8E705A9474806F072
:104A900081FC0399464813F06DFA20B9384600F0BE
:104AA0001DF9444AE1E74F993846FFF71BFD08B16D
:104AB000414ADAE74F9808B1FFF782FB7223A6E775
:104AC00005A93E480DAA06F065FC4F993846FFF748
:104AD00009FD0028ECD14F9810B10DA9FFF7AAFCF1
:104AE00073234F9A21462846FFF7B0FE21683448C9
:104AF00006F050FC2868216806F0B2FC314806F048
:104B000049FCABE70DF134092F484A4605A906F0E8
:104B100041FC4F9830B3FFF7CCF8032801D02B4A63
:104B2000A3E74F98FFF70CF913F036FA08F10106E6
:104B300006442749304605F055FD074690B14F9889
:104B4000FFF7FEF8234A03463146CDF80090384679
:104B500013F0BCF939464F98FFF76CFC0121384639
:104B600005F044FD61234F9A21462846FFF7DCFCFF
:104B7000BCE7012167E700BFABAC0108CDAC010881
:104B80003DAC0108DEAC01080AAD0108A8AB010884
:104B900060AC010888AC01088EAC010882AB01084A
:104BA0008CAB010896AB010899AB0108B9AB0108C1
:104BB000409C0108CCAB0108CFAB0108E9AB010870
:104BC00002AC0108CBAC010813AC01082CAC010805
:104BD0003EE6010838AC01082DE9F0410C4680465C
:104BE0000D4815461E46069F06F0D4FB04B14DB98C
:104BF0000A4806F0CFFB39463046BDE8F041084A86
:104C0000FFF760BC069733462A4621464046BDE87A
:104C1000F041FFF7BDBE00BF53AD010868AD01080C
:104C20007BAD01087FB504460D4600680C49164669
:104C300000F000FB78B100F06FFC03AB009332464C
:104C4000294602ABFFF7C8FFDDE902122046FFF755
:104C500051FD04B070BD034806F09CFBF9E700BFAE
:104C6000DEAB010842AB010810B10C2105F0BEBC5F
:104C7000704710B1012105F0B9BC704730B513463B
:104C80000D460446AC4207D01BB194E8070083E808
:104C900007000C330C34F5E7184630BD10B5044658
:104CA00038B1FBF75FFA2046BDE81040282105F037
:104CB0009DBC10BD70B50446406AFFF7D5FFD4E92E
:104CC0000656AE4204D02846FBF74CFA2835F8E7E2
:104CD000A06908B1FFF7E2FF204670BDF8B50546B0
:104CE00000242826074FD5E906031B1ADB107B4357
:104CF0009C4205D206FB0400FFF762FA0134F2E79A
:104D0000F8BD00BFCDCCCCCCF8B50446224806F0A7
:104D100041FB224806F03EFBD4E90631994218D007
:104D2000C91A1F4EC91071431E4806F033FB0025F7
:104D30002827D4E906031B1ADB1073439D4205D2D2
:104D400007FB0500FFF708F80135F2E7164806F003
:104D500021FBD4E90931154EC91A89107143144851
:104D600006F018FB00250C27D4E909031B1A9B1039
:104D700073439D4205D207FB050000F071FF01352A
:104D8000F2E70C4806F006FB0B4806F003FBBDE813
:104D9000F8400A4806F0FEBA6AAE0108E9BF010809
:104DA000CDCCCCCC74AE010886AE0108ABAAAAAAC1
:104DB000BFAE0108CBAC0108CFAE01083DA301088E
:104DC0002DE9F043002487B006466846CDE900444B
:104DD000029405F033F9684605F0C8F94FF0280849
:104DE0002F4F304DD6E906239B1ADB107B439C42A4
:104DF0004ED208FB04F302EB0309D35C002B43D132
:104E00004846FEF754FF0146684605F0A1F94846BA
:104E1000FEF74FFF042837D8DFE800F03803101AF8
:104E200024004846FEF747FF0146684605F046F96C
:104E300050BBC2212846FEF7A1FE25E04846FEF7FA
:104E400072FF0146684605F01FF9E8B9C621F1E78F
:104E50004846FEF775FF0146684605F079F998B9AE
:104E6000CA21E7E7494603A8FEF733FFDDE903124D
:104E70006846521A05F044F918B9CF212846FEF7C2
:104E80007DFE0398FFF7F5FE0134ABE7D321D1E7B0
:104E9000684605F093F9029807B0BDE8F08300BFBB
:104EA000CDCCCCCCA2AD01082DE9F04305460E4691
:104EB00000244FF028081A4F8DB0D5E906239B1A1D
:104EC000DB107B439C4224D208FB04293146182284
:104ED000684613F07BF84846FEF7E9FE18220146C3
:104EE0000DEB020013F072F8684606F0B2FB68465C
:104EF00006F0C1FB06A806F0ACFB06A806F0BBFB5B
:104F0000182268460DEB020113F04EF818B1013477
:104F1000D3E74FF0000948460DB0BDE8F08300BF6D
:104F2000CDCCCCCC2DE9F04F06460F4600244FF0F7
:104F30000C09DFF86C808DB0D6E909535B1B9B1020
:104F400008FB03F39C4224D218223946684613F02A
:104F50003DF8182209FB04FB0DEB020055F80B107D
:104F600013F034F8684606F074FB684606F083FBDD
:104F700006A806F06EFB06A806F07DFB1822684620
:104F80000DEB020105EB0B0A13F00EF818B101341A
:104F9000D2E74FF0000A50460DB0BDE8F08F00BFD9
:104FA000ABAAAAAA10B51446FFF77EFF20B121468E
:104FB000BDE81040FFF73EBA10BD0000F8B50C4642
:104FC000064640F201120021224812F010F94FF477
:104FD000807221461F4812F0E6F81E491E4806F06E
:104FE000D9F91E491B4813F021F81C490546002039
:104FF00013F01CF8294607463046FFF755FFA0B9C5
:1050000029463046FFF78EFF044600B30168144876
:1050100006F0C0F9A3683846984701242046F8BD39
:105020003946104806F0B6F9F8E73A4629463046C0
:10503000FFF7B8FF04460028F2D00B4806F0AAF9A3
:105040000A4806F0A7F93046FFF75EFEE6E7294674
:105050000748E7E78C460020E8AE0108EDAA010802
:10506000EEAE010817AF010803AF0108CBAC010891
:1050700030AF010810B54FF4807204460649043081
:1050800005F054F9002805DD2046BDE8104002492E
:10509000FFF794BF10BD00BF8C45002038B5144603
:1050A0001D46FFF701FF28B12A462146BDE83840DA
:1050B000FEF7B8BF38BD10B51446FFF7F5FE20B1B6
:1050C0002146BDE81040FFF7F3B810BD10B51446F7
:1050D000FFF7EAFE10B12146FFF712F8002010BDDD
:1050E00038B514461D46FFF7DFFE28B12A46214693
:1050F000BDE83840FFF7B6B938BD00002DE9F047EC
:1051000000248CB0074603A8CDE90344059404F0BD
:1051100095FF214603A8009405F0ACF8014600284D
:1051200034D0214603A805F02EF840F2E7330446B8
:10513000009300263546DFF8F890009BB34273D900
:10514000214603A805F051F8824600286CD11823A7
:1051500021460DEB030203A804F0D8FF04442146C6
:1051600003A805F050F88046B0B10CAA214642F8D9
:1051700028AD03A804F068FF029A044406A9384643
:10518000FFF799FF00B101350136D6E76A4603A85B
:1051900005F000F80446CCE7214603A805F07DF8A9
:1051A00070B10CAA02F8288D214603A804F076FFFE
:1051B0009DF80820044406A93846FFF787FFE1E779
:1051C000214603A805F03AF8804668B102AB01AA6F
:1051D000214603A804F0ABFFDDE90123044406A93E
:1051E0003846FFF75BFFCDE7214603A805F018F826
:1051F00090B10CAB43F8288D01AA214603A8CDF845
:10520000048004F06CFF9DF808300444019A06A95C
:105210003846FFF765FFB5E7039B4846195D01F087
:10522000E00106F0B7F8AFE728460CB0BDE8F0871C
:10523000F9AD010808B5FFF737FE18B1BDE8084021
:10524000FEF739BD08BD10B5044608461146FFF704
:105250002BFE014620B9C4E90000A060204610BD25
:105260002046FEF736FDF9E708B5FFF71DFE18B139
:10527000BDE80840FEF757BD08BD08B5FFF714FEAE
:1052800018B1BDE80840FEF75BBD08BD037810B556
:10529000044643B1044806F07DF80021204600F0A2
:1052A0008DFA0023237010BDE4AD0108002370B512
:1052B000D1E90025AD1A0446C0E9003383600E46EB
:1052C000284601D006F002F9C4E900000544A560B3
:1052D000D6E90053024629468B4205D00AB10E7822
:1052E000167001310132F7E75B1B184460602046FD
:1052F00070BD38B504460D460B78103000F8103CF0
:105300004B68103140F80C3C51F8083C40F8083C20
:1053100051F8043C40F8043CFFF7C8FF05F11C01BC
:1053200004F11C00FFF7C2FF204638BD2DE9F84309
:10533000D0E90054641B9146A2101F4C064654430A
:10534000B4F5705F0F4602D11C4805F00FF9002C30
:1053500014BF22460122A418A1EB050526D2B4F5FC
:10536000705F23D82CB30C20604306F0AFF8804662
:1053700018EB05031CBF99E8070083E807004246C5
:1053800039463068FFF77AFC716800F10C02384644
:10539000FFF774FC05463068FFF766FC0C2303FB3F
:1053A0000484C6E90085B460BDE8F8834FF4705406
:1053B000D9E7A046DCE700BFABAAAAAACEA801089D
:1053C0002DE9F043054685B008460C4617461E46B3
:1053D00012F0E2FD172803D982212D48FEF7CEFBFB
:1053E000CDE90147D5E9097803962A4AA8EB0706D3
:1053F000B41054430134B4F5705F02D9264805F067
:10540000B5F8EB6ADB1B9B1053439C4215D94FF058
:105410000C0909FB04F91CB1484606F057F804468C
:10542000224641463846FFF729FC686AFFF71CFC14
:1054300026446C624C44AE62EC62EA6AD5E9090328
:1054400014491B1A9B10121A4B4392104A43013302
:10545000934206D9114805F09DFF8C210C48FEF7B8
:105460008DFBD5E90A3293420AD023B104AA12E98E
:10547000070083E807000C33AB6205B0BDE8F0839A
:1054800001AA194605F12400FFF750FFF5E700BF18
:10549000A2AD0108ABAAAAAA93A8010887AD01088A
:1054A000002310B504460370C0E90633C0E9083391
:1054B000C0E90A33C0E90C33064B80214361043054
:1054C00004F0F9FE2046044B044A0549FFF778FF33
:1054D000204610BD0C4500201D55000853AF0108A3
:1054E0005FAF010810B5084C2368DB0709D40748F3
:1054F000FFF7D6FF0123064A06490448236010F04F
:1055000006FA024810BD00BF084500209047002061
:1055100000000020B54C0008FFF7E4BF08B5FFF716
:10552000E1FFBDE80840FFF7EFBB0022C0E9002221
:10553000826010B50C6804600A6042684C68446080
:105540004A6082688C6884608A6010BD70B50E46BF
:1055500005461446B54217D09CB12B7805F11001D1
:1055600023706B6804F110006360AB68A360EB68A4
:10557000E360FFF7DAFF05F11C0104F11C00FFF7FF
:10558000D4FF28342835E5E7204670BD2DE9F843DF
:10559000D0E90064A41BE310234C05465C43B4F53A
:1055A000705F0F46914602D1204804F0DFFF002CC7
:1055B00014BF23460123E418A1EB060623D2B4F559
:1055C000705F20D814B32820604305F07FFF804629
:1055D00018EB060002D04946FFF78BFE39464246DB
:1055E0002868FFF7B3FF696800F128023846FFF723
:1055F000ADFFD5E900690746B14509D03046FAF755
:10560000B1FD2836F8E74FF47054DCE7A046DFE739
:10561000286808B1FFF742FB282303FB0484C5E98F
:105620000087AC60BDE8F883CDCCCCCCCEA8010817
:105630002DE9F047D0E9065704460E46DFF80C8105
:105640008AB0AF421BD029466846FFF752FE684633
:10565000FEF72DFB81463046FEF729FB0146484602
:1056600006F038F830B13046FEF721FB01464046DF
:1056700005F090FE6846FAF775FD2835E1E7D4E9B4
:1056800006892E4AA9EB0807FD1055430135B5F5EB
:10569000705F02D92A4804F069FF236AA3EB08036C
:1056A000DB1053439D4220D94FF0280A0AFB05FA2C
:1056B0001DB1504605F00AFF0546494640462A46B8
:1056C000FFF744FFD4E90689C14505D04046FAF703
:1056D00049FD08F12808F7E7A06908B1FFF7DEFAED
:1056E0002F44A5615544E7612562226AD4E9060387
:1056F00012491B1ADB10121A4B43D2104A430133D2
:10570000934206D90F4805F045FE77210E48FEF773
:1057100035FAD4E90703984209D010B13146FFF7B2
:10572000E8FDE3692833E3610AB0BDE8F08701468C
:10573000324604F11800FFF729FFF5E7CDCCCCCCB9
:1057400093A801084BAE0108A2AD010819AE0108EB
:10575000002313B502A941F8043D094B0422D3E903
:105760000140084B20445B689847044628B106482E
:1057700005F010FE204602B010BD0448F8E700BF57
:10578000DC470020CC470020C5B10108D9B1010891
:1057900008B5084805F0FEFDFFF7A4FEFFF79EFAE6
:1057A000054805F0F7FDFFF79DFEBDE80840FFF74F
:1057B000ABBA00BFF6B101080EB2010873B50546D9
:1057C0004FF400700C4605F081FE064630B92148C2
:1057D00005F0E0FD20212048FEF7D0F94FF40072DB
:1057E0000021304611F003FD314628464FF4007287
:1057F000FFF7E6FA194D014601902CB3184805F061
:10580000C9FDD5E901431C44164DEB681BB1019954
:105810002046083198476B68042210492046984773
:1058200004226B680DEB0201A01898476B68019A7F
:10583000314604F1080098470B4805F0ABFD3046AF
:1058400005F02EFE02B070BD084805F0A3FD6C689F
:10585000DAE700BF5CB0010867B00108DC47002050
:10586000B7B00108CC470020F1B00108D6B001085C
:105870002DE9F74FFFF736FE2F4F06462F4805F06C
:1058800089FDB846DFF8D090DFF8D0A0FCF740FFE4
:105890002B4D38602B68AB462A4C002B37D003F5D4
:1058A0006A436033984232D223782BB9264805F0F8
:1058B00071FD264805F06EFD012330462370FFF789
:1058C000D9FB41F2883352464FF0FF310020FDF7FB
:1058D00067FB0190FCF71CFF019BC8F8000023B98F
:1058E000237813B13046FFF7C5FBDAF80030DA074A
:1058F00044BFD8F800202A609B07C7D50023CBF807
:105900000030D9F80830002BBED09847BCE7237888
:105910006BB100213046FFF751FF0D4805F03AFD0D
:105920000C4805F037FDD9F8083003B1984700233B
:1059300023702B60C5E700BFF447002035B1010894
:10594000F0470020E84700204AB101086DB1010886
:1059500090B10108A2B10108CC470020EC4700201B
:1059600010B5FFF7BFFD04460021FFF727FF2046D3
:10597000FFF7CAF9BDE810400348002301220221C5
:105980000068FDF751BB00BFC847002010B5FFF706
:10599000A9FD04460021FFF711FF2046BDE8104095
:1059A000FFF7B2B92DE9F743194E074688467568E7
:1059B0000AB1B3681D440024DFF8609002A941F8E1
:1059C000084D0422D9F800302846984732680099DB
:1059D0008A4204D00F4805F0DDFC204614E0042282
:1059E000D9F800300DEB0201A818984701990A4830
:1059F00005F0D0FC019A4245EFD8D9F8003039467D
:105A000005F108009847019803B0BDE8F08300BF96
:105A1000DC47002000B101081BB10108CC47002081
:105A2000F0B589B002AC84E80F00039B23B940F2C3
:105A300021117648FEF7A2F8029B23B94FF4917129
:105A40007248FEF79BF894E80F00714D714C85E8A1
:105A50000F000EAB93E8070084E8070012B94FF47B
:105A60008063A360236823B940F22D116748FEF7D5
:105A700085F82368013304D140F22F116348FEF703
:105A80007DF8FFF72FFD0646634B644A6449FFF734
:105A900097FC644B644A65493046FFF791FC644BC0
:105AA000644A65493046FFF78BFC4FF4007005F0FF
:105AB0000DFD0746002870D04FF40072002111F050
:105AC00096FBD4E901032D68042207A91844A847CE
:105AD000002856D02268079B9A4252D1574805F0B9
:105AE00059FC01224FF400713846FFF75BFF044672
:105AF000534805F04FFCFFF72BFE002C3DD001234F
:105B00003370224639463046FFF7F8FA384605F03A
:105B1000C7FC3478FCB94FF4007005F0D7FC05469B
:105B20004FF40072214611F062FB22464FF40071DF
:105B30002846FFF737FF074600283CD105F0B0FCA8
:105B4000284605F0ADFC3F4805F024FCFFF7CAFCF1
:105B50000021FFF733FE3C4BFA22019301233B491E
:105B600000933B480023FCF7B1FB20B94FF4A4712C
:105B70002648FEF703F809B0F0BD364805F00AFCE8
:105B8000347000224FF400713846FFF70BFF0446D3
:105B90000028B6D1384605F083FC2F4805F0FAFB03
:105BA0003046FFF79BF800233370FFF7D1FD2B48F9
:105BB00005F0F0FBADE74FF4007005F087FC0446FC
:105BC00018B987211148FDF7D9FF4FF40072002161
:105BD000204611F00CFB4FF4007221463046FFF7CF
:105BE000EFF808B92046A9E78742FBD10023E15C22
:105BF000EA5C9142F6D101339F42F8D1204605F08C
:105C00004FFC284605F04CFCA5E700BF67B0010833
:105C1000CC470020DC4700208D59000863AF010805
:105C20006FAF01089157000874AF01088FAF0108EA
:105C30006159000897AF0108AFAF0108B4AF010880
:105C4000D8AF01083AB00108C847002051B0010898
:105C500071580008EDAF010816B001080EB2010836
:105C600010B504460168074805F094FB616831B13E
:105C70000B7823B10448BDE8104005F08BBB034806
:105C8000F9E700BF26B2010851A90108CBAC010811
:105C900010B50446C06908B105F002FC206908B1DE
:105CA00005F0FEFB606808B105F0FAFB204610BD68
:105CB00010B504460068FCF729FA204610BD000024
:105CC0001FB50B46546801780294127801925A6805
:105CD000009242681B68024805F05CFB04B010BDEE
:105CE0002BB20108C9210148FDF748BF49B201089C
:105CF000FE2307B502A901F8043D054B18680023EF
:105D000000681A46FBF7F2FE03B05DF804FB00BF23
:105D100004480020D0B51F467423C0E90031002399
:105D2000044683600820164604F03EFCC0E9006784
:105D3000A0602046D0BD00002DE9D043DDE9066714
:105D400099467223C0E9003100239642836077EBC5
:105D500009030446904603DA2B210748FDF70EFF9E
:105D6000102004F021FCC0E90089C0E90267A060AE
:105D70002046BDE8D08300BF93B20108036837B561
:105D8000632B04460D4601D0FFF7ACFF002302AAA7
:105D900042F8043DA168284605F0E2F8019B1BB1DA
:105DA00038210248FDF7EAFE03B030BD93B2010886
:105DB00070B563230025C0E90031044685601A20D0
:105DC000164604F0F1FB1A22294611F010FA31466A
:105DD000A0602046FFF7D2FF204670BD8164704767
:105DE000C16470472DE9F843D0E901738846002566
:105DF0004FF00C09DB1B0A4E9B105E43ECB2B44221
:105E00000BD209FB04724146506812F0B3F8013519
:105E10000028F3D12046BDE8F8834FF0FF30FAE7C1
:105E2000ABAAAAAA2DE9F843D0E904738846002555
:105E30004FF00C09DB1B0A4E9B105E43ECB2B442E0
:105E40000BD209FB04724146506812F093F80135F9
:105E50000028F3D12046BDE8F8834FF0FF30FAE781
:105E6000ABAAAAAA2DE9F0410E4649680446FFF7FD
:105E7000B9FFC0B2FF2803D07C212948FDF77EFE80
:105E8000D4E90123274F9B1A9B107B437E2B03D918
:105E90007F212348FDF772FED4E901120C25E0684A
:105EA000531A9B10121A7B4392107A430133934288
:105EB00005FB03F80ED84144A160D4E9013496E80B
:105EC0000700E31A04E9070016489B1058430138FD
:105ED000BDE8F081404605F0F9FA054618B9692198
:105EE0001148FDF74BFED4E901C30027A3EB0C03D7
:105EF0009A100C4B5343002B09DD05EB070E0CEBFE
:105F0000070207CA013B8EE807000C37F3E760463B
:105F100005F0C6FA65604544C4E90255CDE700BF07
:105F200093B20108ABAAAAAA38A601081FB56E232E
:105F3000CDE90131002301A90393FFF793FF05B0D9
:105F40005DF804FBFF2270B5002380F828204FF095
:105F500000424FF0FF31C0E90D23C2636FF07F4272
:105F6000C0E910120522254DC0E914232A68044611
:105F700012F00102C0E90033C0E90233C0E9043382
:105F8000C0E90633C0E908330363C0E9123313D113
:105F900001211B4E084632607160FBF7CDFC30607A
:105FA00018B912211748FDF7E9FD0123164A1749D0
:105FB00013482B600FF0ABFC154B1A680AB9104A56
:105FC0001A6014492046FFF7B1FF134B13491870AC
:105FD0002046FFF7ABFF124B124918702046FFF71F
:105FE000A5FF114B114918702046FFF79FFFFE22B5
:105FF0000F4B18700F4B20461A7070BD00480020E0
:10600000784800207F9E010800000020B15C000855
:1060100004480020AAB301080C480020B2B30108CC
:106020000A480020BAB3010808480020BFB301089D
:106030000B4800200948002010B5084C2368DB07F6
:1060400009D40748FFF77EFF0123064A06490448A2
:1060500023600FF05CFC024810BD00BFFC4700202D
:106060002048002000000020915C00082DE9F0414C
:106070000E4649680446FFF7D5FEC0B2FF2803D09C
:1060800087212948FDF77AFDD4E90423274F9B1A7D
:106090009B107B437E2B03D98A212348FDF76EFD9D
:1060A000D4E904120C25A069531A9B10121A7B43E1
:1060B00092107A430133934205FB03F80ED8414412
:1060C0006161D4E9043496E80700E31A04E90700A3
:1060D00016489B1058430138BDE8F081404605F052
:1060E000F5F9054618B969211148FDF747FDD4E9CE
:1060F00004C30027A3EB0C039A100C4B5343002B53
:1061000009DD05EB070E0CEB070207CA013B8EE821
:1061100007000C37F3E7604605F0C2F925614544F6
:10612000C4E90555CDE700BF93B20108ABAAAAAAFE
:1061300038A6010838B5D0E901239B1A074A9B10FD
:106140005343CDB29D42044603D3A6210448FDF734
:1061500015FD0C20636800FB053038BDABAAAAAA68
:1061600093B2010838B5CCB2114905460B6813F05B
:10617000010307D10F4A70201372012310600E48EB
:106180000B605060FF2C10D0D5E904239B1A0B4AFA
:106190009B1053439C4203D3B2210948FDF7EEFC08
:1061A0000C23286903FB040038BD0248FCE700BF4C
:1061B000F847002010480020DDB20108ABAAAAAAC7
:1061C00093B2010810B5D0E90730C9B2D2B2834208
:1061D00009D01C788C4204D15C78944201D1987823
:1061E00010BD0333F3E74FF0FF30F9E72DE9F0413D
:1061F000D0E904239B1A4F4A9B1053430D4609785C
:106200000446994203D393214B48FDF7B7FCD4E9E8
:1062100001239B1A474A9B1053436978994203D341
:1062200094214548FDF7AAFCD4E904239B1A414A6E
:106230009B105343A978994205D3FE2903D0952199
:106240003D48FDF79BFC6A7829782046FFF7BAFFA6
:10625000C3B2FF2B064629D029782046FFF782FFDC
:10626000697807462046FFF765FF3146804620469D
:10627000FFF778FF414602463846FFF721FD2978AF
:106280002046FFF76FFF697806462046FFF752FF6A
:10629000A97807462046FFF765FF39460246304693
:1062A000FFF70EFD9C212448FDF768FCD4E9072385
:1062B000204F9B1A7B437E2B03D99F211E48FDF75D
:1062C0005DFCD4E90762616A931B7B43521A574312
:1062D0000133BB4203EB43080AD8464426622A88AE
:1062E000236A23F8032CAA7803F8012CBDE8F08177
:1062F000404605F0EBF8064618B969210F48FDF74E
:106300003DFCD4E90702131A0A4A5A430023002A23
:106310000ADDC118B1F800C0F71826F803C0897863
:10632000013AB9700333F2E705F0BAF8E661464482
:106330006662D3E7ABAAAAAA93B2010838A60108FD
:1063400013B5FF24084A02AB106803F8044D0A464F
:1063500000681946FBF76EFC012814BF20469DF823
:10636000040002B010BD00BF0448002038B58168A9
:1063700000681D46144605F05FF90346201845EBFA
:10638000E37138BD08682DE9F04172281F461FD01F
:1063900074280FD0632820D1886804F0A1FE00285B
:1063A00071F1000304460D460EDADD210D48FDF7BC
:1063B000E5FB09E08B68D3E90045B5F1004F08BF64
:1063C000002C01D0A4187D4120462946BDE8F0816B
:1063D0008868BDE8F041FFF7C9BF00244FF00045D1
:1063E000F2E700BF93B201082DE9F0410F460646DF
:1063F0000024FFB2FFF7B6FED6E90758454511D095
:106400002B78BB420CD169783046FFF793FE0368C6
:10641000692B05D183681B6803B198470134E4B246
:106420000335EBE72046BDE8F0812DE9F3418046D6
:106430000F460025FFF796FED8F81C40D8F82060DC
:1064400003340336FFB2A6421BD0234633F8032D94
:106450009B78ADF804208DF8063014F8033C9F4279
:106460000DD19DF805104046FFF764FE0368692BC7
:1064700005D183685B6803B198470135EDB20334F9
:10648000E1E7284602B0BDE8F0810000836C73B5F7
:1064900004460D46164623B94FF48C710B48FDF7A0
:1064A0006DFBCDE9006423462A4609490948FBF7FC
:1064B0000DFF012807D04FF48F71044802B0BDE8EA
:1064C0007040FDF75BBB02B070BD00BF93B2010826
:1064D0009FB30108256A000838B590F84730044694
:1064E000032B0D4604D940F231110648FDF746FB57
:1064F00094F847305A1C84F847201C4484F84250D2
:1065000038BD00BF93B2010810B590F8473004467B
:1065100023B94FF49B710648FDF730FB94F84730E0
:10652000013BDBB284F847301C4494F8420010BDB4
:1065300093B20108CBB2FE2B10B504460AD0FFF788
:1065400011FE03686D2B05D1017A2046BDE810408D
:10655000FFF708BE10BD00002DE9F84304460026F1
:10656000114FD4E904239B1A9B107B435FFA86F8F2
:10657000434516D941462046FFF7DCFFD4E90759C9
:10658000A9450CD02B78434507D169782046FFF701
:10659000D1FDA9782046FFF7CDFF0335F0E701369E
:1065A000DFE7BDE8F88300BFABAAAAAA38B5054665
:1065B000002495F84730A34207DD2B1993F84210C9
:1065C0002846FFF7CFFD0134F3E738BD00232DE95E
:1065D000F74FC0E9043388461946D8E907594FF008
:1065E00000430446C0E90213C0E90013FF208A46B5
:1065F0009B46D2B2207401924D45D4E900671FD06A
:106600002B78019A934219D169784046FFF792FDA1
:10661000DDE90C2301464046FFF7B4FE594508BFAB
:1066200050450BD05F4508BF564503D0B04271EBD3
:10663000070303DA6B78C4E9000123740335DBE751
:10664000B7F1004F08BF002E08D0DDE90C23B21AC5
:1066500067EB030316461F46C4E90267204603B0F2
:10666000BDE8F08FF8B50D460B4B896806464B43E5
:106670004FF47A71B3FBF1F1FFF762FE0446C7B243
:10668000B06C03681B689847FF2FC6E90E010CBF6A
:10669000287C2046F8BD00BF40420F0038B5C36CCF
:1066A00004460D461BB9BDE83840FFF7DBBF806CE0
:1066B000134903685B699847A06C0368DB689847D7
:1066C000A06C03689968D5E900238847A06C03682B
:1066D0001B699847E36C9847A06C0368DB68984790
:1066E000A06C03681B689847C4E90E01002120468E
:1066F000FFF726FEC0B2FE2808BF287C38BD00BFC9
:10670000F15C0008F8B5D1E90067B7F1004F08BFA8
:10671000002E05460C4608D11AB1BDE8F840FFF737
:10672000A1BFBDE8F840FFF7B9BFD1E90267012E6C
:1067300077F1000301DA087CF8BD8AB121462846CA
:10674000FFF790FF237CC0B28342F5D1D5E90E67F5
:10675000D4E90023964277EB0303B8BFFF20EBE7B1
:10676000D0E91423964277EB0303E7DBFFF796FFAC
:10677000E8E700002DE9F04389B004460D46FFF735
:10678000F1FC03680646702B04D04FF49E713C4820
:10679000FDF7F4F9A06C03681B6898472A46C4E922
:1067A0000C01CDE90001214602A8FFF70FFF2946A1
:1067B0002046FFF719FE9DF818300746FF2B05D13C
:1067C00020B940F247112E48FDF7D8F9D4E90C0161
:1067D00004F060FD01462B4804F0DCFD39462A48F0
:1067E00004F0D8FD9DF81810FF2920D100224FF0A9
:1067F0000043CDE90423254F327A02A92046FFF752
:1068000081FFC3B2FF2B804632D1D4E90E23DDE9EC
:106810000201801A61EB030189468046CDE90489B3
:1068200004F04EFD0146384604F0B4FDE4E720468E
:10683000FFF780FCD0E90078DDE9020104F02AFDD1
:10684000424603463946124804F0A4FDD4E90C231D
:10685000DDE90201801A61EB030188460746CDE9B4
:10686000047804F02DFD01460A4804F093FDC2E7C8
:1068700029462046FFF7D9FD404609B0BDE8F08320
:1068800093B20108EBB201080AB3010867B301082B
:1068900025B3010849B3010870B504460D46FFF75A
:1068A00061FC03686D2B11D0702B09D0612B14D1C2
:1068B000836894F8411094F84000BDE87040184790
:1068C00029462046BDE87040FFF754BF034840F218
:1068D0002B11FDF753F94FF0FF3070BD93B2010853
:1068E0002DE9F04790F828300446FF2B04D14FF4EF
:1068F000D6714848FDF742F994F828102046FFF772
:1069000031FC94F82830DFF8188184F8463094F888
:1069100046102046FFF726FC036805466D2B2046EF
:1069200094F846100BD1FFF7D7FD297A204684F85A
:106930004610FFF717FC2046FFF738FEE7E7FFF7A2
:10694000ABFFC3B2FF2B06460BD140F2C111314859
:10695000FDF714F940F2C1112F4B304A2D4810F0C9
:10696000CFFA024694F846102046FFF72BFCC5B23A
:10697000FF2D09D140F2C7112648FDF7FFF8264B3D
:10698000264A40F2C711E9E794F84610FE2D20464A
:1069900021D1FFF7B9FD074601462046FFF7E2FB8C
:1069A000324639462046FFF70DFCC5B2FF2D0DD10A
:1069B00031462046FFF7BEFB40F2D3111548FDF7E4
:1069C000DDF8154B154A40F2D311C7E72046FFF713
:1069D000EDFD3946DAE7FFF7C5FB314607462046AD
:1069E000FFF7A8FB294681462046FFF7BBFB8246FE
:1069F000404604F0CFFC524649463846FFF760F95E
:106A000094F8463084F8416084F8403084F8465069
:106A10007DE700BF93B2010815A90108C7B30108BB
:106A20008FB3010808B5FFF707FBFFF759FFD0B593
:106A30001F461646FFF77EFB03688468742B01D05F
:106A4000FFF750F9C4E90067D0BDD0B5044616463B
:106A50001F46FFF76FFB32463B4601462046BDE826
:106A6000D040FFF78FBC0000836C10B5044623B9FB
:106A70004FF41F710248FDF781F8A06C10BD00BFF4
:106A800093B20108FF23054A1370054A1370054AA3
:106A90001370054A1370054A137070470C480020A4
:106AA0000A480020084800200B4800200948002020
:106AB000014B1878704700BF0848002010B5044605
:106AC0000068FBF723FB204610BD00002DE9FF48BE
:106AD00005F040FE4FF6FF712E4A2F4C13888B4273
:106AE0001CBF01331380FFF7A7FAFFF7BDFF036850
:106AF0001B689847637806460F4603BB274BDB8825
:106B0000EBB1274AD2E900BCBCF1004F08BFBBF192
:106B1000000F0FD083457CEB010210DA214AB0EB65
:106B20000B0002FB03F261EB0C01D317904271EBF7
:106B3000030304DB1C4804F02DFC012363700023D5
:106B4000ADF80C3063782BB101238DF80C30144B69
:106B5000C3E900672378154CBBB1012514488DF8B3
:106B60000D5004F017FC2570124B13481A78134B84
:106B70001978002300930068039B05F02DFF30B1C6
:106B80000F4B187804B0BDE8F0882370ECE70D4B8C
:106B9000F7E700BFC2480020A4480020B04800200A
:106BA00068000020805101000CB50108AD480020AC
:106BB00035B50108A7480020A0480020A6480020BD
:106BC000084800200A4800201D4B10B5DB882BB96F
:106BD0001C4804F0DFFB1C4B187810BD1B4BD3E99D
:106BE0000023B3F1004F08BF002A01D01848F0E796
:106BF000184C23780133DBB2032B237001D91648DC
:106C0000E7E7012B0BD90A21002004F015FD134BF7
:106C100058434FF47A73B0FBF3F0FBF7CBFE2178C7
:106C20000F4804F0B7FB00230E4A13700E4A13708E
:106C30000E4A13600E4A1370012353700D4BCBE7BD
:106C4000B04800204AB50108084800206000002034
:106C500066B50108D848002080B5010840420F0001
:106C600097B50108A7480020A6480020A0480020AA
:106C7000A44800200B48002008B500231A46FAF764
:106C800035FF431E5842584108BD000007B50B7838
:106C9000012B12D005D3022B13D00C4804F07AFB41
:106CA00008E0002302A941F8043D094B1B6818685D
:106CB000FFF7E2FF03B05DF804FB02A94FF0FF33DA
:106CC000F1E7034B04311B68F1E700BFFDB5010894
:106CD000904800201FB57023CDE90131002301A9A0
:106CE0008DF80C30FFF7C2F905B05DF804FB000029
:106CF0002DE9F04F474B85B01A780446002A40F042
:106D00008580012744491F70FFF710F9434B444920
:106D100018702046FFF70AF9DFF854A141498AF8B4
:106D200000002046FFF702F9DFF848910A2200230D
:106D300089F800003C4901A8FEF7ECFF01A92046B4
:106D4000FFF790F8394E3A4930702046FFF7EEF8D9
:106D5000384B394918702046FFF7E8F8374B384967
:106D600018702046FFF7E2F8364B374A187037495B
:106D70002046F9F7B7FDDFF800B1354A8BF800007F
:106D800034492046F9F7AEFD334905462046FFF762
:106D9000A1FF70230193314B804601A92046029345
:106DA0008DF80C70FFF762F907462D4A2B461278D2
:106DB0009BF800102046F9F7A0FD43469AF8002002
:106DC00029462046F9F799FD3B4699F800202946C7
:106DD0002046F9F792FD2B46327841462046F9F7D6
:106DE0008CFD2B46327839462046F9F786FD1D4A40
:106DF0002B46127829462046F9F77FFD1A4B1B4A8D
:106E00001B78127829462046F9F777FD05B0BDE8D2
:106E1000F08F00BFD948002053B70108A8480020D0
:106E20005DB7010868B7010874B7010889480020F8
:106E300081B70108C04800208DB70108C448002070
:106E40009AB70108C5480020CD6A0008A8B7010814
:106E5000397C0008B2B70108C6B70108D9B70108E4
:106E6000084800200B480020094800200C4800205A
:106E7000AC48002088480020AA48002008B505F04A
:106E800047FC18B1BDE8084005F064BC08BD00002F
:106E900030B5044685B00D46FFF72AFF6D22064B3C
:106EA00001A91B782046CDE901258DF80C30FFF7AC
:106EB000DDF805B030BD00BFAA4800202DE9F84F2D
:106EC000424B434D1A68044612F0010F01BFFF22E6
:106ED0002A7001221A602B78FF2B73D1FFF708FF6D
:106EE0003C4A3D492046F9F7FDFC3C4A28703C49A4
:106EF0002046F9F7F7FC3B4F3B4A38703B492046A8
:106F0000F9F7F0FC3A4E3B4930702046FFF7C0FFDE
:106F1000394982462046FFF7DDFE38498346204640
:106F2000FFF7D8FE8146364A3B781278297820460A
:106F3000F9F7E3FC334ADFF8E080337812782978F8
:106F40002046F9F7DAFC337898F8002039782046A3
:106F5000F9F7D3FC2B7898F8002031782046F9F720
:106F6000CCFC294A5B46127839782046F9F7C5FCF3
:106F700026493B780A7820465946F9F7BEFC244A50
:106F80004B46127839782046F9F7B7FC1F493B7811
:106F90000A7820464946F9F7B0FC1A4A5346127857
:106FA00031782046F9F7A9FC337898F8002051464B
:106FB0002046F9F7A2FC174A2B7812783178204640
:106FC000F9F79BFC2878BDE8F88F00BF84480020C3
:106FD000DB480020A1760008E9B801080572000826
:106FE000F3B80108A9480020C96B0008FDB80108E2
:106FF000AB48002007B9010813B9010821B90108FD
:10700000A84800200B480020AC48002089480020F8
:107010000A480020084800200C48002038B50446E3
:107020000D46FFF765FE034A29462046F9F75AFC4C
:1070300038BD00BF71740008344B2DE9F04F1A8938
:107040000023044689B0CDE90023039100230022E8
:107050002F4905A8FEF770FE05A92046FEF702FF9E
:107060002C4982462046FFF735FE2B4983462046B1
:10707000FFF7D4FF294A804629492046F9F732FC18
:10708000284A054628492046F9F72CFC0646274F92
:10709000DFF8A8903B7899F8002029462046F9F7B8
:1070A0002CFC234A5B46294620461278F9F725FC3A
:1070B000204A4346294620461278F9F71EFC3346FB
:1070C000524659462046F9F718FC33465246414687
:1070D0002046F9F712FC184A3B78414620461278C0
:1070E000F9F70BFC3B7899F8002031462046F9F778
:1070F00004FC6D230593039B05A9204606938DF898
:107100001C50FEF7B3FF09B0BDE8F08FB048002077
:1071100030B901083DB901084DB90108C17700082F
:107120005EB90108B16A00086DB90108094800207C
:10713000C4480020C5480020C1480020084800205D
:107140002DE9FF4790468A461E4A1F490446F9F733
:10715000C9FB1E4905462046FFF7BCFD1C49814678
:107160002046FFF75BFF06461A4A4B462946204653
:107170001278F9F7C2FB184A184F334629462046C1
:107180001278F9F7BAFB3B78424649462046F9F7B0
:10719000B4FB3B78424631462046F9F7AEFB104A35
:1071A0003B78127831462046F9F7A7FB6D2301A9F9
:1071B0002046CDE9013A8DF80C50FEF757FF04B098
:1071C000BDE8F087E5770008BEB80108C8B8010837
:1071D000D8B80108C4480020C5480020094800204C
:1071E000C148002070B50D460446FEF725FF04494E
:1071F00022462B46BDE870400978FFF718BC00BF57
:1072000089480020F7B55E4C2668A6B9082003F02F
:10721000CBF9054606600120324668600421FAF782
:107220008BFB286018B912215648FCF7A7FC56487A
:10723000256005F0A5FA554D554F2968554801318F
:10724000296004F0A7F805F085FA3B781BB9012303
:107250003B7005F0ABFA002302A941F8043D236816
:107260004D4A1868FAF7E6FC012807D04B4804F0AD
:1072700091F840F28D114A48FCF780FC019E731C86
:1072800051D1484804F086F82B68042B0FD9FEF73B
:1072900043F903785BB1444804F07CF84FF47A700A
:1072A000FBF788FB4FF4CC713D48FCF767FC0023EB
:1072B0003B702B681E22013BDBB21E2B28BF1E2316
:1072C00002FA03F3394A934226D8B3F5616F1E469A
:1072D0004FF0000722D2B3F5167F77F1000320DAD2
:1072E0003C2E77F10003ACBF1E210A21002004F0E0
:1072F000A3F9341847EBE0752946204603F0E0FF78
:1073000001462B4804F046F820462946FFF76AFF5D
:10731000284B187803B0F0BD0027244E4FF41671A7
:10732000E4E73C21E2E74EB13146234804F032F86D
:1073300001980021FFF756FF204BEAE720482E6016
:1073400004F028F805F0C0F9FEF776FEFFF78CFB95
:1073500003681B6898471B4BC3E9000123686BB1A6
:10736000304605F00DFA256835B12868FAF7CEFEEB
:107370000821284603F03AF900232360124BC8E79E
:10738000904800207F9E01088D6C0008D4480020A2
:10739000D0480020ECB30108A0860100FFB301082B
:1073A00019B401086DB4010884B4010800A30200F7
:1073B000D1B401080A480020E7B40108AC48002015
:1073C000FCB40108580000200C480020054B187040
:1073D000054B1A700022054B1960054B1A705A7044
:1073E000704700BFA7480020A6480020A048002002
:1073F000A4480020027901684079FFF7E7BF08B58B
:1074000005F0E2FAC0B2DE2828BFDE2008BD000089
:107410004FF47A7337B5002403FB00F2074802A942
:10742000056841F8044DB2FBF3F22868FAF702FC54
:10743000012814BF2046019803B030BD8C480020BD
:107440004FF47A7337B5002403FB00F2074802A912
:10745000056841F8044DB2FBF3F22868FAF72CFDF9
:10746000012814BF2046019803B030BD8C4800208D
:107470002DE9F04F8FB0FEF7DFFD4FF00009064613
:1074800090F846B0FFF7FAFCDFF8C4A0DFF8C4803C
:10749000B06C02AD036808AC1B6898475A46CDE94A
:1074A0000001314608A8FFF791F80FCC0FC5DDE9C0
:1074B00008012368B1F1004F08BF00282B70DDE9F7
:1074C0000A4516D11C4803F065FF002501271B4C17
:1074D0004FF47A73A4FB030103FB0511FFF7B0FF20
:1074E00010B30122164B5A72164B18780FB0BDE834
:1074F000F08F03F0CFFE29460746204603F0E0FE5A
:1075000039460246504603F045FFA04579EB050396
:1075100008DA0021094803F0D3FE01460A4803F0C7
:1075200039FFD2E70027D3E71FB1084803F032FF45
:10753000AEE79DF81800D9E785B601088051010033
:1075400094480020C1480020BFB60108D8B6010801
:107550009DB6010885510100022818BF002005F0E2
:10756000B1BB0000F8B53B4B05461E78002E6FD12D
:1075700001271F7004F0C0FD37492846FDF774FE4F
:10758000C31F052B354C42D820710E2334492846A1
:107590006371FDF772FE3349074610F0EBFC0028DB
:1075A0003AD1E06030492846FDF744FE2F4960702B
:1075B0002846FDF759FEB0F57A7F3AD8E0802C498D
:1075C0002846FDF751FE42F21073984236D82081CA
:1075D00028492846FDF72EFE2749A0702846FDF7CA
:1075E00043FEB0F57A7F2ED2608124492846FDF70C
:1075F00021FEE07036B1224803F0CCFE7121214813
:10760000FCF7BCFAE068BDE8F840FFF7A5BF1E48EC
:1076100003F0C0FE3E46B8E71C49384610F0AAFC0D
:1076200010B90223E360BDE7194803F0B3FE012659
:10763000B8E7184803F0AEFE0126C0E7164803F08D
:10764000A9FE0126C4E7154803F0A4FE0126CCE7F5
:10765000F8BD00BFDA480020EDB70108B0480020AF
:1076600006B80108A9B8010829B801082DB8010811
:1076700054B80108DEAB01087CB80108A6B80108BF
:10768000ABB8010819B40108F0B70108CAD0010865
:107690000DB8010836B801085DB8010887B80108BF
:1076A00070B5234BC0B21B78984206D1FDF734FF6A
:1076B000FDF7ECFD1F4B187870BD1F4DFDF72CFF3B
:1076C000FFF750FF95F9050006F0B6FE05F01EFA2B
:1076D000287906F07FFE05F00DFA687805F0ECFADF
:1076E000164B1A681C4612F0010213D10421144EE5
:1076F000084632607160FAF71FF9306018B912213C
:107700001048FCF73BFA01230F4A10490C4823604C
:107710000EF0FDF80E4B1A680AB9094A1A600D48B6
:1077200005F0D6FAEB780BB10B4BC4E70B4BC2E775
:10773000AB4800200C480020B048002080480020C2
:10774000C84800207F9E010800000020BD6A000894
:107750008C480020BD7B0008A84800200B48002072
:10776000034B93F83230022B0CBF022000207047ED
:10777000C000002008B5FFF7F3FF30B904F0C8FFE0
:1077800018B9BDE8084004F09FBFFFF7E9FF0228E1
:1077900006D104F0BDFF18B1BDE8084004F0DABF1F
:1077A00008BD000008B5FFF7DBFF02280CBF024B45
:1077B000024B187808BD00BFC5480020C44800200F
:1077C000054B1B8913B9054B18787047044B5B7A3E
:1077D000002BF8D1FFF7E6BFB04800200848002092
:1077E00094480020FFF7DEBF01232DE9F348394C10
:1077F000002000216372FFF723FE10B1364B18788A
:107800001AE02368984718B9344B1B78002B3CD0FA
:1078100005F064FA012871F1000306460F460EDBFD
:107820002F4803F0B7FDFEF707FC32463B46217AAE
:10783000FFF7FDF8FFF7B6FF02B0BDE8F088236858
:107840009847054688B1274803F0A4FD00236468E3
:107850000093ADF80430FFF7D2FD01466846A0471B
:107860006846FFF7C7FD204BC9E71C4B1B7863B187
:107870001E4803F08FFD1E4B1B88022B28D82A467A
:1078800029462846FFF7A2FDEDE71A4D6B89EBB1BB
:10789000EB78DBB1FEF7D0FBFFF7E6F803681B6877
:1078A00098476B89144A154D5A43D5E90067861BE2
:1078B00061EB0707D317B242BB4107DA104803F068
:1078C00069FD40F249310F48FCF758F90023637213
:1078D0000D4B94E794480020C1480020C648002082
:1078E0002BB601083CB60108C04800204EB601087E
:1078F000C2480020B04800208051010058000020FC
:1079000065B6010819B40108084800202DE9F04FB8
:107910000446444D87B0C5E90023019100230A22A3
:10792000414903A8FEF7F6F903A92046FEF79AFAA3
:107930003E4A824628723E492046F8F7D3FF3D4929
:1079400005462046FFF7A4FA3B498DF80300204680
:10795000FFF7C0F9394983462046FFF75FFB3849F6
:1079600080462046FFF768FB0746364A364EDFF86A
:10797000EC902B46014612782046F8F7BEFF33788C
:1079800099F8002039462046F8F7B7FF337899F880
:10799000002029462046F8F7B0FF2A4A33782946C6
:1079A00020461278F8F7A9FF284A9DF803302946A7
:1079B00020461278F8F7A1FF254A2B469DF80310C0
:1079C00020461278F8F799FF224A5B46294620465E
:1079D0001278F8F792FF2B46524659462046F8F7A0
:1079E0008CFF1D4A4346294620461278F8F785FF4A
:1079F0002B46524641462046F8F77FFF337899F8E8
:107A0000002041462046F8F778FF6D230393019B41
:107A100003A9204604938DF81470FEF727FB07B0E6
:107A2000BDE8F08F944800207CB90108E977000890
:107A30008CB901089AB901085DB7010868B7010857
:107A4000A6B901080848002009480020C0480020C5
:107A50000C480020C4480020C5480020C148002030
:107A6000F8B51D4600234171BDF8181004460360A7
:107A7000C180174602B115B923712046F8BD0749E8
:107A8000284602F0AFFD064610B920712660F4E7E3
:107A90002A4639460FF087FB2571F7E73EE60108D5
:107AA00010B50446006808B102F09EFD204610BDE6
:107AB00070B5364E86B03268044622B940F2CB111A
:107AC0003348FCF75BF8002C5DD00022314B1A8064
:107AD000D4E91C2313431FD02F4B1D68FAF718FE5F
:107AE00001462E48A847D4E91C0103F0D3FB226FBE
:107AF00001462B4803F04EFCD4E91C2303A803F0F5
:107B000061FBD4E91C23274903A8C1E900232649C6
:107B1000C1E9002308F006FEFEF78EFAFEF7A4FF87
:107B200003681B689847214B214AC3E90001237A67
:107B3000C3F3C0031370637F2BB3237F1BB31D49B3
:107B4000082002F043FD054630B16289237F617F42
:107B50000092A26EFFF784FF0395A5B10023306861
:107B60001A4603A90068F9F70BFF01280BD0124849
:107B700003F010FC039C34B12046FFF791FF08216D
:107B8000204602F033FD06B070BD00BF8C480020D7
:107B900019B40108C2480020C0000020EEB6010858
:107BA000FBB601086000002068000020580000209B
:107BB000C64800203EE6010828B7010810B5044673
:107BC000FFF776FF24B12046BDE8104006F09EBFC7
:107BD00010BD000038B542F2107004F0D7FD044625
:107BE000124803F0D7FBECB12578022D16D160685E
:107BF0000021FFF7F7FAD4F89800FFF759FF237A2E
:107C00002BB10B4803F0C6FB00220A4B1A7020462A
:107C100005F0DAFC032D06D1284638BD032DEAD144
:107C20000020E5E70125FFF7A5FDF5E7B2B501085E
:107C3000D0B50108AD480020002310B5144C84F8DD
:107C4000363004F065FD08B104F084FDFFF7C2FF93
:107C5000032815D8DFE800F005020A080D4803F0F4
:107C600099FB0D4B187810BD0C4BFBE7FFF778FD27
:107C7000022809BF01230A4B84F83630094BF1E78B
:107C8000094840F2BA21FBF779FF4FF0FF30EAE7ED
:107C9000C0000020E3B501080C4800200B4800207C
:107CA000AC4800208848002019B40108FF230021B7
:107CB0000D4A13700D4A13700D4A13700D4A13705C
:107CC0000D4A13700D4A13700D4A13700D4A13704C
:107CD0000D4A13700D4A13700D4A13700D4AC2E914
:107CE00000111372704700BFAA480020A948002065
:107CF000AB480020C1480020C0480020C5480020F3
:107D0000C4480020A8480020AC4800208848002033
:107D1000894800209448002010B504460068FAF70E
:107D2000F5F9204610BD00002DE9F843054616463A
:107D30000446DFF838900C4F00EB01084445A4EBF3
:107D400005020FD046B13AB1B2FBF6F306FB13239E
:107D500013B9484603F01EFB14F8011B384603F024
:107D600019FBEBE7BDE8F883049E010863D0010826
:107D700013B50B4B02AC04F8010D18680023214623
:107D80001A460068F9F7B2FE064B186828B10023BE
:107D900021461A460068F9F7A9FE02B010BD00BFDF
:107DA000E0480020E4480020C0F3C70342071CBF9E
:107DB0000133DBB218467047052910B501D8002001
:107DC00012E04378013B032BF9D8DFE803F00E0EF5
:107DD00002020024043003F009FC44B1FFF7E4FF81
:107DE00080B2FA28EBD8C0B210BD0124F2E74000FF
:107DF000F6E700000023194A70B5C0E9002381604E
:107E00004E234FF416510446C0E903130A230820F9
:107E10000121C4E905030E23114D23772A686177F8
:107E20000A40A17713D14FF480700E4E326070601B
:107E3000F9F782FD306018B912210B48FBF79EFE5E
:107E400001230A4A0A4907482B600DF060FD094BDF
:107E50001A680AB9034A1A60204670BD0001000280
:107E6000DC480020E84800207F9E01080000002038
:107E7000197D0008E048002002468068036819B1B7
:107E80001B6802F10C0118475B6818472DE9F3479E
:107E90001C469DF8285006468DF807108DF80620E0
:107EA0000DF1070101224FF6FF7002F0A1FB012244
:107EB0000DF1060102F09CFB2A46214602F098FBD8
:107EC00081464FEA202A9DF80620C7B29DF8071088
:107ED0001B4803F05FFA29461A4803F05BFA29466B
:107EE00001222046FFF720FF174803F053FA5246BD
:107EF0004B463946154803F04DFAB0689DF8071017
:107F00000368013C9B689847B0689DF806100368B9
:107F10005FFA8AF89B6898472544B068A5420368D1
:107F20009B6803D014F8011F9847F6E73946984735
:107F3000B068414603689B68984702B0BDE8F08787
:107F4000FEB9010829BA0108CBAC010844BA0108FE
:107F50000B4670B505460A11D1B2092A03F00F038A
:107F60008068D4BF30313731092B94BF03F130041E
:107F700003F1370403689B689847A8682146BDE869
:107F8000704003689B6818472DE9F0470646904605
:107F90001C4689469DF820701144C9B21A1BD2B202
:107FA000974204D913F8012B1144C9B2F6E74942AC
:107FB0004246CDB21D48494603F0ECF939461C480B
:107FC00003F0E8F9012239462046FFF7ADFE1948D3
:107FD00003F0E0F92946184803F0DCF9B0683A21CB
:107FE0000368013C9B68984749463046FFF7B0FF5D
:107FF00041463046FFF7ACFF2744BC4205D014F899
:10800000011F3046FFF7A4FFF7E729463046FFF788
:108010009FFFB0680D2103689B689847B0680A21EC
:10802000BDE8F04703689B68184700BFFEB9010828
:1080300029BA0108CBAC01085FBA010830B4456821
:108040009DF808401DB1012D05D030BC7047029449
:1080500030BCFFF71BBF029430BCFFF795BF000098
:108060002DE9F04F85B090466A4600AF7B600388EB
:10807000464C0733DB08A2EBC3039D4605468A4600
:108080006E46A3462368002207F10F011868F9F72E
:10809000D1FD0128F6D0A8683D49036800245B693A
:1080A0009847FAF735FB4FF47A7300F57A79DBF8E5
:1080B00000001A4607F10F0100683B60F9F7BAFDAE
:1080C00001280AD1621C92B2F97B012A31551DD0D8
:1080D00029883B6891421BD814463CB331785145FE
:1080E0001AD1A868002103685B699847214629488E
:1080F00003F050F9002221463046FFF715FE2648CE
:1081000003F048F9032C1FD8244815E04FF47A7384
:108110001446CCE70022FBE7214803F03BF9FAF7CD
:10812000F7FAA9EB0003B3F57A7FF3D9A868002129
:1081300003685B6998471B4803F02CF9002420462C
:108140001437BD46BDE8F08F331913F8012C13F82E
:10815000025C023C05EB02253146A2B24FF6FF70ED
:1081600002F046FAADB28542014604D02A460E48D6
:1081700003F010F9E2E77B68E4B29C4228BF1C469A
:108180003146224640460FF00EF8D8E7E04800207E
:10819000717D00086EBA0108CBAC0108D1BA0108A4
:1081A0008CBA0108BABA01080ABB01082DE9F04FE0
:1081B00085B016466A469846438800AF0733DB0809
:1081C000A2EBC3039D46724C824689466D46A34688
:1081D0002368002207F10F011868F9F72BFD012829
:1081E000F6D0DAF808006B4903685B69984700230A
:1081F000DBF8000041F2883207F10F0100687B6074
:10820000F9F718FD01287B6826D1FA7B5C1CA4B223
:1082100002F07F02012CFA73EA5408D92B1913F8E3
:10822000022C0D2A03D113F8013C0A2B03D0BAF813
:108230000230A3420ED8DAF80800002103685B6917
:1082400098475CB9544803F0A5F820461437BD465A
:10825000BDE8F08F2346CBE71C46ECE7082C10D88E
:108260004E4803F097F821464D4803F093F828460E
:1082700001222146FFF758FD4A4803F08BF80024FD
:10828000E3E72B783A2B08D12B1913F8022C0D2A8F
:1082900003D113F8013C0A2B01D04348E1E72946FA
:1082A0002A46E01EC0B25FFA85FCA2EB0C03DBB2EB
:1082B00083420BD212F8013FA3F1300EBEF1160F2C
:1082C00002D83A3B062BF0D83848CAE7C30705D591
:1082D000374803F05FF821463648C6E72C46401081
:1082E000C3B2A1EB0C02D2B293422AD994F801E0B6
:1082F000AEF13002D2B2092A07D9AEF14102052A05
:108300008EBF0022AEF13702D2B294F802A0120161
:10831000AAF1300E5FFA8EFEBEF1090FD2B20AD971
:10832000AAF1410EBEF1050F8EBF4FF0000EAAF16B
:10833000370E5FFA8EFE42EA0E0201F8012B02347C
:10834000CFE7002211460138D4B2844202F1010283
:1083500003DA2C5D2144C9B2F6E749422A5CC9B26E
:10836000914203D0144803F015F888E72A784A456B
:1083700002D00A461148F6E7013BDCB2444528BF6B
:1083800044462946224630460EF00DFF5DE700BF09
:10839000E0480020717D0008BABA01084DBB010811
:1083A0006EBA0108CBAC010886BB0108A2BB01086C
:1083B000ECBB01081BBC01083ABC01087DBC0108EC
:1083C0002DE9F0411F46104B04461B680D4616462A
:1083D00023B940F2E9110D48FBF7D0FB63681BB1EC
:1083E000012B09D0BDE8F0813B46324629462046A4
:1083F000BDE8F041FFF734BE3B46324629462046F1
:10840000BDE8F041FFF7D2BEE0480020B1B9010855
:108410002DE9F34704460D469046994680689DF83D
:1084200028A0036801211B6A0B9E9DF830709847B5
:1084300042464B4629462046CDF800A0FFF7FEFDF8
:10844000A068002103681B6A98473B4632462946CC
:10845000204602B0BDE8F047FFF7B2BFF0B51646C0
:108460000C4685B09DF828704A781D460978CDE9FC
:108470000137B31EDBB20093A31CFFF7C9FF60B93D
:10848000022F0AD9012E08D9237803202B70637894
:1084900063F07F036B700B23AB7005B0F0BD000081
:1084A00010B504468068002103681B6A9847A068DD
:1084B00002490368BDE810405B691847717D0008F8
:1084C000034A0260002202710274C0E9022270476E
:1084D000BCBC010870B50646084802F05BFF0024EA
:1084E00006F108053379A34206DD55F8040B013483
:1084F00003689B689847F5E770BD00BFD0BC0108D2
:1085000070B50646002400F108053379A34206DD64
:1085100055F8040B01340368DB689847F5E770BD34
:1085200038B5047900F1080500EB84040834AC4246
:1085300005D054F8040D03685B699847F7E738BD28
:1085400070B50646002400F108053379A34206DD24
:1085500055F8040B013403681B699847F5E770BDB3
:1085600038B503790446012B0D4603D93921074854
:10857000FBF704FB6968064802F00CFF23795A1CDC
:108580000233227144F8235038BD00BFE8BC010813
:108590002BBD010870B504460D4603680121DB6858
:1085A00098472368294620461B6998472368204638
:1085B000BDE87040DB68002118478069704740695A
:1085C000704738B5036804461B6998470546236819
:1085D00020469B699847284638BD8368C0E9033325
:1085E000002383617047000038B50025094B04461D
:1085F000C0E900310B68C0E90355C0E905551B68A7
:1086000008469847A5606061C4E90355A561204606
:1086100038BD00BF9CBD0108D0E90332934291BF31
:10862000D01A40698018C01A7047000038B5054656
:108630000C46FFF7F1FF884203D213210648FBF7EF
:108640009DFAE9686A69AB68214413449942E9607C
:1086500024BF891AE96038BD42BD010808B501464A
:10866000FFF7DAFF4B69181A08BD00002DE9F04743
:1086700002EB030899464369044698450E4617469F
:1086800003D93C211C48FBF779FA6369A568606847
:108690001D4423690121ED1A03681B699847A84509
:1086A00060680DD80368E1685D6832463B4649441E
:1086B000A84760680021BDE8F04703681B691847B8
:1086C0000368A945D3F804800FD2E168A5EB09053A
:1086D0002B4632464944C0476068A1680368721956
:1086E000D3F804807B1BC047E3E7A1683B464944BD
:1086F0003246491BF7E700BF42BD010807B5042217
:1087000000230DEB0201FFF7B1FF019803B05DF804
:1087100004FBF8B5064617460D4679B184695CB18D
:10872000FFF7ECFF87423C4628BF0446042322465D
:1087300029463046FFF79AFF2046F8BD0C46FBE776
:1087400083690BB1FFF7DABF1846704738B5836904
:1087500004466BB1FFF7D2FF054604212046FFF720
:1087600065FF29462046FFF761FFA369013BA3612E
:1087700038BD000038B5436905468B420C4603D22C
:108780005F210748FBF7FAF929696A69AB68214458
:1087900013449942296124BF891A296138BD00BF59
:1087A00042BD01082DE9F04116461D4A04461368F2
:1087B0000F4633441360FFF751FFB04203D22B2121
:1087C0001848FBF7DBF96369A56860681D442369F5
:1087D0000121ED1A03681B6998476068AE4203687F
:1087E0000FD89D683A4633462169A8476068002142
:1087F00003681B69984731462046BDE8F041FFF702
:10880000B9BFD3F808803A462B462169C047606853
:108810007A190368A168D3F80880731BC047E5E79D
:10882000F048002042BD010807B502AB43F8041D23
:1088300004221946FFF7B6FF03B05DF804FB70B5DC
:10884000144605460E46FFF709FF231D98420DD337
:1088500021462846FFF7E8FF224631462846FFF723
:10886000A1FFAB690133AB61204670BD0024FBE77B
:1088700038B50A4C05460121204607F031FD00239A
:1088800020461A46012107F069FC85F001022046C6
:10889000BDE83840012107F02FBD00BF00000240B5
:1088A00008B50120FFF7E4FFBDE80840032008F009
:1088B000C5BC0846FFF7DCBF10B50446024B036099
:1088C00002F010FF204610BDC4BD010810B50446DB
:1088D000054B503040F8503C044B40F8083CFFF743
:1088E000EBFF204610BD00BFA0C1010804C4010871
:1088F00010B50446FFF7E0FF2046082101F076FEA0
:10890000204610BD10B50446FFF7E0FF2046782151
:1089100001F06CFE204610BD024B0121186803686F
:108920001B68184700490020021C18BF01220321C0
:10893000014807F0E1BC00BF0004024010B50C463E
:10894000FAF720FA022808D14FF47A704443B4FBB6
:10895000F0F0BDE81040FAF72DB82046BDE8104011
:1089600007F018BA0321014807F0CFBC0004024009
:1089700010B5094C094802F00DFD20460B2107F007
:10898000AFFC002320461A460B2107F0E7FBBDE8A9
:10899000104007F0E5B900BF000002403AC10108ED
:1089A00008B5022007F040F907F0A2F900F060FCDA
:1089B00007F0C8F900F04CFE07F02CFF0C48FBF75D
:1089C000A7F84FF4E13008F095FA0A4B1A680AB993
:1089D000094A1A60094B1A680AB9074A1A60084816
:1089E00002F0D8FCBDE80840064802F0D3BC00BF46
:1089F000A1880008E0490020950D0108E449002005
:108A000034BE01084CBE0108F7B50446FFF758FD17
:108A1000234600252146214A04F1480043F83C2B17
:108A2000E5635D601E4B1F4E41F8443F01F04EF878
:108A30001D4B84F85C50A3651C4BC4E91A55236692
:108A40001B4B84F8705063661A4B1B48636702F037
:108A5000A1FC3368194F01933B68194D00932B68B3
:108A6000184A1B2104F121000FF030FA296804F1A3
:108A7000110002F0C9FD396804F1150002F0C4FDCF
:108A8000316804F1190002F0BFFD296804F11D00EE
:108A900002F0BAFD204603B0F0BD00BFA0C101083E
:108AA00094C201086400F81F30C3010860C30108C4
:108AB0004CC30108CCC201086EC101085400F81F64
:108AC0005000F81F83C1010810B5094CFFF768FF7B
:108AD0002368DB0709D40748FFF796FF0123064AFE
:108AE0000649044823600CF012FF024810BD00BF85
:108AF000F84800200449002000000020CD8800082C
:108B000038B5064D064C2B6813F0010F04D1FFF762
:108B1000DBFF012320602B60206838BDFC4800206B
:108B20007C4900204FF4FA71FFF734BD08B50B21E2
:108B3000054807F0EFFB28B1BDE808400B210248CB
:108B400007F0FCBB08BD00BF0000024008B519B12A
:108B5000BDE80840FFF70CBF044802F01BFCBDE86D
:108B6000084002220B21024807F036BB56C101081B
:108B700000000240F8B50446384804F1440502F00C
:108B800009FC2846002100F08BFD0021284600F05A
:108B90009DFD334D2046FFF7C3FC03F095FD2046B5
:108BA0000021FFF7D3FF0BF0C1FC0BF0E5FF012222
:108BB0000C21284607F010FB07F04AFF04F148009B
:108BC00000F066FF23682046DB6804F1640600219C
:108BD0009847244F0021304600F07CFE07F00CFC43
:108BE000214802F0D7FB08F061F807F0ABF83846EF
:108BF00001220D2107F0F0FA012238460E2107F07C
:108C0000EBFA0021084607F0E1FE04F1580000F0FD
:108C1000F1FD0121304600F05DFE4FF4E13008F037
:108C200069F9124802F0B6FB28460C2107F058FB00
:108C3000002328461A460C2107F090FA0120002153
:108C400007F02AFF0BF0AAFF0BF096FB07F0FEFEE1
:108C50002046BDE8F840FFF773BC00BF08C101081B
:108C600000040240000002402CC1010806C00108B7
:108C700038B50546FFF75AFF044628B100212846BB
:108C8000FFF764FF07F06CF806F072FF05460CB1C1
:108C9000FFF76EFE284638BD70B50C4606461549EE
:108CA00020460DF023FF20B9002120460DF000FFE3
:108CB00070B1114920460DF05DFD0DF021FF014618
:108CC0000E4802F067FB4FF4BB710D48FAF756FFF0
:108CD0003046FFF72BFF054648B93046FFF7C8FF7F
:108CE000014620460DF002FF08B1FFF741FE28467D
:108CF00070BD00BF3333534000007A4462BE0108A8
:108D000091BE010870B52D4AD6B013680546DB0741
:108D100005D42B4900F164030B600123136029493A
:108D20002846FFF7B9FF0646274802F033FB00212B
:108D300005F1440000F0CAFC244C254BE360254BB0
:108D40002361254BA360254B6360254B2360254B96
:108D50006361254BA361254BE36104F110030FCB45
:108D60008DE80F0094E80F000CF042F9002305A8ED
:108D7000EB632B640CF0C8F89DF8143005F13C044B
:108D8000012B14D1DDF8153005A8EB63DDF819309F
:108D90002B640CF089F8164802F0FCFA08212046F2
:108DA00002F05EFBBDF91611124802F0F3FA3146EB
:108DB0002846FFF7CBFE56B070BD00BFF448002038
:108DC0000049002000004040CDBD0108585100205E
:108DD00095FD00081DFD0008198900086589000837
:108DE0002989000895B300080537000845370008B1
:108DF000EEBD010814BE010808B5FFF739FF0349AD
:108E00000DF0B8FC0DF0A2FE80B208BD00007A445F
:108E100070B507490546FFF73FFF06460CF00CF812
:108E2000044631462846FFF791FE204670BD00BF3C
:108E3000000040407FB5F82300F1580504AC064619
:108E4000284604F8013D00F0DBFC02232146009394
:108E50000122A123284600F0D7FC4FF4004308224A
:108E6000009306F16801A1230446284600F0F6FCB1
:108E70000440E4B2284600F0C5FC204604B070BDB2
:108E800030B58BB0044608F007FA0146574802F0A7
:108E900081FA574802F07EFA204600F08FFB04F179
:108EA000580500F0C1FA00F06BFA5248524902F03E
:108EB00071FA284600F09EFC38B9504802F06AFA70
:108EC00040F233114E48FAF759FE06F049FF2046AA
:108ED000FFF7B0FF20B94FF49C714948FAF74EFEF6
:108EE00094F86F0094F86A30049094F86E0094F847
:108EF0006920039094F86D0094F86810029094F83B
:108F00006C00019094F86B0000903E4802F042FA29
:108F1000284600F037FA284600F098FA04F1440594
:108F200084F8700004F1740000F016FC002128465B
:108F300000F0B6FB012000F0D7FD0021284600F02C
:108F4000C5FB012000F0EEFD2046FFF7DBFE00F040
:108F5000C9FA2D4802F01EFA4FF4FA700EF0E4F848
:108F6000054600283AD1294802F014FA284802F0B0
:108F700011FA284802F00EFA274802F00BFA2748A7
:108F800002F008FA264802F005FA264802F002FA32
:108F9000254802F0FFF9254802F0FCF9244A25494A
:108FA000254802F0F7F92549254802F0F3F925484C
:108FB00002F0F0F904F12101234802F0EBF907A8CF
:108FC00007F0C0FB07A802F03BF901461F4802F07A
:108FD000E1F9104802F0DEF90BB030BD1C4802F098
:108FE000D9F928460EF0A8F8C0E700BFD9BE01089D
:108FF000EFBE010806BF0108A086010021BF0108DD
:1090000091BE010837BF01086CBF01089FBF01086E
:10901000CAAC0108DDBF01080EC001081DC001086F
:109020003FC0010862C0010886C00108CBAC01083E
:1090300097AA010872AA0108A9C00108B9C00108CD
:10904000C0C00108CBC00108EBC00108F6C0010890
:10905000D3BF01082DE9FF4100F15805284600F073
:10906000CFFB04240226284F013C14F0FF0433D028
:10907000A123012239460096284600F0C5FB4FF493
:109080000043804600930422A12302A9284600F051
:10909000E5FBB8F1000F01D10028E5D09DF80830BC
:1090A000442B20D19DF809306E2B1CD10DF10A0004
:1090B00002F09CFA0223013084B221460DF109002E
:1090C0008DF8083002F0B3FA002303220093A023A6
:1090D00002A9284600F098FB284600F093FB2046A2
:1090E00004B0BDE8F0814FF488430024ADF80830A7
:1090F0006E2300210DF10B008DF80A3002F097FA73
:109100000094A0230522E3E7CCBD010838B50C4646
:109110001131054603F0AAF9214651F8683F284667
:109120002B604B686B6038BD024B186803685B6846
:10913000184700BF8C490020024B186803689B68E1
:10914000184700BF8C4900202DE9FF410023154638
:109150001370022206460D4F04AC386804F8011D56
:1091600003680092D3F80C80012233462146C047A1
:1091700048B14FF4004238682946036800921C69E0
:1091800001223346A04704B0BDE8F0818C4900209D
:1091900030B585B08DF80D200022074B8DF80C10EE
:1091A0001C6803A923680092DD680222034620465A
:1091B000A84705B030BD00BF8C49002037B54FF43B
:1091C0000045064B1C68236800951D6913460A4636
:1091D00001462046A84703B030BD00BF88490020A3
:1091E00037B50025054B1C6823680095DD681346DC
:1091F0000A4601462046A84703B030BD88490020F2
:1092000037B50225054B1C6823680095DD681346B9
:109210000A4601462046A84703B030BD88490020D1
:10922000024B186803681B68184700BF8849002074
:10923000024B186803685B68184700BF8849002024
:10924000024B186803689B68184700BF88490020D4
:109250004FF47A735843B0FBF3F0F9F7ABBB10B59A
:109260000446FFF74DFC2146BDE81040FFF7F2BE73
:1092700010B5424C0BF0ACF920460222002106F05A
:10928000ABFF01222046114606F0A6FF2046012230
:10929000022106F0A1FF20460222032106F09CFFD6
:1092A00020460022042106F097FF204602220821D2
:1092B00006F092FF20460122092106F08DFF20468C
:1092C00001220A2106F088FF204602220B2106F027
:1092D00083FF06F037FD002320461A460C2106F0D6
:1092E0003DFF204600220C2107F006F82046002210
:1092F00004F580640F2106F06FFF20460122002153
:1093000006F06AFF20460022022106F065FF204693
:109310000022032106F060FF20460222062106F00B
:109320005BFF20460022082106F056FF204600225F
:10933000092106F051FF204601220C2106F04CFFC6
:10934000204602220D2106F047FF204602220E2170
:1093500006F042FF204602220F2106F03DFF0023C7
:1093600004F5806420461A460D2106F0F7FE2046DB
:10937000BDE8104000220D2106F0BEBF00000240F3
:1093800007F048BA1D4B00B51A6889B0D2075FBF15
:109390001B4A106001221A601A4B1B4A04931B4B94
:1093A00005931B4B03931B4B02931B4B079308AB7B
:1093B00043F8082D93E803008DE8030002AB0FCBC0
:1093C0000BF0CAFC90B1154801F0E4FF00221448EC
:1093D000114606F001FF0F2302220021104806F07B
:1093E0009BFD09B05DF804EB0BF050BC69210D4802
:1093F00009B05DF804EBFAF7C1BB00BF8449002057
:109400008C490020299100085192000839910008E8
:10941000499100089191000895B3000832C20108F3
:109420000000024043C20108002307B5ADF8043034
:1094300001238DF8063001980BF026F806F082FC27
:1094400003B05DF804EB0BF071B80000194B10B5D8
:109450001A688CB0D2075FBF174A106001221A60E9
:10946000164B0793164B0593164B0693164B089312
:10947000164B0993164B0A93164B0B930CAB13E93F
:1094800007008DE8070005AB0FCB0BF04BF9044646
:1094900001220F21104806F09FFE3CB10F4801F059
:1094A00079FF0BF01DF920460CB010BD0C4801F0FF
:1094B00071FFF8E78049002088490020BD9100082D
:1094C000E191000801920008219200083192000801
:1094D0004192000895B3000800000240B4C10108A1
:1094E000E7C101082DE9F0479EB002F035FCDFF836
:1094F000C890284C284E294F16AD50B9CDE91944D3
:10950000CDE91776CDF85890009495E80F0002F059
:1095100029FC234B4FF0000A1793224B4FF0010810
:109520001693214B09A91893204B28461993204BD9
:10953000CDE91C76CDE91A340423CDE9093A8DF83A
:10954000298009F0F1FA09F0E3FA0EF057FC5146D0
:1095500010220CA80DF04BFE164BCDE910441593CC
:1095600003238DF836800B9302AC0BAD0FCDCDE904
:109570001376CDF848900FC42B68236014AB93E8A2
:1095800003008DE8030010AB0FCB02F099FF1EB073
:10959000BDE8F08795B30008A1B40008CDB4000879
:1095A000B1440108794301088942010821420108B8
:1095B000354201085F920008010801082DE9F047D3
:1095C000044606F0D5FA1E4905460DF0D3F80DF015
:1095D00097FA01461B4801F0DDFE4FF08041284616
:1095E0000DF066FA48B30025DFF86090DFF8508090
:1095F000154E06F0BDFA494607460DF06DFAA8B9BA
:10960000414638460DF0B6F80DF07AFA014630467C
:1096100001F0C0FE236885F001052046DB6829467D
:1096200098474FF47A7006F0B5FBE2E723682046CE
:10963000BDE8F047DB6800211847BDE8F08700BFB0
:1096400000007A4405C2010817C20108000020404A
:1096500008B50D49012006F033FF0C490B2006F038
:109660002FFF0B490A2006F02BFF0A49042006F0C1
:1096700027FF0949072006F023FFBDE808400749F6
:10968000052006F01DBF00BFE93D010805410108A6
:10969000913F01081D42010871410108F94101088B
:1096A000002310B50C461A460D21074806F056FD5A
:1096B00014B1012C00D010BD2246BDE810400D2190
:1096C000014806F019BE00BF00080240002310B593
:1096D0000C461A460C21074806F040FD14B1012C37
:1096E00000D010BD2246BDE810400C21014806F014
:1096F00003BE00BF000002400BF064B908461146EB
:109700001A460BF0FDB9084611461A460BF07AB915
:10971000084611461A460BF0AFB900000C2110B1F3
:10972000024806F0DDBD014806F0E0BD000402403D
:1097300010B561B1FFF7E4F904460BF017F90146E3
:109740002046FFF7A9FABDE810400BF027BABDE8A4
:1097500010400BF011BA000070B588B0FFF7D0F9D7
:109760001D490546FFF798FA0C2106461B4806F0EE
:10977000B7FD00230C211A46184806F0EFFC002123
:10978000012007F089F9102200210DEB02000DF0F5
:109790002EFD134B02AC0293124B0693124B039314
:1097A00008AB13E903008DE8030094E80F000BF009
:1097B0000DFA60B10BF006F901460C4801F0EAFD24
:1097C0003146284608B0BDE87040FFF7BFB90848E9
:1097D00001F0E0FDF4E700BF00004040000402405B
:1097E0001D97000895FD00084D0B01089CC201085B
:1097F000B2C20108014806F0EDBD00BFA08601001D
:1098000006F0B8BD06F0D2BD2DE9F041069F1E4618
:1098100007F00303032B80460C46154603D12F2186
:109820000D48FAF7ABF92046BC07324629460AD55F
:1098300006F00AFE10B10120BDE8F08101230020EE
:1098400088F80430F8E7FB0702D506F00BFEF1E7D5
:1098500006F0ECFDEEE700BFE0C201082DE9F041A3
:10986000069C0D46E107804616461F4603D54C214F
:109870000D48FAF783F9A20703D54F210A48FAF7F2
:109880007DF923043A46314628460AD506F0F8FD0C
:1098900010B10120BDE8F0810123002088F80430D8
:1098A000F8E706F0B5FDF3E7E0C2010808B50321CB
:1098B000034806F02AFD003018BF012008BD00BF94
:1098C000000402400A460248032106F015BD00BF0D
:1098D0000004024008B581B1012303211A460A4859
:1098E00006F03CFC0321084806F0FAFCBDE80840FD
:1098F00003220548114606F011BC0122BDE80840CC
:109900000321014806F068BC0004024006F078BF5D
:109910001FB501A801F056FC01A806F003FF05B031
:109920005DF804FB1FB501A801F04CFC01A807F08D
:1099300047F805B05DF804FB06F0B0BF06F0C8BFFD
:10994000084606F03FBEDFB50023CDE90133ADF890
:109950000C3001238DF807308DF808306FF01D03AF
:109960008DF809300723044601A88DF80A3001F06C
:109970004EFC236806461B6820460F4698478642E1
:1099800077EB0103B4BF0120002004B0D0BD7047C5
:10999000704700007FB500F10806054630460C46CA
:1099A00001F0CAFE60BB334801F0F4FCA27C617C8C
:1099B000314801F0EFFC637C3BB16868002103682B
:1099C0001B689847022000F08FF8A37C3BB16868C1
:1099D000002103685B689847022000F0A3F86168E3
:1099E0004E2918D04F2916D0452914D015212348C7
:1099F000FAF7C4F81621224B224A20480DF080FACB
:109A00006421304601F084FE0028CFD142211B485A
:109A1000FAF7B4F8CAE7A268082A0BD0092A09D0D5
:109A2000072A07D023211548FAF7A8F8144B164A3D
:109A30002421E2E7E3680A2B10D009DC052B0ED0C5
:109A400033210E48FAF79AF80D4B104A3421D4E727
:109A50000F2B04D0142BF3D1022300E00123A07CB0
:109A60000290607C0190207C0090206807F07CFAD6
:109A700004B070BD7CC30108DDC3010895C30108B3
:109A800015A9010824C4010888C4010854C40108A8
:109A900010B5044607F03AFA04F10800BDE810409A
:109AA00001F04DBE084607F047BB38B50C468D188F
:109AB000AC4204D014F8010B07F03EFBF8E738BDC8
:109AC00007F04ABA084607F067BB000010B5044625
:109AD000044BC0E900310121083001F03BFE204673
:109AE00010BD00BF04C40108042817D8DFE800F047
:109AF0000309100E1200002303211A46084806F03D
:109B00002DBB00220321064806F066BB0222F9E7BE
:109B10000122F7E70321024806F084BB704700BF2B
:109B200000000240042817D8DFE800F00309100EF7
:109B30001200002302211A46084806F00FBB00223B
:109B40000221064806F048BB0222F9E70122F7E7A6
:109B50000221024806F066BB704700BF00000240C9
:109B6000406803681B681847406803685B681847CB
:109B7000406803689B68184740680368DB681847BB
:109B8000406803681B691847406803685B691847A9
:109B900070470000436910B504469BB983698BB9CF
:109BA0008168094801F0F6FBA168084801F0F2FB62
:109BB00041F28830F8F7FEFEBDE81040312104483C
:109BC000F9F7DCBF10BD00BF6BC5010889C50108EE
:109BD000A0C50108C0E903120346002210B5074CD6
:109BE000C0E905224460064C8460064C0460064CC3
:109BF000C0E90741586280F8282010BDE1C501087E
:109C0000E7C50108F4C5010814C60108436970B529
:109C100005460C4633B3012913D002291CD0002974
:109C20004CD10A46184601210BF069FD224602215B
:109C300068690BF064FDE868BDE8704003681B6963
:109C400018470A4618460BF05AFD22466869022159
:109C5000BDE870400BF053BD0E21BDE870401846C2
:109C60000BF0AEBC806948B301290CD0022914D096
:109C700021BB0A4601210BF038FE22460221A869C9
:109C80000BF033FED7E70A460BF02FFE22460221E7
:109C9000A869BDE870400BF028BE1A4601210BF000
:109CA00024FE01222146A8690BF01FFE0122042197
:109CB000A8690BF01AFE01220821E9E770BD80684F
:109CC000FFF7A4BF38B504460C2000F06DFC054634
:109CD00021690BF051FC656128460BF0FDFC38B39F
:109CE00042F26252A168144801F054FB002384F848
:109CF00028300C2000F058FC054621690BF012FDBD
:109D0000A56128460BF058FDA0B14FF41552A1688B
:109D1000094801F03FFBF021A0690BF0DCFD0123B5
:109D200084F828302046BDE838400221FFF76EBF96
:109D30006061DEE7A061F5E7C0C401080221FFF71A
:109D400065BF034640690A4610B104210BF0D7BC39
:109D5000986910B104210BF0C8BD704700000000E5
:109D60002DE9F04790F8284006460F46002C3CD0DD
:109D7000FEF7C6FE0546002F51D0FFF73DF80F2431
:109D800040F64759DFF8B08048450EDC01464046B2
:109D900001F000FB2B684FF47A711B692846984745
:109DA0002846FFF729F8013CEED1B168204801F0C0
:109DB000F1FA00213046FFF7C4FF1E24DFF87CA033
:109DC000DFF87C802846FEF753FF81460CF062F8EE
:109DD00015A3D3E900230CF045FB48B12B6840F2F2
:109DE000DC511B69284698473C462046BDE8F08771
:109DF000514648460CF0BEFC0CF082FEB1680246AB
:109E0000404601F0C7FA2B6864211B692846984731
:109E1000013CD7D101213046FFF793FFE5E7B16858
:109E2000044801F0B7FAF5E76666666666660640BE
:109E300019C5010855C50108E1C4010800007A44AC
:109E40002EC50108F0B508B90020F0BD002746680E
:109E50004D1CB5421760F7D803685C185B5C03F0D3
:109E60001F03A3F1180103298FBF38460D49C918F4
:109E700011F8180C0544AE42E6D304280DD8DFE8EB
:109E800000F00403070C0C00637813600130DCE77A
:109E9000B4F801305BBA9BB2F7E7D4F801301BBAD3
:109EA000F3E700BF38C60108F7B51F4643681646FA
:109EB0004A1C9A4205460C4617D803685B5C03F0BF
:109EC000C003402B11D196B101AAFFF7BBFF50B1DF
:109ED000019A04446B68A118994206D82968104475
:109EE0000C4434603A6003B0F0BD0020FBE730461C
:109EF000F9E72DE9F7439946436817464A1C9A4209
:109F000080460D4624D803685B5C03F0C003402BF9
:109F10001ED1FFB101AAFFF795FF0446A0B1019E33
:109F200009F10109B14513D30544D8F80430721979
:109F30009A420DD8D8F800103246294438460DF020
:109F400032F900233444BB55204603B0BDE8F0830A
:109F50000024F9E73C46F7E7F0B5002931D0172A8D
:109F60001CD8D3B2A3F11804032C8CBF0024164CC8
:109F70008D689CBFE41814F8184C6F1C4E6804EBF5
:109F8000070CB4451DD20E6818438F607055002031
:109F90000130231A5D1C0BD1601CF0BDFF2A05D9CE
:109FA000B2F5803F2CBF1A231923DBE71823D9E72A
:109FB0008E680D68DB00771C22FA03F38F60AB55C7
:109FC000E6E70020E9E700BF38C60108172BF8B51F
:109FD0000D4616461C4612D8DBB2A3F11802032A1E
:109FE0008FBF0022144A9B1813F8182CAB6801325B
:109FF000234413446A6893420BD30020F8BDFF2B1F
:10A0000005D9B3F5803F34BF19231A23E5E7182398
:10A01000E3E722462946FFF79FFF07460028ECD0DA
:10A020002868AB68314618440DF0BDF8AA68E019FD
:10A030002244AA60E2E700BF38C6010818B1002335
:10A04000C0E9001283607047436873B514464A1C28
:10A050009A4206460D4602D9002002B070BD036840
:10A060005B5C13F0C00FF7D1002CF5D001AAFFF70D
:10A07000E9FE0028F0D03268019B525D12F0E00F3B
:10A0800018BFDB432360E8E70A1EABBF0146014669
:10A090000020D243B8BF2020FFF75EBF03685B5C9F
:10A0A00003F0E001E02907D132B1A3F1F5014B4201
:10A0B0004B4113700120704700207047836810B532
:10A0C00044685A1CA24208D2002914BFF524F42483
:10A0D000016882600120CC5410BD0020FCE7F0B480
:10A0E00046684F1CB74208D805686C5C04F0E00471
:10A0F000402C02D1F0BCFFF7D7BE0020F0BC704767
:10A1000013460A4601464020FFF760BFF0B4466898
:10A110004F1CB74208D805686C5C04F0E004602C62
:10A1200002D1F0BCFFF7E5BE0020F0BC7047F0B4F0
:10A1300046684F1CB74208D805686C5C04F0E00420
:10A14000602C02D1F0BCFFF7AFBE0020F0BC70471E
:10A1500070B5054608460C460DF01EFF2246034624
:10A160002946BDE870406020FFF730BF8368416832
:10A170005A1C8A423FBF8260BF220168012034BF5F
:10A18000CA54002070470368585CA0F1BF035842CE
:10A190005841704713B5036814465B5C03F0E00355
:10A1A000A02B07D142B101AAFFF74CFE019B23600F
:10A1B00002B010BD0020FBE71046F9E78368416854
:10A1C0005A1C8A423FBF8260FF220168012034BFCF
:10A1D000CA540020704730B18068013888428CBF73
:10A1E0000020012070470120704708B50246FFF7A4
:10A1F000F2FF30B91268505CA0F1FF035842584199
:10A2000008BD0120FCE743688B4207D903685B5C0B
:10A2100013F0C00F0CBF01200020704700207047D2
:10A2200043688B4208D90368585C00F0E000A0F155
:10A2300040035842584170470020704743688B42A2
:10A2400008D90368585C00F0E000A0F160035842B0
:10A25000584170470020704743688B4208D9036813
:10A26000585C00F0E000A0F1A0035842584170474C
:10A270000020704710B50446FFF7EEFF50B1636849
:10A280008B4208D92368585C00F01F00A0F11F031F
:10A290005842584110BD0020FCE743688B4208D962
:10A2A0000368585C0C30C0B201288CBF002001202C
:10A2B0007047002070470023C0E901330369016043
:10A2C000C360704703468068F0B51D68013090FB9D
:10A2D000F5F405FB14005C68A04224D000269642E9
:10A2E000304601D11046F0BD8F5DD3E902452F55B0
:10A2F0009C681D68671C97FBF5F405FB14745F6888
:10A300009C60BC4204F1010402BF94FBF5F705FB1D
:10A3100017475F6094FBF5F705FB17445D68AC4297
:10A32000E1D00136DBE70020DDE70000F8B5036887
:10A330000446002B0D46164603DC3E212948F9F75A
:10A340001DFC3246002128460CF051FFD4E9017073
:10A35000B8420CD00021236801EB070C9CFBF3F200
:10A3600003FB12C2904205D10020884204D14FF075
:10A37000FF3031E00131EFE7C21992FBF3FE03FB3E
:10A380001E2ED4F80CC01CF80EE0BEF10A0F26D128
:10A3900028B3013A92FBF3F103FB1122002106F1ED
:10A3A000FF3E71450ED2E7686368FB5C6B546768DB
:10A3B0002668013797FBF6F306FB137701318842D5
:10A3C0006760EEDA1CF802300D2B4FF0000304D169
:10A3D000054405F8013C0138F8BD2B54FCE7013079
:10A3E000C3E700BF3CC601084B1C017343738B1CC1
:10A3F00003318373C17370472DE9F04107468846E6
:10A400001E4615461AB952211548F9F7B7FBD7E988
:10A410000143A34221D2E41ADEB1A3B9A5420ED36F
:10A420003B7B3370BB6839682246194440460CF0C8
:10A43000BAFEBB682344BB602046BDE8F0817B7B4D
:10A4400033702C46EEE7A54201D3FB7BE9E7BB7BEB
:10A45000F6E7AC4228BF2C46E4E70024ECE700BF57
:10A460008CC601080023C0E900128360704710B554
:10A4700004460846C4E900120021A16021730CF0D3
:10A48000B6FE204610BD000038B51546D0E90123C0
:10A4900004465819904202D9257B55B1D51A206837
:10A4A0002A4618440CF07FFEA3681D44A5600125D0
:10A4B00003E01B210248F9F761FB284638BD00BFC5
:10A4C000D0C6010807B502AB03F8011D01221946E9
:10A4D000FFF7DAFF03B05DF804FB0068704780689F
:10A4E0007047002383607047D0E90120101A70473D
:10A4F000026880681044704738B5D0E901230D46E2
:10A5000059189142044602D9017B21B1D51AA1689C
:10A510002944A16038BD49210148F9F72FFBF6E72E
:10A52000D0C6010813B5044601A801F080F8022244
:10A5300001A92046FFF7A8FF02B010BD13B50446DD
:10A54000684601F06AF8052269462046FFF79CFF3D
:10A5500002B010BD13B5044601A801F068F802224C
:10A5600001A92046FFF790FF02B010BD08B50146D3
:10A57000044800F00FFFBDE808400C210248F9F73D
:10A58000FDBA00BF10C701082EC7010808B504486E
:10A5900000F000FFBDE808401E210248F9F7EEBABE
:10A5A00099C70108C6C7010810B500F08FFF04461F
:10A5B00030B9044800F0EEFE27210348F9F7DEFA2F
:10A5C000204610BD87C70108C6C7010800F07EBF3E
:10A5D00010B9024800F0DEBE00F062BF72C7010889
:10A5E000FFF7E2BF00F072BFFFF7F2BFFFF7F0BF67
:10A5F00010B5074C0A44914200D110BD11F8013B3F
:10A600004340DBB234F8133083EA1020F3E700BF95
:10A610000AC80108F8B50E46054680B14F1C3846F9
:10A6200000F054FF044640B13A4600210CF0DFFD33
:10A630003246294620460CF0B6FD2046F8BD0446B9
:10A64000FBE738B50D46044628B10DF0A5FC2346BE
:10A650002044834201D1002038BD13F8012BAA42C7
:10A66000F7D10120F8E737B504460D460CF074FC2D
:10A67000002201A9026020460DF0BAFD04460CF04C
:10A680006BFC0368222B08D0019B1B782BB9002C94
:10A6900003DB20462B6003B030BD012300202B607C
:10A6A000F9E700002DE9F04F05464FF0010B0026B9
:10A6B00087B0CDE9031206F10903122B8CBF0320EA
:10A6C000022000F003FF0090E8B1324636490DF059
:10A6D00031FC039B53F82690EDB90024009800F05C
:10A6E000DFFEBBF1000F02D1284600F0D9FE84B195
:10A6F000049B0136B34225464FF0000BDBD12046C8
:10A7000007B0BDE8F08FBBF1000F02D1284600F082
:10A71000C7FE0024F3E7254B4FF00008B9F1000F06
:10A7200008BF994648460DF037FC019000980DF09F
:10A7300033FC0290284649460DF05DFCB8B9284626
:10A740000DF02AFCDDE9012301309B1A08FB030010
:10A7500000F0BCFE04460028BFD003462F4618F187
:10A76000FF3809D2394618460DF00EFCB6E7019BBA
:10A7700008F101081844DEE74946384605930DF014
:10A780003AFC059BA0EB070A5246394618460DF0E5
:10A790001DFC009950440DF0F7FB019A029B924476
:10A7A000C3185744DBE700BFA2AA0108CCAC0108DC
:10A7B00030B580B10346021F00F1180452F8045F5F
:10A7C0008D4208D0A242F9D11C301A4614680433D5
:10A7D000013401D1116030BD8342F6D1FBE770B581
:10A7E000044680B1064600EB8105AE4204D1204606
:10A7F000BDE8704000F054BE56F8040B0028F4D0B9
:10A8000000F04EFEF1E770BD2DE9F74F894600924A
:10A81000002838D00027C45D8CBB054683462646F9
:10A8200000EB070AD34538D104B10136002E6FD0B2
:10A830000137384600F04AFE8346002866D03A4683
:10A8400000210CF0D4FCB00000F040FE04460028CB
:10A8500060D04FF000084146AA4532D131B1584688
:10A86000FFF7D8FE002855D044F82800584600F0DD
:10A8700017FE009B1E60204603B0BDE8F08F013735
:10A88000B7F5807FC7D100242646204600243146F4
:10A89000FFF7A5FF009B1C60EDE79BF800304B45E0
:10A8A00005D10CB1002401360BF1010BBAE70CF015
:10A8B0002DFC9BF80030184443781B0758BF013427
:10A8C000F2E72B784B4513D181B15846FFF7A2FE32
:10A8D00000B308F1010344F8280000213A46584625
:10A8E00001930CF084FC019B002198460135B3E7ED
:10A8F00001910CF00BFC2B7801991844407810F072
:10A90000080F04BF0BF801300131EFE70446BCE744
:10A910003446B0E7584600F0C3FDB6E72DE9F743EB
:10A92000002506460820884691461F46009500F0FF
:10A93000CDFD0446002868D0C0E9005530460DF032
:10A940002BFB01280FD133782A2B0CD109F1FF33CF
:10A95000C4F80080636022684A4502D263684B45B0
:10A9600043D32B4B0EE02D213046FFF76AFE054600
:10A97000C0B902A941F8040D3046FFF774FE019BEF
:10A9800063B1244B3B6000992846FFF728FF002C59
:10A9900037D0204600F084FD002432E0C4E90000F6
:10A9A0001D46D8E76A462D213046FFF72DFF009B54
:10A9B0000546013B012B01D9174BE3E7002302AE0B
:10A9C00046F8043D31460068FFF74DFE2060019BCC
:10A9D0000BB1124BD6E731466868FFF744FE606062
:10A9E000019B002BB7D00E4BCCE7424501D343452A
:10A9F00001D20C4BC6E700992846FFF7F0FE002372
:10AA00003B60204603B0BDE8F0830546BBE700BFCE
:10AA1000E6CA010860CA01087FCA0108A8CA01087D
:10AA2000C7CA010806CB010838B590B1451E15F814
:10AA3000014F0CB9204638BD0CF068FB234620447A
:10AA4000427802F00302022A08BFA4F120032B700F
:10AA5000EDE70120EFE708B520B34A1C22D0062914
:10AA600020D8DFE801F0040D101316191C00002394
:10AA700003600CF09FFC0840431C5842584108BD3D
:10AA800000234360F5E700238360F2E7002383613E
:10AA9000EFE70123C360ECE700230361E9E700234C
:10AAA0004361E6E70120EAE770B506460D1F01F1B4
:10AAB000180455F8041F4B1C03D1A542F9D10020FE
:10AAC00070BD3046FFF7C7FF0028F6D0F8E708232F
:10AAD0004A4291FBF3F302F0070201F0070158BF6D
:10AAE00051420122DBB2C9B202FA01F1C25C114348
:10AAF000C154704708234A4291FBF3F302F0070266
:10AB000001F0070158BF51420122DBB2C9B28A40AD
:10AB1000C15C21EA0201C1547047082391FBF3F3A1
:10AB2000DBB2C05C4B4203F0070301F0070158BFE2
:10AB30005942C9B2084100F0010070472DE9F047C1
:10AB4000089E8A4690461D46DDF82890074610B1BB
:10AB50001446A24507D875B9012200240B9B1A6040
:10AB60002046BDE8F08721463846FFF7D6FF00288B
:10AB700061D10134EDE7099B023B042B04D8DFE8E7
:10AB800003F0282C2C3034006B6801336B602846AE
:10AB90000CF010FC013108BFB0F1FF3FDCD03146B2
:10ABA0002846FFF758FF0028D6D12FB30446214688
:10ABB0003846FFF7B2FF002841D10134A245F6D153
:10ABC0000446013E042E19D8DFE806F02B2D2F3164
:10ABD0003300AB680133AB60D9E7EB680133EB605E
:10ABE000D5E72B6901332B61D1E76B6901336B61C9
:10ABF000CDE7002DE5D1AFE73C46E2E72C602846E3
:10AC00000CF0D8FB013108BFB0F1FF3FA4D0B9F17F
:10AC1000000FA1D049462846FFF746FF00289FD0E5
:10AC20009AE76C60EBE7AC60E9E7AC61E7E7EC6002
:10AC3000E5E72C61E3E7A045DBD1444690E7A0457A
:10AC4000BFD1FAE700232DE9F04F06468BB01C2058
:10AC50000C469046099300F039FC0546002800F0A8
:10AC6000E4801C2000F032FC0746002800F0DD8064
:10AC70004FF0FF31021F2B1F05F1180043F8041F8E
:10AC8000984242F8041FF9D100230121D4F800A012
:10AC90000DF12409CDE90031CDE902793C212346AB
:10ACA00052463046FFF74AFF099900296ED1824586
:10ACB00002D12846FFF77CFD02234FF0010AD4F8A9
:10ACC00004B0CDE900A3CDE9025923465A463C2100
:10ACD00006F10800FFF732FF099B002B56D1834590
:10ACE0004CD151462846FFF763FD03234FF0020A7B
:10ACF000D4F808B0CDE900A3CDE9025923465A465D
:10AD0000182106F11000FFF719FF099B002B3DD118
:10AD1000834546D151462846FFF74AFD40F26F1B56
:10AD2000A3690593E368049306F114030693DDF821
:10AD300010A006F11303079351460698FFF7EDFEA6
:10AD400028B105990798FFF7E8FE002836D1BBF136
:10AD5000010B33D0E36820460133E3600CF02AFB9B
:10AD6000013108BFB0F1FF3F24D0A3692946204636
:10AD7000D4F80CA00593FFF797FEDDE74246214685
:10AD80003046FFF75FFF09900028AED0284600F05C
:10AD900087FB17B1384600F083FB09980BB0BDE87C
:10ADA000F08F424621463046FFF74CFF09900028BD
:10ADB000ECD1B3E701234FF0000A0993099B002B64
:10ADC000E4D1049B534520D104212846FFF7F0FC31
:10ADD00005230622D4F810A0CDE90032CDE90259AE
:10ADE000234652460C2106F11800FFF7A7FE099BE7
:10ADF000002BCBD18245C9D06369A3EB0803042B98
:10AE00000CD94FF0FF330993C0E742462146304644
:10AE1000FFF718FF09900028B8D1D9E7424621462C
:10AE20003046FFF70FFF0990B0E74FF0FF3309936B
:10AE3000002DB2D00027A9E72DE9F04F002487B0FC
:10AE4000924606AA894642F80C4D2C219846109D40
:10AE5000FFF7DAFC074688B93E4B2B60039938466A
:10AE6000FFF7BDFC07B0BDE8F08FD0F800B0726806
:10AE70005A451CD2304600F013FB0134039BA34219
:10AE8000ECD957F824602F213046FFF7DAFBA8B938
:10AE90002B46304642465146FFF740FD2B6806469A
:10AEA000002BE2D00028D9D000F0FAFAD6E75946B4
:10AEB0004846FFF70CFE0BF1010BD8E700232F21CA
:10AEC000304604AA0493FFF79FFC049906464B1EE4
:10AED000012B04D9204B2B60FFF781FCBEE74246D3
:10AEE0002B4651460068FFF719FD2A6883462AB1B0
:10AEF00008B100F0D5FA04993046EDE72D2130680D
:10AF0000FFF79FFB18B908F1FF32CBF804200023AC
:10AF100006A941F8043D7068FFF7A5FB059A00906B
:10AF20001AB10E4A58462A60E3E7DBF80020DBF846
:10AF30000410914205D230460499FFF750FC584660
:10AF400099E7114648460192FFF7C1FDDDE900325D
:10AF50001A44ECE72BCB01083DCB010862CB01087A
:10AF60002DE9FF4100230E460393144602B902ACBB
:10AF7000236048B90546564B236003992846FFF7DE
:10AF80002EFC04B0BDE8F08103AA2021FFF73CFCB1
:10AF9000039B0546062B02D04E4B2360EDE71A2299
:10AFA000002130460CF023F9009400223C23314666
:10AFB0002868FFF741FF2268002ADED100943C2375
:10AFC00006F108016868FFF737FF2268002AD4D12C
:10AFD0000094182306F11001A868FFF72DFF2368DD
:10AFE000002BCAD16869FFF71FFD07223A4968693B
:10AFF000FFF758FB80460CF0CFFF012806F113073E
:10B0000006D198F800303F2B04BF2A2388F800307F
:10B0100000220823394640460094FFF70DFF4046C2
:10B0200000F03EFA2268002AA7D107213846FFF730
:10B0300074FD30B111463846FFF749FD0721FFF78F
:10B0400059FDEF6806F1140838460CF0A5FF0128F9
:10B0500004D13B783F2B04BF2A233B7020230022DE
:10B06000414638460094FFF7E7FE00214046FFF7CF
:10B0700041FD2368002B80D12F693846FFF7D4FCAF
:10B0800000287FF47AAF38460D221449FFF70AFBF7
:10B09000074600283FF471AF183600940D230122B3
:10B0A0003146FFF7C9FE384600F0FAF9012421467F
:10B0B0003046FFF732FD30B1611E3046FFF707FD25
:10B0C0002146FFF717FD01340D2CF0D155E700BFE5
:10B0D0000ACA010822CA0108700000208C00002062
:10B0E000F0B58DB0CDE90023054628B94FF0FF300B
:10B0F0004FF0FF310DB0F0BD2422002103A80CF069
:10B1000076F803A968460BF051FF04460028EDD0FD
:10B110000CF050F94A1C08BFB0F1FF3F06460F463D
:10B12000E4D0626921462846FFF78CFD0028DDD176
:10B1300020460CF03FF94B1C08BFB0F1FF3FD5D0C3
:10B140008F4208BF864203D020460CF033F9D1E786
:10B1500023682046013323600CF02CF9013108BF2D
:10B16000B0F1FF3FC2D0626921462846FFF76AFD71
:10B170000028E9D0BAE770B53C258AB0DDE90E6455
:10B18000019496FBF5F405FB14640294182493FBD8
:10B19000F4F505FB1433CDE90330481E0C2190FB78
:10B1A000F1F301FB13010023CDE907339DF8403093
:10B1B000A2F26C7201A80591069209930CF0FAF8BC
:10B1C0000AB070BDF7B5044602A860E902230BF08F
:10B1D000DBFE0269037A551C426990F804C0077BC4
:10B1E00002F26C71067EC2690068A37000332070A1
:10B1F00018BF01232046013284F801C0E770257191
:10B20000A4F80510E6712272637203B0F0BD30B588
:10B21000457A85B0C4788378B0F805200179029525
:10B2200005780195407800902046FFF7A4FF05B00F
:10B2300030BD904271EB0303B4BF01200020704782
:10B24000032210B5104986B00B78013393FBF2F25C
:10B2500002EB42029B1A0D4A0B7052F8234002780F
:10B26000B0F80530049242781A2103928278029253
:10B27000C2780192027920460092054A0CF026FE1F
:10B28000204606B010BD00BFDE4900200CCC0108EE
:10B29000D1CB0108B1F1004F08BF00281FB502460D
:10B2A0000B4608D001A8FFF78DFF01A8FFF7C8FFE4
:10B2B00005B05DF804FB0148FAE700BF03CC0108C4
:10B2C0002DE9FF4703220D462B4900280B78044641
:10B2D00003F1010393FBF2F202EB4202A3EB020340
:10B2E000264A0B7052F8236075F100033EDA4FF0E6
:10B2F000010A444265EB4505214A002320462946C0
:10B300000BF044FC1E4A07460023204629460BF05A
:10B310003DFC104619464FF4616200230BF036FCE9
:10B320004FF4616280460023204629460BF02EFC34
:10B33000104619463C2200230BF028FC3C22814693
:10B340000023204629460BF021FCCDF80080CDE9F2
:10B3500001923B46BAF1000F0BD00A4A1A2130463F
:10B360000CF0B4FD304604B0BDE8F0874FF0000AA1
:10B37000C2E7054AF2E700BFDE4900200CCC010815
:10B3800080510100EFCB0108F0CB01080FB404B0ED
:10B39000704700000FB437B51B4C256855B9032220
:10B3A00029460120F6F7C8FA2B462A46294620608E
:10B3B000F6F7E6FA154D2A68013A03321ED86421E1
:10B3C0002068F6F7C9FC8022002111480BF00FFF1E
:10B3D00007AB069A80210E4801930DF079F97F287A
:10B3E00003DD0C490C480CF0CFFD2B68084898474A
:10B3F000002320681A461946F6F7C2FA03B0BDE8E2
:10B40000304004B0704700BF684A0020E049002087
:10B41000E849002082C70108634A00200FB410B534
:10B420000D4CA2B02268013A033210D825AB249A01
:10B43000802102A801930DF04BF97F2804DD074914
:10B440000DF183000CF0A0FD236802A8984722B0FC
:10B45000BDE8104004B07047E449002082C70108ED
:10B4600070B50446054E4518AC4200D170BD14F8C5
:10B47000011B3046FFF78EFFF6E700BF049E010870
:10B4800038B50C461546FFF785FF20462946FFF7DD
:10B49000E7FFBDE838400148FFF77CBFCBAC0108AF
:10B4A00010B5044670B1F8F755FA2046F8F7F6FAE9
:10B4B000F8F728F9BDE81040034A938801339380D8
:10B4C000F8F740B910BD00BFCC50002070B5214C3A
:10B4D0008AB0226806460132632A22601E4D0BDDC7
:10B4E000F7F74AFC0523002201A9F7F707FCF7F755
:10B4F0000FF9002328602360F7F70AF92B6803F59A
:10B500007A73984204D9F7F703F90023286023607F
:10B51000124A134C13781BB9236063600123137024
:10B52000F8F718FA3046F8F727FA054668B13246B8
:10B5300000210BF05CFEF8F7E5F823880133238047
:10B54000F8F700F928460AB070BD638801336380BC
:10B55000F8E700BF704A0020744A00206C4A0020BF
:10B56000CC500020A0F14103052B02D83738C0B2DF
:10B570007047A0F16103052B01D85738F7E7303841
:10B58000C0B20A2828BFFF2070470022013910B539
:10B590000144441E8C4204D014F8010F08B1002A63
:10B5A00001DA104610BDFFF7DDFF0F2802D840EA90
:10B5B0000212EFE74FF0FF32F3E700687047D0F870
:10B5C000010000BAC117704700687047006800BAF0
:10B5D0007047837842781B04007843EA02231843BB
:10B5E00070474278007840EA02207047027840783D
:10B5F00040EA022070470B12017043700B140916C9
:10B600008370C170042070470B1603700B144370D5
:10B610000B128370C170042070470370130E4370C7
:10B62000130C8370130AC3700271052070470B124C
:10B63000037041700220704738B505460C460CF087
:10B6400001FC611B013190FBF1F303FB1100284465
:10B6500038BD38B5451E15F8014F04B938BD0BF09B
:10B6600055FD23462044427802F00302012A08BF18
:10B6700020332B70EFE72DE9F04106460CF08CFCEF
:10B6800030B3002734180BF041FD14F8013C354667
:10B6900018444378621E19070DD42F463B78A4EB5B
:10B6A000050801355BB908F1010239463046BDE8AD
:10B6B000F0410BF083BD04F8017C1446E3E70BF086
:10B6C00025FD15F8013C184443781B07E5D4EAE74B
:10B6D000BDE8F08108B50CF04DFCB0FA80F04009EF
:10B6E00008BD000010B50446034B03604068F6F740
:10B6F0000DFD204610BD00BF68CC010810B5044602
:10B70000FFF7F0FF20460821FEF770FF204610BD2E
:10B7100038B5436804460D461BB90E210548F8F7B5
:10B720002DFA29466068F6F717FB431E5842584128
:10B7300038BD00BF18CC01084068F6F79BBC08B5BF
:10B74000002340681A461946F6F71AF9431E584274
:10B75000584108BD38B50D4600210B4B04464160E9
:10B76000036003220120F6F7E7F8606018B957215B
:10B770000648F8F703FA2DB1002360681A46194607
:10B78000F6F7FEF8204638BDC4BD010818CC010804
:10B79000014BDB68184700BF784A00200120704742
:10B7A00001B1096818B1806A431A5842584170477C
:10B7B00038B50C4B0546186800F02FFB10B9002374
:10B7C000184638BD4FF47A7403686C431A68A24275
:10B7D000F6D000F019FB0028F1D003681A689442F3
:10B7E000F6E700BF784A002010B5044618B9D22108
:10B7F0000748F8F7C3F9074B5B689847D4E9062375
:10B80000904271EB0304B4BF101A002010BD00BFBA
:10B81000A8CC0108784A00202DE9F849884604465A
:10B8200010B10369012B03D1E7211748F8F7A6F9F6
:10B83000D4E906BC5BEA0C0323D0D4E90867BBEB70
:10B8400006006CEB07010AF057FF05462069013836
:10B850000AF038FF014628460BF040F805464046FE
:10B860000AF030FF29460AF085FF29460AF078FEE3
:10B870000BF06CF9321847F1000310461946C4E981
:10B880000601BDE8F88900BFA8CC010841F658328E
:10B89000A0F55223A3F61833934224D8A0F55423DD
:10B8A000A3F1F902622A1ED96FF454729A18C62ABB
:10B8B00019D9A3F21353302B15D9104B984214D930
:10B8C00003F6B833984212D903F51673984210D98B
:10B8D00003F5167398420ED903F5E173984294BFAD
:10B8E0000520062070470020704701207047022085
:10B8F0007047032070470420704700BFE8320D00F6
:10B90000F8B5054618B9F3212248F8F737F9224E61
:10B91000306800F082FA00283BD0002D39D003684F
:10B920001A79AA4231D11F7B00F06EFA20BB87B38F
:10B93000062D03D940211748F8F720F9174B53F883
:10B94000354024BBFE211348F8F718F9306800F0A1
:10B9500064FA0646E8B17C4337683B79AB4204D1D0
:10B9600021463846FFF758FF3C61304600F04CFA5C
:10B9700006460028F0D10CE003681A79AA42D3D118
:10B980001B7B002BD0D00137CEE70027CCE7012C62
:10B99000DCD1F8BDA8CC0108784A002070CC0108A1
:10B9A00010B5074C206848B100F040FA30B120686B
:10B9B00000F033FA00F028FA0028FBD110BD00BFD8
:10B9C000784A0020F8B5114C0646227E0F4622B96F
:10B9D0004FF4B1710E48F8F7D1F8206810B900257E
:10B9E0002846F8BD0B4B002E08BF1E4600F015FA86
:10B9F00004460028F3D0256839462846B047002879
:10BA0000EED1204600F000FAF2E700BF784A0020AD
:10BA1000A8CC01089DB700082DE9F04F394C92469B
:10BA2000227E91B08346894622B94FF4C9713648C7
:10BA3000F8F7A4F8206820B90024204611B0BDE82A
:10BA4000F08F324BB9F1000F08BF994600F0E5F9CD
:10BA500080460028F0D00468237BDBB94FF0FF3626
:10BA600000240027404600F0CFF98046F8B9BAF12B
:10BA7000000F01D0CAF80060002EDED1012FDCD902
:10BA8000791E3046FFF7D8FD10AB03EB800050F86D
:10BA9000404CD2E7A3685B45E0DB00212046C84765
:10BAA0000028DBD02046FFF79FFE0646D9E7D8F8EE
:10BAB00000502B7B002BD5D0AB685B45D2DB00213F
:10BAC0002846C8470028CDD02846FFF78DFE38B954
:10BAD0000F2F9FBF10AB03EB870343F8405C013788
:10BAE0006CB186420AD8BDD1D4E90823D5E9080152
:10BAF000FFF79FFB002818BF2C46B3E706462C46ED
:10BB0000B0E700BF784A0020A8CC01089DB7000824
:10BB1000F8B50D46044620B940F2E1111A48F8F78D
:10BB20002DF8236923B94FF4F1711748F8F726F877
:10BB3000164B5B6898470F4606462069C4E90867BC
:10BB40000AF0C0FD29460AF015FE29460AF008FD54
:10BB50000AF0A0F90AA3D3E900230AF01DFB09F0BB
:10BB6000DBFE0AF089FC321847F100031946104643
:10BB7000C4E90601BDE8F840FFF712BFAFF300804B
:10BB80000000000080842E41A8CC0108784A0020E3
:10BB900008B5FFF77BFE003018BF012008BD00008C
:10BBA0000A4B10B51B7E044623B94FF407710848B1
:10BBB000F7F7E4FF44B1237B33B1002320792373EB
:10BBC000BDE81040FFF79CBE10BD00BF784A0020C2
:10BBD000A8CC01080A4B10B51B7E044623B94FF4CC
:10BBE0000A710848F7F7CAFF44B1237B33B9012330
:10BBF00020792373BDE81040FFF782BE10BD00BF5F
:10BC0000784A0020A8CC0108F8B5144E0546337ECA
:10BC100023B94FF40D711248F7F7B0FF306808B937
:10BC20000020F8BD002DFBD000F0F7F804460028F6
:10BC3000F6D023689D420CD12F792846FFF7A8FD46
:10BC40002146306800F000F93846FFF759FE012020
:10BC5000E7E7204600F0D8F8E8E700BF784A002080
:10BC6000A8CC01082DE9F8432A4D07462B7E8846CB
:10BC7000914623B940F2F9112748F7F77FFF38467C
:10BC8000FFF786FF18B900242046BDE8F883384640
:10BC9000FFF78EFD08B1FFF7B7FF2B7E1BB97621AA
:10BCA0001D48F7F76BFFAB68302098470446002823
:10BCB000E9D0302200210BF09AFA3846FFF7E6FD72
:10BCC0000646207118B9EB6820469847DBE706283E
:10BCD00003D940211048F7F751FF104B214603EBE1
:10BCE000C60253F83630526823614FF47A73A2606B
:10BCF0005F4300220023C4E9062301232760C4E92F
:10BD00000A892373286800F069F82079FFF7F8FDA5
:10BD1000BAE700BF784A0020A8CC010870CC01081F
:10BD200038B50A4C0546227E22B94FF41C710848EA
:10BD3000F7F724FF23682BB1064C29462046FFF76E
:10BD400041FE00B938BDFFF723FDF6E7784A002031
:10BD5000A8CC0108A1B70008014B187E704700BFAE
:10BD6000784A002084B070B504AC84E80F00104C11
:10BD7000237ECBB9251D04AE0FCE0FC533682B60D3
:10BD80000BB90C4B636123690BB90A4B2361E36860
:10BD90000BB1A3681BB9084BE360084BA36000F02C
:10BDA0000FF8012320602376BDE8704004B070478F
:10BDB000784A00208DB30008397101082971010803
:10BDC00010B50820FFF782FB0446F6F799FC002324
:10BDD000C4E90034F6F73AFD204610BD70B50546BB
:10BDE0000C200E46FFF772FB044660B10660F6F7C2
:10BDF00087FC002363606B68A3601C6004346C6084
:10BE0000F6F724FD012070BD10B50446F6F778FC66
:10BE10006468F6F71BFD204610BD10B50446F6F722
:10BE20006FFC2468F6F712FD204610BD10B50446DD
:10BE3000F6F766FC236800241BB9F6F707FD2046D9
:10BE400010BD01345B68F7E738B50C460546F6F7D8
:10BE500057FCD4E901324BB19A60A2681360F6F73F
:10BE6000F5FC2046BDE83840FFF71ABB6A60F4E7EE
:10BE700070B50446044E451814F8011B3046FFF710
:10BE800089FAAC42F8D170BD049E010870B5154620
:10BE90000022C0E901150270C0E90332C0E90522A1
:10BEA000C0E907224262DDE90412044600F11C06E3
:10BEB000F8F7D8FA38B929460748FFF76BFA2B216B
:10BEC0000648F7F75BFEDDE9042331462046F8F724
:10BED000B6FA204670BD00BF989D0108C39D0108B9
:10BEE000F0B50126044608270D468DB0694B6A4A15
:10BEF0003146009602A8F4F793F902A92046F9F713
:10BF000097FB02A8F4F72EF9644BCDE900571A46C7
:10BF100004210DEB0700FFF7B9FF0DEB07012046E9
:10BF2000F9F786FB0DEB0700F4F71CF9EB195C4AF7
:10BF30000197009304215B4B0DEB0700FFF7A6FF71
:10BF40000DEB07012046F9F773FB0DEB07001027F7
:10BF5000F4F708F9EB190093534B04211A460197A3
:10BF600002A8FFF793FF02A92046F9F761FB2035ED
:10BF700002A8F4F7F7F84D4B4D4A009504210197BC
:10BF800002A8FFF783FF02A92046F9F751FB02A898
:10BF9000F4F7E8F80C23474A00930221464B02A825
:10BFA000F4F716F902A92046F9F742FB02A8F4F7C4
:10BFB000D9F8424B424A3146009602A8F4F730F9CC
:10BFC00002A92046F9F734FB02A8F4F7CBF80322C4
:10BFD000002303923B4D3C4A3C4902A88DF80830AF
:10BFE0000495CDE90523CDE90733CDE909330B935A
:10BFF000F8F720FA38B929463548FFF7CBF9202160
:10C000003448F7F7BBFD0025304A09A902A8F8F724
:10C01000DBF902A92046F9F70BFB02A8F4F7A2F816
:10C020002D4B2E4A0095022102A8F4F7D1F802A95F
:10C030002046F9F7FDFA02A8F4F794F8284B294AAC
:10C040000095022102A8F4F7C3F802A92046F9F7E7
:10C05000EFFA02A8F4F786F80121234B234A009156
:10C0600002A8F4F7DDF802A92046F9F7E1FA02A8E0
:10C07000F4F778F81E4B1F4A0095022102A8F4F746
:10C08000A7F802A92046F9F7D3FA02A8F4F76AF84C
:10C090000DB0F0BDFACC0108A6B801080DCD01081D
:10C0A0007ED0010865D001081BCD010886D00108AB
:10C0B000B0D00108EDB7010822CD01087BCD010801
:10C0C00029B8010806B80108B7D00108A9B80108C5
:10C0D000989D0108C39D0108CCD001082DB8010826
:10C0E0000AD1010854B8010845D10108DEAB0108A6
:10C0F00061D101087CB8010830B504468DB0014615
:10C100007A4A6846F9F79FF8794A214603A8F9F771
:10C110009AF8784A214606A8F9F795F87649204614
:10C12000F9F788F805467548FFF734F90123039AB3
:10C1300002F11001914205D011F8010D002818BF3D
:10C140000023F7E7002B53D06D48FFF723F95DB3C9
:10C150006C48FFF71FF96C4A214609A8F9F773F8F4
:10C160006A48FFF717F908210098FFF781FE684831
:10C17000FFF710F908210998FFF77AFE6548FFF7E5
:10C1800009F910210698FFF773FE6348FFF702F9DB
:10C190000998069A009900F057FE09A8F8F71EFBC7
:10C1A0005E48FFF7F7F861E05D48FFF7F3F85D4898
:10C1B000FFF7F0F80699009800F0A4FD5A48FFF741
:10C1C000E9F8042100980844FFF752FE5748FFF7AA
:10C1D000E1F810215648FFF74BFE5648FFF7DAF812
:10C1E00010215548FFF744FE4B48FFF7D3F8D7E737
:10C1F000102206980AF0C8FF5049514B002808BF8A
:10C2000019465048FFF7C6F8002D3DD03D48FFF7CE
:10C21000C1F83D4A214609A8F9F715F84A48FFF741
:10C22000B9F808210098FFF723FE4848FFF7B2F855
:10C2300008210998FFF71CFE4548FFF7ABF81021CD
:10C240000398FFF715FE4348FFF7A4F8102106985E
:10C25000FFF70EFE3048FFF79DF80998039B069AFA
:10C26000009900F009FE09A8F8F7B8FA2A48FFF784
:10C2700091F806A8F8F7B2FA03A8F8F7AFFA6846FB
:10C28000F8F7ACFA0DB030BD2548FFF783F8324817
:10C29000FFF780F8039A0699009800F077FD22488E
:10C2A000FFF778F8042100980844FFF7E1FD2B48D8
:10C2B000FFF770F810211E48FFF7DAFD2848FFF756
:10C2C00069F810212748FFF7D3FD2748FFF762F8E8
:10C2D00010212648FFF7CCFD2548FFF75BF81648EC
:10C2E0001021FFF7C5FD0C485BE700BF0DCD01082D
:10C2F000B0D001081BCD0108A6B80108ADCD0108DA
:10C30000C4CD0108DFCD01087ED00108E5CD0108CC
:10C31000F6CD010808CE0108CBAC0108B0CE01086B
:10C3200028CE01082DCE01085FCE010871CE01088C
:10C33000680100209DCE010898010020CCAC0108C6
:10C3400096CD0108CFCE0108ECCE0108FECE010843
:10C3500011CF010831CF01087ACF0108B4CF01080D
:10C3600020D001087801002037D001088801002082
:10C370004ED0010810B5084CD4F82C211AB964210C
:10C380000648F7F7FBFBD4F82C010023BDE810406A
:10C3900003222021F6F748BEC00000208DD20108FC
:10C3A000F0B51F461446C7B005460E46F1220021DF
:10C3B00009A80AF01CFF09AA1021384602F03CF92E
:10C3C00020460BF0E9FD07461022002101A80AF0E3
:10C3D0000EFF102F3A46214628BF102201A80AF06E
:10C3E000E2FE09AA05A901A802F0A0F9324605A9B2
:10C3F00028460AF0D8FE47B0F0BD000038B50C4C16
:10C400000C4D94F83230022B0ED1082394F8FF2003
:10C41000D4F80011012002F0C5F86B6B002098479A
:10C42000042384F8303038BDEB6A98470123F8E7DD
:10C43000C00000207CE1010810B5044601F084F83A
:10C4400020B92046BDE8104001F054B810BD0000EE
:10C45000054B93F8212022B993F8350080F00100B4
:10C4600070470020704700BFC0000020F0B5702763
:10C470009DB006460D463A46002168460AF0B7FED2
:10C4800008212B460DEB010004AC0B4AFFF788FF97
:10C490002B462046094A102108ADFFF781FF94E89A
:10C4A0000F0085E80F003A46694630460AF07BFEE9
:10C4B00030461DB0F0BD00BF7ED2010886D2010813
:10C4C00084B070B58AB00EAC84E80F00754C4FF4A0
:10C4D0009C722546002120460EAE0AF088FE0FCE43
:10C4E0000FC596E8030014AE85E803000FCE04F1F3
:10C4F00018050FC533682B600E9B0BB96A4B236080
:10C500000F9B0BB9684B2360109B23B94FF4A971A3
:10C510006648F7F733FB129B23B94FF4AB716348BE
:10C52000F7F72CFB119B23B94FF4AD715F48F7F778
:10C5300025FB139B23B94FF4AF715C48F7F71EFB43
:10C54000A3690BB90323A361E3690BB90A23E36170
:10C5500094F8233013B9012384F8233001F0B8FD97
:10C5600094F8243013B9012384F8243001F0A8FD95
:10C57000A36A0BB94E4BA36201F096FD06F016F9C3
:10C58000C4F828010138033004D963684948984742
:10C5900000207FE0032200210120F5F7CDF9C4F847
:10C5A000300120B940F287114048F7F7E7FA00223E
:10C5B0000421E069F5F7C0F9606420B940F28B11FD
:10C5C0003A48F7F7DBFA00220421E069F5F7B4F9FD
:10C5D000A06420B94FF4C7713448F7F7CFFA0022AE
:10C5E00004210120F5F7A8F9E06420B940F2911187
:10C5F0002E48F7F7C3FA082384F80931042384F896
:10C600000A31002384F83630012384F80D31FFF716
:10C61000A3FB05AD68B9A368226905932368079257
:10C620000893E26863680692009395E80F00FFF7AD
:10C6300099FB01F073FD23681F4E0793636806F1B1
:10C64000A0020893236904960693E368DC360593F9
:10C650000AAB43F81C2D93E803008DE8030095E82E
:10C660000F0002F0EBF90196A3694FF4CD7200932D
:10C67000124901231248F5F729FE012805460ED17B
:10C68000002303220421D4F82C01F6F7CDFC284620
:10C6900084F834500AB0BDE8704004B07047636855
:10C6A000084874E7C00000208DB300088DD201084F
:10C6B00008E6D333B0D1010810010020E3D101080E
:10C6C00025C80008EBD1010810B50F4CD4F82C3167
:10C6D00023B94FF4DF710D48F7F750FA0023032216
:10C6E0000421D4F82C01F6F79FFC42F21071D4F823
:10C6F0003001F5F731FB0023D4F830011A46BDE8CC
:10C7000010401946F5F73CB9C00000208DD2010851
:10C7100038B50E4DD5F8303123B940F2CF110C4861
:10C72000F7F72CFA0021D5F83001F5F715FB0128B1
:10C73000044608D10023D5F830011A461946F5F70A
:10C740001FF9204638BD0020FCE700BFC0000020D4
:10C750008DD2010810B5FFF7DBFF68B1074C00234D
:10C76000D4F82C0103220821F6F75EFCD4F82C0142
:10C77000BDE81040F5F742BF10BD00BFC00000206B
:10C78000014BD863704700BFC0000020002307B5ED
:10C7900002A941F8043D044B0246D86CF5F74AFA69
:10C7A000019803B05DF804FBC000002038B5FFF726
:10C7B000AFFF194D044620B16B6818489847002018
:10C7C00038BD686CF5F756FCEB698342F7D3214618
:10C7D000204602F063F905460028F0D0047000F00E
:10C7E00077FE044618B9284602F090F9E7E70C4AAC
:10C7F00013680133136063B9136801331360636016
:10C8000001236370032320462370FFF715FE606841
:10C81000D6E71368F3E700BFC00000201BD2010871
:10C82000944A00202DE9F8430123604C604F614E8B
:10C8300084F830300A235E4A4FF0FF310020F6F7CB
:10C84000AFFB01286AD1386843071AD5337833B172
:10C8500005F010FF002005F061FF00233370F6F7AC
:10C8600051FFF6F76FFF022384F830300023D4F82D
:10C8700030011A461946F5F783F80020F6F712F949
:10C88000D8E710F0080521D033787BB941F2883021
:10C8900005F01CFF18B9A0214748F7F76FF9474882
:10C8A00005F03CFF01233370FFF7A8FD0020F6F7E9
:10C8B000A9FC4FF4FA61D4F83001F5F74DFA0028DD
:10C8C000B8D1A7213C48F7F759F9B3E710F0200099
:10C8D00043D03378FBB194F83030042B1BD1DFF810
:10C8E000E4802A464146D4F82801F5F7E5FA012804
:10C8F000814610D198F80030072B22D1284600F04D
:10C90000E7FD40B10522C0E90155056180F80190BD
:10C910000270FFF791FD0020F6F774FC3378002BCE
:10C9200088D000F029FE0546002883D0032384F830
:10C9300030300378052B35D8DFE803F01219192AB7
:10C940002A312A464146D4F82801F5F773F901281F
:10C95000E1D1404605F0E8FEDDE7F6F753FC69E774
:10C96000D6211548F7F70AF9FFF748FD62E7FFF708
:10C970006FFD38B9284600F0A3FA60B1284600F0F0
:10C98000B9FDF1E72846FFF757FDFFF70FFFEBE78B
:10C9900001F0C2F9F1E72846FFF74EFDE4E700F0A9
:10C9A00067FDEBE7636806489847E7E7C0000020AB
:10C9B000A84A0020984A00208DD2010875C30008BB
:10C9C00090D101089C4A0020024B93F8FC0001F032
:10C9D0005FBD00BFC0000020F0B585B007460C4623
:10C9E0001546ADF80430FFF793FE3E4E28B173684C
:10C9F0003D489847002005B0F0BD706CF5F73AFB54
:10CA0000F3698342F6D3FFF7DFFF8442F2D8002DAB
:10CA100045D1002CEED12146384602F03FF80446BD
:10CA20000028E7D09DF80530002B3BD0042323706D
:10CA30009DF804303BB10D2304A901F8043D012207
:10CA4000204600F0D5FE96F8312096F83230934219
:10CA500003D196F83330934217D02023022A18BF0F
:10CA600000228DF80C3094F8783003A90BBF43F006
:10CA7000040343F001038DF80D208DF80D202046AE
:10CA800084F87830022200F0B3FE6577204600F08B
:10CA90001FFD054640B9204602F038F8AAE7DF2D11
:10CAA000A8D8B8E70223C2E70023104A83601368BE
:10CAB0000133136093B91368013313606B600A9BF1
:10CAC00028462B6101236B702B7000F025FD38B9CF
:10CAD000284600F00FFD736805488AE71368EDE704
:10CAE000686888E7C00000201BD20108944A002033
:10CAF00056D20108082808BF0120034B83F8230001
:10CB000083F8FC00704700BFC0000020024B83F890
:10CB1000240083F8FD007047C000002008B5FEF730
:10CB200055FD014B586508BDC0000020034630B5D7
:10CB3000054C00F11005224618685968083303C2F5
:10CB4000AB421446F7D130BD88010020034630B512
:10CB5000054C00F11005224618685968083303C2D5
:10CB6000AB421446F7D130BD78010020034630B502
:10CB7000054C00F11005224618685968083303C2B5
:10CB8000AB421446F7D130BD68010020034630B5F2
:10CB9000054C00F11005224618685968083303C295
:10CBA000AB421446F7D130BD9801002010B50446C1
:10CBB000FFF7BCFF2046FFF7C9FF2046BDE8104045
:10CBC000FFF7D4BF30B51025C3B0224CF1220021AD
:10CBD00005A80AF00CFB2A46002101A80AF007FB71
:10CBE00094F8673005AA8DF8053094F86630294628
:10CBF0008DF8063094F8653004F178008DF8073030
:10CC000094F864308DF8083094F863308DF809306A
:10CC100094F862308DF80A3094F861308DF80B305A
:10CC200094F860308DF80C3001F006FD052305AA5C
:10CC300004F1980101A88DF8043001F077FD062376
:10CC400005AA04F1880101A88DF8043001F06EFDF9
:10CC500043B030BDC00000200246024B006851685E
:10CC600003C37047180100200246024B0068516858
:10CC700003C3704720010020034630B5054C00F186
:10CC80001005224618685968083303C2AB4214469F
:10CC9000F7D130BD28010020034630B5054C00F126
:10CCA0001005224618685968083303C2AB4214467F
:10CCB000F7D130BD38010020014B83F822007047C6
:10CCC000C0000020014B83F831007047C0000020F5
:10CCD000014B1864704700BFC000002013B500244A
:10CCE000064B02AA42F8044D054993F8FD00FEF7F1
:10CCF00093FE2146019802B010BD00BFC000002085
:10CD0000B1CE000830B50430C7B00D46FFF706FFBE
:10CD10001C4B0DF1050203F10C0153F8040B8B427F
:10CD200042F8040BF9D11B880124138000238DF8ED
:10CD30001330022309AA102128468DF8043001F08F
:10CD40007BFC09AA05A901A801F0F0FC05A8FFF7E2
:10CD50001DFF09AA102128468DF8044001F06CFC43
:10CD600009AA05A901A801F0E1FC05A8FFF71EFF2B
:10CD70001022054B83F8214083F8202083F85020AF
:10CD800047B030BD47D20108C000002030B50430A4
:10CD9000C7B00C461546FFF7C1FE294B0DF1050241
:10CDA00003F10C0153F8040B8B4242F8040BF9D148
:10CDB0001B882046138000238DF8133002230124A2
:10CDC00009AA10218DF8043001F036FC09AA05A942
:10CDD00001A801F0ABFC05A8FFF7D8FE09AA1021B5
:10CDE00028468DF8044001F027FC09AA05A901A8EE
:10CDF00001F09CFC05A8FFF799FE032309AA05A9E9
:10CE000001A88DF8043001F091FC05A8FFF79EFE03
:10CE1000042309AA0DEB030005A98DF8043001F0E5
:10CE200085FC05A8FFF7A2FE1122064B83F82140DE
:10CE300083F8202083F8502083F8074147B030BDA5
:10CE400047D20108C000002038B50D461446FFF750
:10CE500003FF2846FFF708FF2046FFF70DFF204697
:10CE6000FFF71AFF0022034B83F82120102283F8DA
:10CE7000202038BDC000002070B50E4615461C4667
:10CE8000FFF7EAFE3046FFF7EFFE2846FFF7F4FE15
:10CE90002046FFF701FFBDE870400022034B83F8F6
:10CEA0002120112283F82020FFF78CBEC000002033
:10CEB00028B1836A012B01D1007B704700207047A5
:10CEC0002DE9F04F054689B010B10378012B03D04E
:10CED0001C218448F6F752FE6B691BB91D2181485D
:10CEE000F6F74CFE6B691B78042B05D0022B03D0A0
:10CEF0001E217C48F6F742FE00267B4C08AA94F8D7
:10CF0000FF3094F8FD800293D4F8003142F80C6DA4
:10CF10007649404694F8FCB094F8FEA00393FEF7DF
:10CF20007BFD074638B9284600F08AFB01273846C2
:10CF300009B0BDE8F08F059B8BB1FEF731FD059977
:10CF4000042904D9284600F0B3FB0027EFE768481E
:10CF500041434FF47A70B1FBF0F0F5F72BFDAB686D
:10CF60000133012BAB600FD1D4F8F0306869013385
:10CF7000C4F8F03094F80831013384F8083100F037
:10CF8000F3FB686900F054FC636D6E697360D4F85C
:10CF9000F030738194F80431002B63D0002384F8BF
:10CFA0000431337A43F00403337294F8FC3038468A
:10CFB00086F87C3001F0F4F886F87D00012168697C
:10CFC00000F0E8FB94F80D214FF47A7312F00F0291
:10CFD00008BF012200265A4307AB019306AB00931A
:10CFE000394602F57A736869069600F05DF90746DE
:10CFF000002898D0F5F78CFBE860069860B13146C0
:10D0000000F0C8FB069B1B78052B04BF012384F8A6
:10D010000431002384F80631069800F081FBDDE935
:10D02000060100F029FE069BFBB11B7A13F00403F6
:10D030002FD0B94694F80B31AB606A691278022A96
:10D0400002D194F80B21AA6000F0AEFA064610BB9C
:10D050008A212448F6F792FD264B274A8B21214846
:10D0600009F04EFFA6F87A309FE79946ECE7314683
:10D07000686898476420F5F79DFC304600F0A4FAF4
:10D0800094F80B31AA689A42BFF451AF032333706E
:10D090005BE79946D1E78022696918300AF083F886
:10D0A00000229DF808300699F373039BC6F8981088
:10D0B00029787272336194F83530C6F88020337560
:10D0C0002B6986F80CB086F80D8086F80EA03270B9
:10D0D000717086F80890002BC9D1304600F08EFAA6
:10D0E000CEE700BFE3D20108C0000020B1CE0008A7
:10D0F00040420F0028D30108D5D201082DE9F043A2
:10D1000085B006460C468DF80F202BB101220DF19B
:10D110000F01002005F074FEF5F7FAFA1C4B1D4DC7
:10D12000DFF878809DF80F1007469B6A20469847E5
:10D1300041F288322946D8F82801F4F77BFD28B35C
:10D140002B78012B1DD12846AC6805F0EDFA4FF481
:10D150007A70A4EB070909FB000009F0B3FA014655
:10D160003046FEF7D5FC9DF80F10CDE90049D8F800
:10D1700000503B4632680848A847204605B0BDE845
:10D18000F083284605F0D0FA0024F6E70446F4E7D9
:10D190007CE10108AC4A0020D4D30108C000002083
:10D1A0002DE9F84F394E9846736B0546894614466B
:10D1B0004FF47A7A9847DFF8DCB0354F0AFB05F276
:10D1C00002F59C328032B2FBFAF23249D7F82801DC
:10D1D000F4F730FD20B9336B98474FF0FF302FE064
:10D1E0009BF80030072B07D1584605F09DFA4FF405
:10D1F0007A6505F089FDE1E7032B366B22D1DBF878
:10D20000045028792968844228BF044648462246AB
:10D2100009F0C9FF3F6895F90830B5F90620A988DB
:10D220001D48B847B8F1000F05D0EB88A8F80030CA
:10D230002B7A88F80230174805F076FAB047204676
:10D24000BDE8F88F042B0BD1124805F06DFAB047FA
:10D250003C68F5F75DFA01461048A0470020EFE76B
:10D26000052B0AD10B4805F05FFAB0473C68F5F78B
:10D270004FFA01460A48A047AFE7D3210948F6F71D
:10D280007DFC044805F050FAB047A6E77CE10108B0
:10D29000C0000020B84A002039D3010863D3010838
:10D2A0007BD3010891D301082DE9F04FC9B089461D
:10D2B000174608A9FF2202901E46DDF84C8101F0B6
:10D2C0003FFC824618B9002049B0BDE8F08F634C9E
:10D2D000D9F8002094F8FC1094F8FE5008468D42CE
:10D2E0009ABF4D1BEDB20025D4F800B00592049111
:10D2F00001F07AF8039094F8FD0001F08BF8DDE975
:10D300000412039B00905648D847D9F800202846BD
:10D31000D4F800B0039201F067F8039A0346294657
:10D320005048D84794F8FF10D4F800210846D4F8A4
:10D3300000B00492039101F057F8DDE903120346AF
:10D340004948D84794F8FD3094F8FC20D9F80010EB
:10D35000002001F027F90023524608A94846FFF7AC
:10D36000CDFE04460028AED0029B93F8783013F02F
:10D37000050F0BD013F0040F0CBF00220222374B15
:10D3800093F83210914218BF83F83220FF22002117
:10D3900008A809F02CFFD9F800104FF47A792A4632
:10D3A0000823012001F0FEF809FB07F1A1F51C415B
:10D3B0004039B1FBF9F106A80694F5F7BBFAFF2254
:10D3C000434608A94FF44D70FFF7EAFE421C05469C
:10D3D0003FF479AF002821491ADD0E68F5F798F976
:10D3E0002346024629462148B047B8F1000F02D033
:10D3F000012388F803300023529A9D42136005DD13
:10D40000E9B208A801F00EFF529B186001205BE70B
:10D4100091F8FF200823D1F80011012001F0C2F893
:10D4200009FB06F1A1F51C414039B1FBF9F107A850
:10D430000794F5F77FFA4346FF2208A94FF44D7091
:10D44000FFF7AEFE431C05463FF43DAF0028D2DD9A
:10D45000B8F1000FCFD00223CBE700BFC0000020FF
:10D460004BD401087ED40108A5D40108CCD401080E
:10D4700070B5C2B001ABFF2202A94FF47A60FFF78A
:10D480008FFE061E1EDD114DF1B26A6D02A801F07D
:10D4900099FC0446B0B10378052B01D0032B0DD1C4
:10D4A0000021204600F076F9204600F039F92046A8
:10D4B000019900F0E1FB2B6C204613B901F026FB2B
:10D4C00000E09847304642B070BD00BFC000002069
:10D4D00038B5074B0546DB6818209847044620B14D
:10D4E0001422002109F083FE6561204638BD00BF8B
:10D4F000C000002010B5044650B1406901F006FBA1
:10D5000000236361034B2046BDE810401B691847A8
:10D5100010BD00BFC0000020037807B5052B4FF0F9
:10D52000000302A941F8040D06481A460CBF806C9E
:10D53000406CF4F725FA431E5842584103B05DF899
:10D5400004FB00BFC000002007B5037802A941F822
:10D55000040D0848052B4FF000024FF001030CBFEB
:10D56000806C406CF4F70CFA431E5842584103B0EB
:10D570005DF804FBC000002037B5002202AC094D65
:10D5800044F8042D2146A86CF4F754FB019B33B9F1
:10D5900095F836201AB92146686CF4F74BFB0198D0
:10D5A00003B030BDC0000020064B10B5DB68A020E2
:10D5B0009847044618B1A022002109F018FE204621
:10D5C00010BD00BFC000002070B5044690B1D0F877
:10D5D0008000094D08B12B699847D4F8980020B114
:10D5E00001F094FA0023C4F898302B692046BDE876
:10D5F0007040184770BD00BFC00000201FB50E4C22
:10D600000190E06CF4F748FD024638B903A9E06CDC
:10D61000F4F710FB10B10398FFF7D6FF002301A920
:10D620001A46E06CF4F7ACF920B94FF4B471034832
:10D63000F6F7A4FA04B010BDC000002091D3010891
:10D64000F8B50423437003780546032B0ABF144B37
:10D650000469DC6BFFF7A8FF0646B0B940F277110A
:10D660001048F6F78BFA104B104A4FF4BC710D4876
:10D6700009F046FC31466868A0473046FFF7A4FF32
:10D68000FA20F5F797F93846F8BD01272B7807708F
:10D690004370002CEED1FFF7B1FF2046F4E700BF46
:10D6A000C000002091D3010831D3010807D401083C
:10D6B000F8B503780646032B08BF154B0F460CBF81
:10D6C000DC6B0469FFF770FF0546B0B94FF4C87111
:10D6D0001048F6F753FA104B104A40F291110D48DA
:10D6E00009F00EFC29467068A0472846FFF76CFF3A
:10D6F000FA20F5F75FF90120F8BD022303703378B3
:10D7000047604370002CEDD1FFF778FF2046F3E728
:10D71000C000002091D3010831D3010823D40108AF
:10D7200008B5104A10B1002382F8083192F822306F
:10D73000BBB192F8083192F809118B4211D95B1AEA
:10D7400092F80A1193FBF1F201FB12334BB900F08E
:10D75000C7FC30B900F0D2FC18B9BDE8084000F0B1
:10D76000DDBC08BDC0000020094B93F822206AB13F
:10D77000027A42F00102027293F8082193F809310B
:10D780009A4282BF037A43F002030372704700BFDC
:10D79000C000002070470000064A1378FD2BDFBF51
:10D7A00000780549C8540133DABF01201370002006
:10D7B000704700BFC54B0020C64A002038B1007832
:10D7C000032803D0431F5842584170470120704737
:10D7D000052307B502A800F8013DFFF7DDFF034868
:10D7E000FFF7DAFF03B05DF804FB00BFC44A002076
:10D7F000037A70B51B09D61804460F2E00F10C00F1
:10D800001546184409DC09F0CEFC0120237A05EB0B
:10D81000131565F30713237270BDC3F10F0209F0EE
:10D82000C2FC237A002043F0F0032372F4E70000E7
:10D8300037B5114C0546227822B11049FFF7D8FFC1
:10D84000002323700E4C94F806213AB1082302A954
:10D8500001F8043D01222846FFF7CAFF94F807317A
:10D8600043B140F2011302A921F8043D02222846E7
:10D87000FFF7BEFF03B030BDC54B0020C64A0020F5
:10D88000C00000200122044B00F00F0083F80D01BE
:10D8900083F80621704700BFC00000200000000090
:10D8A0002DE9F04F17461E464FF000088BB0CDE92A
:10D8B00001019DF85050C04CA84502D30BB0BDE803
:10D8C000F08F16F8083006EB080A013B1F2B00F218
:10D8D000CE81DFE813F02000CC012C006601DC00D3
:10D8E000C0001E01600166014701CC01790194006E
:10D8F00092019501CC01CC01CC01CC01CC01CC0131
:10D90000CC01CC01CC01CC01CC01CC01CC01CC01AF
:10D91000CC01CC01B701A5EB0803DBB2012B4FF022
:10D92000000920D084F807914FF002091BE04FF066
:10D930000009A5EB080B5FFA8BFB8DF81C9009F131
:10D9400004035B4503DA1AF80930032B0DD0B9F153
:10D95000000F08D003230AA800F8083DFFF71CFFBA
:10D9600007A8FFF719FFC1448AE00AEB09014B78C9
:10D9700009F102001A09504403F00F0305910492C3
:10D980000393FDF72EFE0599049A097909F105091B
:10D99000062AC1F3021C5FFA89F901F00F01039B0B
:10D9A00021D90F2A05D19DF81C2042F002028DF8E2
:10D9B0001C205A1E062A19D90F2B05D19DF81C30A0
:10D9C00043F004038DF81C3009B184F80B11BCF14D
:10D9D000000F0ED100F06EFC9DF81C3043F00103E7
:10D9E0008DF81C30ABE784F8FC20DCE784F8FD30D0
:10D9F000E4E7BCF1060FA2D14FF6FF70EAE7A5EB12
:10DA00000803DBB2052B40F22F810AF10100FDF77C
:10DA1000DBFD9AF905300021002B18DB62A3D3E966
:10DA2000002312184B4191469A46002394F80D2189
:10DA300019EB02004AEB0301022F02D1013041F140
:10DA40000001019BC3E91C014FF006098BE758A3B5
:10DA5000D3E90023E5E706230AA800F80C3DFFF709
:10DA60009BFE029B0DF1280903F01F0309F8083DF6
:10DA70005248FFF791FE4846FFF78EFE08F1010974
:10DA80005FFA89F9C8453FF419AFC84614E7A5EB1A
:10DA90000803DBB2042B40F2E780DAF80120DFF85C
:10DAA00024910892D2B2C2F3021384F8FE3099F89E
:10DAB0000030C2F30302052A43F0040394BF43F08D
:10DAC00002036FF341030DF1210098BF84F8FF209A
:10DAD00089F800304FF0640AFDF77BFD0AFB00FA7D
:10DAE000504605F013F978B199F80030C4F800A158
:10DAF00043F00103012289F80030314B1A70FFF71F
:10DB000067FE4FF005092EE799F8003060F3000337
:10DB1000F0E7A5EB0803DBB2052B40F2A5805346E6
:10DB200053F8010F9AF803101A799AF80430090291
:10DB300041EA03419AF802300890194364239AF8A5
:10DB4000010059438DF8242000F04CFB07238DF889
:10DB500018000AA800F80C3DFFF71EFE06A8FFF704
:10DB60001BFE71E7A5EB0803DBB2042B7CD9642113
:10DB7000DAF80100030A5943C0B200F065FB0A233A
:10DB80008DF81C000AA800F8083DFFF705FE07A85D
:10DB9000FFF702FEB5E79AF8010000F00F00FFF76B
:10DBA00071FE08F102096BE76E3DD512000000001E
:10DBB0006F3DD51200000000C0000020CC01002005
:10DBC000C54A0020C44A0020A5EB0803DBB2012BA4
:10DBD0004AD001239AF801200AA8110902F00F0285
:10DBE00003FA01F1934084F80A310C2384F80911F7
:10DBF00000F8083DFFF7D0FD96E608F103093FE77E
:10DC0000A5EB0803DBB2012B2ED0A3689AF8019094
:10DC100098470122174B8DF81C20C3E900014FEAF9
:10DC200019130A3302FA03F3C4F8183109F00F0389
:10DC3000C4F81C310F230AA800F8083DFFF7ACFD1B
:10DC400007A8D7E7A5EB0803DBB2012B0CD09AF8A5
:10DC500001300BB1022B07D194F833209A423FF4E4
:10DC600063AE84F833305FE64FF000097BE6C146CF
:10DC700008E700BFD001002030B585B0039104460D
:10DC8000174B30B91B7803B305B0BDE83040FFF740
:10DC90009FBD00259DF90E109DF80F201D70FFF708
:10DCA0008DFD90B10F48237A90F822502DB113F0DA
:10DCB000010518BF012580F805511B0907D0009305
:10DCC00004F10C032046FFF7EBFD05B030BD637F88
:10DCD000002BFAD1237F002BF7D00093A36EF1E73E
:10DCE000C54A0020C000002010B5044678B1836A00
:10DCF000012B0CD1C36A1BB910210648F5F73EFF72
:10DD0000E36A587802288CBF0020012010BD002053
:10DD1000FCE700BF00D501082DE9F04F054689B0AA
:10DD200018B10378033B012B03D92221C148F5F731
:10DD300025FF6B690BB11B781BB12321BD48F5F79B
:10DD40001DFF0027BC4C94F8FF3094F8FD8003932E
:10DD5000D4F8003194F8FCB0029394F8FEA000F0DF
:10DD6000AFF900F0B5F908AA42F80C7DB349404676
:10DD7000FDF752FE064620B92846FFF761FC012652
:10DD80000AE0059BA3B1FDF70BFE0599042907D90D
:10DD90002846FFF78DFC3E46304609B0BDE8F08FBF
:10DDA000A74841434FF47A70B1FBF0F0F4F702FE5C
:10DDB000AB6894F820200133102AAB602DD1012BE1
:10DDC00009D1D4F8F0300133C4F8F0309D4B5B69D1
:10DDD0009847A4F8E800B4F8E8300133A4F8E83034
:10DDE000002707AB019306AB0093314641F27073F5
:10DDF00041F28832686994F8FF90069784F8FF70C2
:10DE0000FFF752FA0646A8B92846FFF719FC06980C
:10DE100000F07CFE84F8FF90B1E7112A05D1636918
:10DE200089489847A4F8E800DAE750218148F5F7D7
:10DE3000A5FED5E7069A84F8FF9012B11378012B5E
:10DE400006D02846FFF7FCFB069800F05FFEA3E72C
:10DE500094F82030102B40F0A0801023002784F885
:10DE60005030069BDA68626503F15302002F00F020
:10DE7000A3801121DFF8D4C184F8501003F1630EA0
:10DE8000674610685168083203C77245BC46F7D12F
:10DE9000DFF8BCC103F1230203F1330E67461068BB
:10DEA0005168083203C77245BC46F7D1DFF8A4C1F8
:10DEB00003F1330203F1430E6746106851680832DC
:10DEC00003C77245BC46F7D1DFF88CC103F14302AA
:10DED00003F1530E674610685168083203C7724554
:10DEE000BC46F7D1544F9A68BA631A7CC2F3030256
:10DEF00087F8FF201A7CC2F3021287F8FE20587CB4
:10DF0000FFF7C0FC0022069897F83110437C1230CE
:10DF1000012B98BF87F8062111F0FD0F18BF87F875
:10DF20003120C7E93D22C7F8F02087F8322087F872
:10DF3000332000F0E1F9FDF733FD012384F835309B
:10DF4000FFF732FB802207466969183009F02BF988
:10DF50000023069AC7F88030C7F8982094F8352037
:10DF60007B723A753B709DF80C202B78FA737B70AE
:10DF7000029AE36B87F80CB087F80D8087F80EA043
:10DF80003A61002B52D03946686898476420F4F70C
:10DF900011FD3846FFF718FBFEE6112B07D192F86A
:10DFA0002270002F3FF459AF84F8503059E77D219B
:10DFB0002048F5F7E3FD54E71021DFF890C084F81E
:10DFC000501003F1630E674610685168083203C7AA
:10DFD0007245BC46F7D1DFF878C003F1230203F1A4
:10DFE000330E674610685168083203C77245BC4655
:10DFF000F7D1DFF860C003F1230203F1330E674667
:10E0000010685168083203C77245BC46F7D1DFF883
:10E0100048C003F1230203F1330E674610685168CC
:10E02000083203C77245BC46F7D15BE73846FFF7B5
:10E03000E5FAB1E600D50108C0000020E9DC0008DF
:10E0400040420F007CE101081801002098010020E7
:10E050008801002078010020680100204378827840
:10E060001B02007843EA024303430A20B3FBF0F0AB
:10E070007047000038B5044681B10D7884B1A36AB9
:10E08000012B0DD1E36A1BB95D210648F5F776FD3A
:10E09000E36A5878431B5842584138BDFF25EDE7E5
:10E0A0000020FAE78CD50108044B93F8252083F86B
:10E0B000FF209A6AC3F80021704700BFC00000200B
:10E0C000024B93F8242083F8FD207047C000002005
:10E0D000024B93F8232083F8FC207047C0000020F7
:10E0E000054B93F8242093F8FD1091423ABF01208C
:10E0F00083F8FD2000207047C0000020064A92F8F7
:10E10000FC3092F8231099423DBF03F1FF33012008
:10E1100082F8FC3000207047C000002010B5FFF7E7
:10E12000C3FF0120FDF7FCFD5023164C0121237095
:10E130000023224614486370FDF794FD18B932217C
:10E140001248F5F71BFD50230121114A1148A37015
:10E15000E170FDF787FD18B936210C48F5F70EFD83
:10E160005023237102230C4A01210C486371FDF7EF
:10E1700079FD28B9BDE810403A210448F5F7FEBC06
:10E1800010BD00BFD4500020043F0D008CD5010805
:10E19000D6500020CC3F0D00D850002094400D00F8
:10E1A000836A10B5012B044608D1C36A1BB94B2101
:10E1B0000348F5F7E3FCE36A587810BD0020FCE75C
:10E1C0008CD5010807B502A901F8010D0448FDF737
:10E1D000F9FB08B1FDF718FD03B05DF804FB00BFC3
:10E1E00075E000082DE9F0414FF47A769046B1FBD6
:10E1F000F6F6C8F30317052F044630468CBF0027F8
:10E2000001274FF00005FDF7C3FC18B10F2C8CBFA0
:10E210000020012067F3000560F3410505F00303CA
:10E22000032B0CD12046FFF7CDFF064B012103EB5A
:10E230004402547003F814803046FDF713FD28465D
:10E24000BDE8F081D45000200F282DE9F0410546AB
:10E250000F461FD8164B03EB40035C78231A5C4231
:10E260005C414FF47A78B7FBF8F0FDF791FC4FF082
:10E27000000360F3000364F3410303F00303032B83
:10E28000064609D04FF0000066F3000064F3410039
:10E29000BDE8F0810024E4E72846FFF793FF044A35
:10E2A000012102EB450208FB07F0FDF7DBFCE9E783
:10E2B000D4500020002373B5044602AD0D4E05F87E
:10E2C000013D9DF807300F2B01D902B070BD2946E2
:10E2D0003046FDF777FB18B1E30708D5FDF77AFC68
:10E2E0009DF80730640801338DF80730E9E7FDF742
:10E2F00057FCF5E775E0000838B504460320FFF742
:10E3000061FF0420FFF75EFF0520FFF75BFF06209B
:10E31000FFF758FF0720FFF755FF2046FFF79EFE47
:10E320000546FDF735FC48B15023294A0121937178
:10E330000323063253702846FDF794FCE01CFFF7D8
:10E340008DFE0546FDF724FC48B15023204A0121EB
:10E3500013720423083253702846FDF783FCA01D76
:10E36000FFF77CFE0546FDF713FC48B15023184A21
:10E370000121937205230A3253702846FDF772FC7F
:10E3800004F10900FFF76AFE0546FDF701FC48B1FC
:10E3900050230F4A0121137306230C325370284671
:10E3A000FDF760FC04F10C00FFF758FE0446FDF792
:10E3B000EFFB58B15023064A204693730723D373CB
:10E3C0000121BDE838400E32FDF74CBC38BD00BF1E
:10E3D000D45000200738C0B205289ABF014B185C02
:10E3E0000820704743D5010806289ABF014B185CE6
:10E3F0000020704749D50108052804D9062803489C
:10E4000018BF002070470248704700BF90D003003B
:10E4100048E80100072810B5044604D940F243112A
:10E420000348F5F7ABFB034B13F9240010BD00BF05
:10E430008CD5010850D50108142810B5044613DD09
:10E440004FF4A4711148F5F799FB062C14DD082C44
:10E4500014DD0A2C14DD0C2C14DD0E2C14DD152C0F
:10E46000B4BF0020082010BD022803DD0428ECDC26
:10E470000620F8E70720F6E70520F4E70420F2E796
:10E480000320F0E70220EEE70120ECE78CD501083D
:10E4900008B50F280DD8DFE800F0181818081A1A68
:10E4A0001A0A0A0C0C0C0C0C0C0A732008BD002074
:10E4B000FCE74FF4C1710748F5F760FB064B074ACC
:10E4C00040F28311034808F01BFD3320EEE7DE2005
:10E4D000ECE700BF8CD5010815A9010870D501082B
:10E4E0002DE9F0468DB0924699462A4A149B07467C
:10E4F00093420C4608D0284A934203D0A6212748CD
:10E50000F5F73CFB002600E00126254DEB6A984715
:10E510002046EB689847012F4FF0000422D10823D2
:10E520000A22CDE90132AB6931460B93CDE9087778
:10E53000CDE90644CDE90444039400943B464A46A1
:10E5400002200B9EB0472146FF2004F051F908201D
:10E5500004F044F9342139202B6C0B930DB0BDE845
:10E56000F04618474FF47A630127CDE907430823A3
:10E57000CDE90173EB69CDE905440B93CDE9034780
:10E5800022465146CDF80090334602200B9CA0470E
:10E590003946D9E790D0030048E80100D1D50108F9
:10E5A0007CE101082DE9F3410446104615460E466C
:10E5B0009846FFF721FF07462846FFF715FFC5B22B
:10E5C0001DB9C5210948F5F7D9FA64B94046FFF7E6
:10E5D00021FF024600972B4631462046FFF780FF79
:10E5E00002B0BDE8F0810022F4E700BFD1D50108F8
:10E5F0000A680368534003604A68436853404360B5
:10E600008A68836853408360CA68C3685340C360A4
:10E6100070470B6810B514686340036054684B681A
:10E620006340436094688B6863408360CB68D268C2
:10E630005340C36010BD0000A1F11003DBB2102BEA
:10E640002DE9F0470C46154608D84FF0010909FAA4
:10E6500003F303F0013323F080732BB90023FF2071
:10E6600085F8F030BDE8F0870A460146284608F0F4
:10E670009AFD04F11C0E4FEA8E0E5FFA8EFE4FEAF1
:10E680001E13013B85F8F03023462749B3FBF4F213
:10E6900004FB1232E81812F0FF0210F804AC10F874
:10E6A00003CC10F8027C10F8016C32D111F80C8008
:10E6B0004FEAD91289EA080811F807C08F5D11F8EE
:10E6C0000A604FEA420A5244C24602EBC20282EAA0
:10E6D00049025FFA82F91A1BD2B215F802802A4465
:10E6E0008AEA080A05F803A092F8018004338CEA4C
:10E6F000080C80F801C092F802C0DBB287EA0C0770
:10E700008770D2789E4586EA0206C670BED8002081
:10E71000A8E7182CDFD9102A01BF11F80AA011F8B8
:10E720000CC0CF5D8E5DD6E713D801082DE9F04F00
:10E7300092F8F030A1B01A911892002B00F05D8190
:10E7400001461CA8FFF765FF4FF00108AC4CAD4D2A
:10E75000AD4E189B9DF875E003EB081319939DF8D7
:10E7600070309DF87AA00093009A9DF87F90A05C8D
:10E770009DF8742014F80A100192019F9DF87920E9
:10E78000E75D02920697029F9DF87E20E75D039267
:10E790000797A25C9DF87870049208979DF8732003
:10E7A0009DF87D70059214F8093014F80EC0A25C33
:10E7B00009979DF872700A97E75D0B979DF877703F
:10E7C0000C97E75D0D97089FE75D0E97099FE75D42
:10E7D0000F979DF87C7010979DF8717011979DF8B8
:10E7E00076701297E75D13979DF87B701497E75D3D
:10E7F0001597109FE75D1697119FE75D1797189F74
:10E8000097F8F07047453ED88DF870009DF81800D5
:10E810008DF872108DF874009DF82C109DF838005A
:10E820008DF87A108DF878009DF810109DF858003A
:10E830008DF876108DF87C009DF84C109DF81C002A
:10E840008DF87E108DF875009DF854109DF83C00F1
:10E850008DF87F108DF879009DF834109DF85C00DC
:10E860008DF87B108DF87D008DF877201A98199A15
:10E870001CA98DF871C08DF87330FFF7CAFE002017
:10E8800021B0BDE8F08F81EA03071B97009F43404A
:10E8900015F807B01B9F80EA0C008BEA070716F8F3
:10E8A0000EB081EA0C0187EA0B078DF8707015F83D
:10E8B0000E707B4016F80A707B408DF8713015F8A9
:10E8C0000A30584016F809305840009B8DF8720005
:10E8D00016F803C0049B8CEA010115F809C05340E7
:10E8E00081EA0C018DF8731001991CA8695C4B40FA
:10E8F0000299715C4B408DF87430069B5A40029B24
:10E90000EB5C5A40039BF35C5A408DF87520DDE9BF
:10E9100006325340039AAA5C5340059AB25C5340B6
:10E920008DF87630079A049B5340019AB25C5340AD
:10E93000059AAA5C53408DF877300D9A0B9B534093
:10E94000089AAA5C5340099AB25C53408DF878301B
:10E95000DDE90D325340099AAA5C53400A9AB25C31
:10E9600053408DF87930DDE90E3253400A9AAA5CA3
:10E9700053400C9AB25C53408DF87A300B9B0F9A3F
:10E980005340089AB25C53400C9AAA5C53408DF8ED
:10E990007B30159A139B5340109AAA5C5340119AEE
:10E9A000B25C53408DF87C30DDE915325340119A4A
:10E9B000AA5C5340129AB25C53408DF87D30DDE979
:10E9C00016325340129AAA5C5340149AB25C5340D8
:10E9D0008DF87E30179A139B5340109AB25C5340C7
:10E9E000149AAA5C199953408DF87F30FFF700FE06
:10E9F00008F101035FFA83F8ABE6FF2040E700BFB0
:10EA000013D8010813D6010813D70108006870470E
:10EA100082B0034660B16A4659680068013B03C290
:10EA200007221DF8021012F1FF3203F8011FF8D27D
:10EA300002B070470FB404B07047000030B585B025
:10EA40006D4685E80F00104C95E80F0084E80F0034
:10EA500004F1100208A903C982E803000BB90B4BAB
:10EA6000E360A3680BB9094BA36063680BB123682B
:10EA700033B9A36806489847064B6360064B23608A
:10EA80000123237605B030BDC84B002035EA0008CD
:10EA900089D9010839710108297101082DE9F0416E
:10EAA000184D80462B7E0E461BB973211648F5F78C
:10EAB00065F8DE2E03D974211348F5F75FF82B684B
:10EAC00080209847044680B18022002108F08FFB07
:10EAD000B8F1000F12D08EB12B6830469847074628
:10EAE00030B920466B6898473C462046BDE8F08127
:10EAF0003246414608F057FB2677A766002363702D
:10EB0000F3E700BFC84B00203CD9010870B50A4CA0
:10EB10000546237E1BB98F210848F5F72FF855B11C
:10EB2000A86E636810B198470023AB6663682846F7
:10EB3000BDE87040184770BDC84B00203CD90108A3
:10EB40002DE9F0479C4B17461A7E92B005460E46BB
:10EB500098461AB9A7219948F5F710F8032F01D85C
:10EB60000024D8E02A786B7843EA421333702B787C
:10EB7000022B02D0042B40F08D800023042F8DF84F
:10EB80002630EDD06B6873706B681B0AB370EB882E
:10EB9000F370EB7933716B68CDF822309DF8263035
:10EBA000002B40F0C180052FDAD006242A7AC2F368
:10EBB000400302F001019B0143EAC11343EA12132F
:10EBC000C2F3800243EA4213737195F808904FEA4A
:10EBD0001919631C9F42C3DD6A89DBB232556A8909
:10EBE0000234120AF254D8F810301A886B899A420B
:10EBF00004D040F247117148F4F7C0FFD8F8142050
:10EC0000D8F8103011781B6810290A930DD9029397
:10EC10000DF1220301930123297A00935832002336
:10EC2000090905F10C0000F0E5FCB9F1000F0BD06B
:10EC300004EB090A574593DB30194A4605F10C01EC
:10EC400008F0B1FA5FFA8AF42B7F002B77D0BC4230
:10EC500086D26B7F04F1010933556A7F5FFA89F927
:10EC6000D8F81430002A68D158330693AB6E06A941
:10EC700007932B7F06EB0900ADF8203000F0ACFBCA
:10EC80004844C4B2A7425AD240F275114B48F4F737
:10EC900075FF65E7032B01D0052B01D101236DE73B
:10ECA000002B3CD1082F7FF65BAFD8F81440701CC6
:10ECB000224652F8083FC6F8013053684360FFF718
:10ECC000A7FE102F7FF64CAF224652F8103F06F1F8
:10ECD0000900C6F8093053684360FFF799FE122F08
:10ECE0007FF63EAFB4F8983006A97374B4F8983044
:10ECF00005A81B0AB37413232834CDE90646ADF8E2
:10ED0000203000F033FB162F7FF62AAF1724059B27
:10ED1000C6F813306B66204612B0BDE8F087D8F80D
:10ED20000C30274898471BE740F23D112348F4F781
:10ED300025FF4FF0000905244BE7883395E7E31CD6
:10ED40009F427FF70DAFD8F814301A78102A0DD1F2
:10ED5000783306A905A8CDE90636ADF8204000F0C5
:10ED60006CFA059B33510434E4B2D4E7112A1DD167
:10ED700003F1780268330B930DF122030F930A9B82
:10ED80000BA91093B5F87A3005A8ADF8443095F882
:10ED90007C300C928DF8463095F87D300D968DF8CC
:10EDA0004730ADF8384000F080FADAE74FF4CB7125
:10EDB0000248F4F7E3FEAEE7C84B00203CD9010857
:10EDC00013D901082DE9F04F8F4DA3B02B7E0646D5
:10EDD0000F46904623B940F2A3118C48F4F7CEFEBB
:10EDE000022F2CD92B6880209847044630B9EB6855
:10EDF00087489847204623B0BDE8F08F8022002145
:10EE000008F0F5F933785B0923703278072B02F0AC
:10EE10000302627003D1EB687E4898470CE0B8F1BA
:10EE2000000F00F0EF81012B40F0C581AB687A48FC
:10EE3000F3E74246794898476B6820469847002494
:10EE4000D8E701F18802A0E1F3465068227A4FEA40
:10EE5000DC1E6EF300024FEA5C1E6EF382024FEA84
:10EE60001C1E6EF3C3026CF30712227282B24A4573
:10EE70004FEA104C84BF0CF1010C1FFA8CFC09EB1B
:10EE80000C4906EB0800CDF83090FFF7BFFD0DF1FF
:10EE9000880A68314AF8681D6066514607A800F084
:10EEA000CCF9079B626E934204D0EE685C495D48E2
:10EEB000B047C1E72A6909F10101BBF1000F2CD06D
:10EEC0005160227A04F10C03049313091A4606F1E7
:10EED00008010498059308F066F96A691178102909
:10EEE0000CD90DF12A0101910021CDF80890009173
:10EEF0005B46DDE90401583200F07CFB237A1B09F4
:10EF000003F10C0297422DD903F10D02974206D16D
:10EF1000002345482377EB686BE79160D1E709331D
:10EF2000A8EB0300617FC0B220776A6961B95832EB
:10EF30001E4408920996ADF828002B689847A066F1
:10EF400020B9EB68394868E78832F1E7514600F0AC
:10EF500043FA00283FF74EAFEB68354898476B6897
:10EF6000A06E5AE700232377A36643E7212F01D140
:10EF700001232AE1EB682F484FE79DF83F30043F1B
:10EF800009EB0700DB09FFF741FD6E696066A3B37B
:10EF90000DF1580A00213022504608F028F9FF23CD
:10EFA00032468DF8583052F8083F0DF15900CDF82F
:10EFB000593053683836CDF85D30FFF729FDB6F883
:10EFC00060303A468DF8613049461B0A0DF1630006
:10EFD0008DF8623008F0E7F8CDE9086A08F1070813
:10EFE00008A907A8ADF8288000F0C0F9636E079A59
:10EFF0009A4223D0EB6810480FE72836CDE908691C
:10F00000A8F10408ECE700BFC84B00203CD9010878
:10F01000B6D90108CED90108FCD901084BDA01089C
:10F0200062A2010886DA0108CBDA0108FFDA0108DA
:10F0300031DB010857DB0108C9DB01089DF83760A7
:10F040009DF83630360446EA03269DF835300DF13A
:10F050003B001E4366609DF83A709DF839303F04CE
:10F0600047EA03279DF838301F43A760FFF7CEFC1F
:10F07000E0609DF83F20237CD10961F3C71311099B
:10F0800061F3061362F3030323749DF84030637445
:10F0900094F8213003B322AB33F8472D9B7862827A
:10F0A000237522AB33F8442D9B78A4F81520E37523
:10F0B00022AB33F8412D9B782283A37622AB33F821
:10F0C0003E2D9B78A4F81B20637722AB33F83B2DB1
:10F0D0009B78E28384F820306D6994F9102005F163
:10F0E000280C002AB5F8981004F1230004F153030A
:10F0F000CDF858C016AA12DA05F11807ADF8681055
:10F100000092083504F1430204F13301CDE917768A
:10F11000199500F0FCF9012384F822306AE6ADF875
:10F1200064101946CDE9176700F0B0F90023F3E742
:10F13000EB68394871E6701CFFF768FC80450146B2
:10F140006060EB687FF475AE414634489847002311
:10F15000052F6377A7F1040807D9737903F00F032C
:10F1600008339845C4BFF35C6377F37996F806904B
:10F1700096F805C049EA0329637FA4F80A906969F3
:10F18000002B7FF45EAE01F158024FF0010E0878BB
:10F19000CDE9082662681028CDF82A20ADF828802D
:10F1A0008DF82EE02A6902D9002B7FF44DAE9068CD
:10F1B0004FF0000B4AE6032BBDD0052BBBD0012B33
:10F1C000B6D1112F7FF4D2AE002384F821306B69C1
:10F1D0001FFA87F828330893731C099308F1FF334B
:10F1E000ADF82830337808A90DF135008DF83430AA
:10F1F00000F0D4F800280DF134093FF7BEAEEB68FB
:10F2000007480AE6032B01D0052BD8D1701CFFF765
:10F21000FDFB60609BE700BFFEDB01081BDA010815
:10F22000A6DB01080022FFF7CDBD0B0A0170437079
:10F230000B0C090E8370C170704770B51025CEB0ED
:10F240000C462A4606460021684607F0D0FF4923AF
:10F250008DF80030A37BD4F80A100DF106008DF86C
:10F260000530FFF7E2FF21690DF10A00FFF7DDFF2E
:10F27000238908A88DF80F3000F000FA216808A84B
:10F2800000F00CFA2A46694608A800F00DFA228917
:10F29000616808A800F008FA08A90DEB050000F065
:10F2A0006EFA049B33604EB070BD492370B50025E3
:10F2B0000C460646CEB08DF800300B8BCDE90155DB
:10F2C0008DF801301B0A8DF802308B7E03958DF886
:10F2D0000330CB7E0DF106008DF804300B69196800
:10F2E000FFF7A3FF61690DF10A00FFF79EFFA389F5
:10F2F00008A88DF80F308DF80E5000F0BFF9216886
:10F3000008A800F0CBF9694608A8102200F0CCF953
:10F31000A289A16808A800F0C7F908A904A800F00C
:10F320002EFABDF8103008A833808DF804508DF8FF
:10F3300003508DF802508DF8015000F09FF961687C
:10F3400008A800F0ABF9694608A8102200F0ACF953
:10F35000A289A16808A800F0A7F908A904A800F0EC
:10F360000EFABDF8103073804EB070BD30B50C464B
:10F37000CBB0054604A800F081F9216804A800F08C
:10F380008DF92289616804A800F08EF904A9684605
:10F3900000F0F5F9009B2B604BB030BD70B50C89C7
:10F3A000BEB006460D46A4B114F00F0411D101AA57
:10F3B00010212868FFF740F92889A04201DC3EB0FF
:10F3C00070BD68683119204401AAFFF7AFF9103405
:10F3D000F2E74FF0FF30F2E72DE9F0430F89C7B0B5
:10F3E00081460D46002F4ED0012410224FEA1718F7
:10F3F000002117F00F0701A818BF08F1010807F056
:10F40000F6FEAB7BD5F80A100DF10A008DF8093035
:10F410008DF80440FFF709FF29690DF10E00FFF791
:10F4200004FF6E68013E444503DD288947B0BDE80E
:10F43000F08309AA102128688DF81340FFF7FCF823
:10F4400009AA05A901A8FFF771F9444510DB002FAF
:10F4500014BF3B46102330464A464B440DF1130C73
:10F46000934207D80134A4B209F110091036DAE743
:10F470001023F0E710F801EF1CF8011F81EA0E01DC
:10F4800002F8011BECE74FF0FF30CFE770B5C2B0D8
:10F49000144606460D46F122002105A807F0A7FEF6
:10F4A0000023CDE90333636810218DF805301A0A73
:10F4B0001B0C8DF80730A3688DF806208DF80830F6
:10F4C0001A0A1B0C8DF80A30A3898DF809208DF8D3
:10F4D0000B301B0A8DF80C30012305AA20688DF82B
:10F4E0000430FFF7A9F805AA314601A8FFF71EF975
:10F4F000022305AA102120688DF80430FFF79CF83C
:10F5000005AA294601A8FFF711F942B070BD2DE9FF
:10F51000F0431025C3B04A9C80460F461646002192
:10F52000F12205A8994607F062FE2A46002101A8AB
:10F5300007F05DFEA26829468DF80520130AEA400F
:10F540008DF80720E2688DF80630D37920688DF8B1
:10F55000083093798DF8093053798DF80A30137992
:10F560008DF80B30D3788DF80C3093788DF80D3002
:10F5700053788DF80E30137805AA8DF80F30238A52
:10F580008DF810301B0A8DF8113001238DF80430EE
:10F59000FFF752F805AA414601A8FFF7C7F8022372
:10F5A00005AA294660688DF80430FFF745F805AADA
:10F5B000494601A8FFF7BAF8032305AA294620689F
:10F5C0008DF80430FFF738F805AA394601A8FFF78F
:10F5D000ADF8042305AA294620688DF80430FFF70A
:10F5E0002BF805AA314601A8FFF7A0F843B0BDE803
:10F5F000F0830000F0B50F29C7B004460D4616464B
:10F600001F4604D94FF4A1711B48F4F7B7FA012340
:10F61000002F019318BF02238DF808309DF8303178
:10F620000DF10A0083F001038DF809304D9B196834
:10F63000FFF7FBFD4E990DF10E00FFF7F6FD4FF4BD
:10F64000807309AA1021304605AEADF81230FEF7DE
:10F65000F3FF09AA314601A8FFF768F80023601EEE
:10F66000DAB2954201D847B0F0BD10F8012FF15C35
:10F6700001334A400270F3E738DC010810B510226C
:10F6800004460021F13007F0B2FD00212046C4F805
:10F690001411F022BDE8104007F0A9BD0B46024648
:10F6A00010211846FEF7C8BF2DE9FF470446D0F8E1
:10F6B00014010E46154604F2011920B3C0F11008DA
:10F6C0009045474628BF174648443A4607F06BFD29
:10F6D000D4F814313B440F2BC4F814311ED9A8457B
:10F6E0001CD204F1F103194613F8012BD87B4B45CA
:10F6F00082EA000203F8012CF6D122460846FFF701
:10F7000015F83E44ED1B0DF1100A102D09D82A46BC
:10F710003146484607F047FDC4F8145104B0BDE82F
:10F72000F08704F1F002731E06F10F0013F8017F59
:10F7300012F8011F834281EA07011170F6D16A466F
:10F7400004F1F1039846174694461868596808333F
:10F75000ACE803004B456246F6D1224639463846AE
:10F76000FEF7E4FF43463A4603CA52451860596023
:10F77000174603F10803F6D11036103DC5E7F0B582
:10F780000C4689B0102200210546684607F02FFD7F
:10F79000224669466846FEF7C9FF9DF900306A4671
:10F7A000002B0DF10F0140DA137812F8010F5B0006
:10F7B0005BB243EAD013914202F8013CF4D19DF8C8
:10F7C0000F305B0083F087038DF80F30D4F81431CD
:10F7D000102B39D1002304F2011211781DF8030017
:10F7E00001334140102B02F8011BF6D104F1F10264
:10F7F000134604F2011712F8011BD07B974281EAED
:10F80000000102F8011CF6D104AA944616461868B5
:10F810005968083303C6BB423246F7D1224629460F
:10F820006046FEF783FF09B0F0BD137812F8010FB0
:10F830005B005BB243EAD0138A4202F8013CF4D188
:10F840009DF80F305B00BFE79DF900206846002A55
:10F8500028DA027810F8016F520052B242EAD6124A
:10F86000814200F8012CF4D19DF80F20520082F063
:10F87000870280218DF80F20E21882F80111002202
:10F8800001330F2B1DD9C4F81431002304F20112E7
:10F8900011781DF8030001334140102B02F8011BC1
:10F8A000F6D1A3E7027810F8016F520052B242EA93
:10F8B000D612814200F8012CF4D19DF80F2052009D
:10F8C000D7E7E11881F80121DAE70000002103E021
:10F8D0000A4B5B584350043109480A4B42189A427C
:10F8E000F6D3094A02E0002342F8043B074B9A4250
:10F8F000F9D300F00DF8F1F751FC704748E9010821
:10F900000000002080040020800400207C510020A2
:10F91000314B82B01A6842F480721A6099682F4A9B
:10F920000A409A601A6822F0885222F001121A6086
:10F930001A6822F480221A609A6822F47D029A6082
:10F940000022DA6001921B6813F4007318BF0123D0
:10F950000193019B012B37D14FF48051204B1A6842
:10F96000A3F5806322F00102C3F80024D3F8002439
:10F9700022F00202C3F80024D3F8002422F004028B
:10F98000C3F800245A6A42F080525A62154A116044
:10F990005168C906FCD49A689A609A689A609A6815
:10F9A0009A605A6822F460425A605A6842F44042AF
:10F9B0005A609A6822F003029A609A689A60064A2E
:10F9C000936813F00C0FFBD14FF00062064B9A6066
:10F9D000064ADA6002B07047003802400CC0FF8867
:10F9E000003C02400070004000ED00E00003FA051A
:10F9F00070B5064688B02E4801F0B0FC2D4B1A6851
:10FA00000092009A91073CD501214FF4007001F05B
:10FA1000FFFE012001F0F2FC274A536843F4003353
:10FA20005360A2F5374253681B07FCD5002401251B
:10FA300002A801F0CDFC02A91D488DF80D400694E6
:10FA40008DF81C508DF80C4001F09CFC2A460623D2
:10FA50003146174801F0DEFC2946154801F0C4FC88
:10FA60000221134801F068FD114801F057FD134DC4
:10FA700001940F4C0221204601F058FD58B108B006
:10FA800070BD1A6842F001021A60009A9207BBD456
:10FA90001A680092F9E7019B01330193019BB3F5CA
:10FAA000805FE7DB38212846F4F768F8E2E700BF1B
:10FAB0000024014000380240002701408BDC01088F
:10FAC00008B5002001F09AFC0021074801F08CFCE9
:10FAD00000214FF4007001F09BFE044A136823F0EC
:10FAE0000103136008BD00BF00240140003802403C
:10FAF00013B5072301220146114801F08BFC0221B6
:10FB00000F4801F019FD0E4801F008FD00230D4CCF
:10FB1000019302210A4801F009FD28B1084802B00A
:10FB2000BDE8104001F0FFBC019B01330193019B34
:10FB3000B3F5805FEDDB4C212046F4F71FF8E8E7D2
:10FB4000002401408BDC010870B506460825FFF74C
:10FB50004FFF00243046FFF7CBFF013D0444F9D1AD
:10FB6000FFF7AEFFC4F3CF0070BD0000000000003F
:10FB700008B51120FFF7E8FF06F0A4FD014608488C
:10FB800006F0ACFE06F086F903A3D3E9002306F0E5
:10FB9000D9F906F091FC08BD2FDD24068195F33FCD
:10FBA00000F07F450F4A536A43F0805353620E4B77
:10FBB0001A465968C906FCD41B68022823F4C053AE
:10FBC00006D143F4C05313605368DB06FCD470477E
:10FBD000012802D143F48053F5E70028F3D143F420
:10FBE0000063F0E7003802400070004010B50C4B95
:10FBF0005A68D206FCD41C6814F4C05F0BD114F40C
:10FC000080500AD114F4006404D106482A21F3F785
:10FC1000B5FF204610BD0220FCE70120FAE700BF37
:10FC200000700040D9DC010838B50546012001F01C
:10FC300093FC022D01BF144A136843F001031360C3
:10FC4000124B1A6842F480721A601A689205FCD549
:10FC50005A6822F4604242F440425A6000229A609C
:10FC60000A4B9C6814F00C04FBD14FF480721A60AC
:10FC7000074B084A28461A60FFF794FF2046BDE864
:10FC8000384001F05DBC00BF003C0240003802403B
:10FC9000F8010020D0FE3F000C4B5A6B900513D4A6
:10FCA0005A6A42F080525A62094A116841F48071DE
:10FCB0001160596B41F480715963596B8905FCD50A
:10FCC000136823F480731360704700BF003802404C
:10FCD00000700040054B5A6B910706D45A6B42F0F6
:10FCE00001025A635A6B9207FCD5704700380240F4
:10FCF000094B5A6A42F020025A629A6942F0200285
:10FD00009A619A6922F020029A610022A3F50933D0
:10FD10001A801A855A62704700380240152102384D
:10FD2000002248430121064B1A85D86299825A6203
:10FD30001A8219801A8AD207FCD500221A807047CD
:10FD400000140040002349F6FE7282B00193019B2B
:10FD5000934201DD02B07047019B01330193F6E746
:10FD6000002340F6FE7282B00193019B934201DDB5
:10FD700002B07047019B01330193F6E7002382B084
:10FD80000193019BB3F5CC7F01DD02B07047019B6D
:10FD90000133F5E7D0B1012801D1FFF7EFBF0C4BDC
:10FDA00000211A684FF47A73B2FBF3F2094B013A5F
:10FDB00092B21A8501220138D8629A825962198258
:10FDC0001A801A8AD207FCD500221A80704700BF19
:10FDD000F80100200014004000F1774303F5780398
:10FDE000B3F5804F2DE9F04106460C4617462DD25B
:10FDF00002F1F73303F608030344B3F5804F25D22D
:10FE0000FFF7F4FE804610B10020FFF7CBFE01F0B3
:10FE1000BBFB01252744361BA7420AD101F0C4FBD6
:10FE2000B8F1000F02D04046FFF7BCFE2846BDE8FF
:10FE3000F08141F6027001F0BFFB301914F8011B8C
:10FE400001F016FC042818BF0025E5E70025EDE7C2
:10FE500010B50C4600F1774101F57801B1F5804FFE
:10FE60000DD202F1F73303F608030344B3F5804FD4
:10FE700005D20146204607F096F9012010BD00206A
:10FE8000FCE7000008B5114B984215D003F58063DC
:10FE9000984213D003F58063984211D003F5806334
:10FEA00098420FD003F5006398420DD0084B094AE1
:10FEB0001421094807F024F8002008BD0120FCE7C0
:10FEC0000220FAE70320F8E70520F6E700000240E9
:10FED00070DD01082ADD010889DD01080F2808B559
:10FEE00005D9094B094A3B21094807F009F80123C4
:10FEF00003FA00F0C043074A51680140516013689B
:10FF00001840106008BD00BFDADD010834DD0108CB
:10FF100089DD0108000401400F292DE9F84F8246D0
:10FF20000D4693461F4605D95A4B5B4A54215B4800
:10FF300006F0E6FF4FF0010909FA05F900F0B8F8FC
:10FF40006FEA0903564E032D7268564C02EA03020B
:10FF50007260326803EA0203534A3360136A43F063
:10FF6000010313622ED80F22A3684FEA850802FA14
:10FF700008F223EA0203A3605046FFF783FFA36859
:10FF800000FA08F01843A0601BF0020F18BFB36816
:10FF9000464A1CBF43EA0903B3601BF0040F1EBFAF
:10FFA000F36843EA0903F360336843EA0903336003
:10FFB0003B01DBB2002D45D182F8063340231360AC
:10FFC000BDE8F88F072D13D80F22A5F10408E368C8
:10FFD0004FEA880802FA08F223EA0203E360504677
:10FFE000FFF750FFE36800FA08F01843E060CBE742
:10FFF0000B2D13D80F22A5F1080823694FEA8808B2
:020000040801F1
:1000000002FA08F223EA020323615046FFF73AFF9F
:10001000236900FA08F018432061B5E70F22A5F123
:100020000C0863694FEA880802FA08F223EA02031F
:1000300063615046FFF726FF636900FA08F0184332
:100040006061A1E7012D03D182F807338023B6E771
:10005000022D04D182F808334FF48073AFE7032DEB
:1000600004D182F809334FF40073A8E7042D04D1BA
:1000700082F80A334FF48063A1E7092D04D882F88F
:1000800017334FF400039AE782F828334FF4807354
:10009000536095E7E6DD01084FDD010889DD0108C1
:1000A00000040140000001400038024000E100E08F
:1000B000144B984205D1144AD36943F00103D3612C
:1000C0007047124B984204D10F4AD36943F00203A0
:1000D000F5E70F4B984204D10B4AD36943F0040370
:1000E000EDE70C4B984204D1074AD36943F008036B
:1000F000E5E7094B9842E3D1034AD36943F0200373
:10010000DDE700BF0000024000380240000402406A
:1001100000080240000C0240001402400323490082
:1001200010B584688B4024EA030484600124022A09
:1001300004FA01F407D0032A0DD0012A07D18368FD
:100140002343836003E083688A401A4382608368A4
:100150001C43846010BD82681343F2E70F29F8B591
:1001600004460F4615461E4603D940211948F3F7A9
:1001700005FD2046FFF79CFF03237A009340DB43F5
:100180002168194021600121D4F800C001FA02F071
:100190004CEA000CB940C4F800C009B266B1A688A8
:1001A000314389B2A180E168012D03EA0103E360D4
:1001B00006D0022D08D0F8BDA68826EA0101F1E795
:1001C000E3680343E360F6E7E36805FA02F21A43E3
:1001D000E260F0E736DE01080F2970B505460C46EF
:1001E000164603D960210E48F3F7C8FC2846FFF7EE
:1001F0005FFF032361008B40DB43EA68012E02EAC4
:100200000302EA6005D0022E03D02A6813402B6057
:1002100070BDEA6806FA01F11143E960F5E700BF35
:1002200036DE01080F2910B505D9074B074A76219C
:10023000074806F065FEFFF73BFF4B00032102680D
:1002400099401143016010BDDADD0108F2DD0108BB
:1002500036DE01080F2938B50446154605D97C213C
:100260001B4B1C4A1C4806F04BFE0F2A03D91B4BA4
:10027000184A7D21F6E7FFF71BFF07294FF00F0310
:1002800018D8006A8A00934020EA03032362236A95
:1002900005FA02F21A4322620322236849008A40C7
:1002A00023EA020323600223226803FA01F11143C7
:1002B000216038BDA1F10802406A9200934020EA13
:1002C00003036362636A95401D436562E4E700BF10
:1002D000DADD010805DE010836DE010823DE01084B
:1002E000012303FA01F189B201837047012303FA64
:1002F00001F189B241837047012303FA01F189B208
:100300000AB10183704741837047008A084100F0B9
:10031000010070470F2938B505460C4603D9A921BD
:100320000548F3F72BFC28686400E04000F0030068
:10033000431E5842584138BD36DE0108808A0841C4
:10034000C04300F00100704710B5084C23681BB98A
:100350000120F1F7B9FB206023682BB9BDE81040FC
:1003600036210348F3F70ABC10BD00BFE44B002060
:1003700085DE010810B50B4C22681AB93C210A48E9
:10038000F3F7FCFB206842F21071F1F7E5FC01285D
:100390000CBF0124002403D040210348F3F7EEFBF7
:1003A000204610BDE44B002085DE010810B5074C47
:1003B00022681AB94D210648F3F7E0FB00232068B4
:1003C0001A46BDE810401946F1F7DABAE44B0020AE
:1003D00085DE010810B50446FFF7B6FFFFF7CAFF38
:1003E00021461022034801F0C1FE0446FFF7DEFF5C
:1003F000204610BD0054004010B5FFF7A5FFFFF7E1
:10040000B9FF01F06BFE0446FFF7D0FF204610BD98
:1004100008B513460A460146034801F0DDFA0030EC
:1004200018BF012008BD00BF0054004008B51346A6
:100430000A460146034801F0D5FB003018BF0120F1
:1004400008BD00BF0054004008B513460A460146E7
:10045000034801F059FC003018BF012008BD00BF5F
:100460000054004008B513460A460146034801F00F
:10047000DBFC003018BF012008BD00BF0054004065
:1004800008B513460A460146034801F025FD003031
:1004900018BF012008BD00BF005400400123064AD8
:1004A00083405169194205D05361044B53F8203001
:1004B00003B11847704700BF00040140E84B00201B
:1004C0000F2838B504460D4603D926210348F3F713
:1004D00055FB034B43F8245038BD00BFD3DE010861
:1004E000E84B00200020FFF7D9BF0120FFF7D6BF5F
:1004F0000220FFF7D3BF0320FFF7D0BF0420FFF790
:10050000CDBF08B50920FFF7C9FF0820FFF7C6FFD8
:100510000720FFF7C3FF0620FFF7C0FFBDE8084034
:100520000520FFF7BBBF08B50F20FFF7B7FF0E2070
:10053000FFF7B4FF0D20FFF7B1FF0C20FFF7AEFF70
:100540000B20FFF7ABFFBDE808400A20FFF7A6BF6E
:10055000FEE7FEE7FEE7FEE7FEE7FEE7FEE7FEE773
:10056000FEE7FEE7FEE7FEE7FEE7FEE7FEE7FEE763
:10057000FEE7FEE7FEE7FEE7FEE7FEE7FEE7FEE753
:10058000FEE7FEE7FEE7FEE7FEE7FEE7FEE7FEE743
:10059000FEE7FEE7FEE7FEE7FEE7FEE7FEE7FEE733
:1005A0000A23B0FBF3F203FB120040EA0210C0B2D0
:1005B00070470000CA22024B5A6253225A627047A7
:1005C00000280040014B1860704700BF284C0020F5
:1005D0004FF400320F4B10B50F4C5A61E368DB0546
:1005E00003D430210D48F3F7C9FAFFF7E3FF4FF4C6
:1005F0000072A36823F48853A360094BC3F88420D6
:10060000FF236362074B1B6813B1BDE81040184716
:1006100010BD00BF000401400028004021DF010898
:1006200000E100E0284C00202DE9F04F9846374BC0
:1006300085B01B78824691469DF838709DF83C60E5
:100640002BB9334B334A8C21334806F059FC431EF7
:100650001E2B59D80C2957D8A2F5FA63632B53D80F
:10066000B8F1170F50D83B2F4ED83B2E4CD802F183
:100670003000C0B2FFF794FF83460846FFF790FFB3
:1006800004465046FFF78CFF40F400554046FFF704
:1006900087FF45EA0B4545EA042504463846FFF73F
:1006A0007FFF000240EA04443046FFF779FF204311
:1006B0001A4CFFF77FFFE36843F08003E360E368D1
:1006C0005B06FCD565602060E36823F08003E3608F
:1006D000124BDA689206FCD5FF2204A85A6200F891
:1006E0000C6D8DF807A08DF80810ADF809908DF805
:1006F00006808DF80570FAF78AFD094BC3E9000101
:10070000012005B0BDE8F08F0020FAE72C4C002056
:10071000A2DF01086FDF010821DF01080028004087
:10072000304C002037B50578C4788378B0F80520C0
:1007300001790195407800902046FFF775FF03B0DE
:1007400030BD000038B52B4B04461B781BB9E421A3
:100750002948F3F713FA294AD36823F02003D3601A
:10076000D3689B06FCD513685268C2F30741080999
:1007700000EB800001F00F0101EB4001C9B201F56F
:10078000FA61A4F80510C2F30721C1F30010850037
:10079000284401F00F0101EB4001D2B22171C2F3F4
:1007A000011101EB810102F00F0202EB4102E27044
:1007B000C3F30742C2F3011101EB810102F00F0202
:1007C00002EB4102A270C3F30722C2F3021101EB54
:1007D000810102F00F0202EB4102DBB26270C3F34F
:1007E000021202EB820203F00F0303EB42032370B9
:1007F00038BD00BF2C4C002021DF0108002800403C
:100800001FB501A8FFF79EFF01A8FAF700FD05B08C
:100810005DF804FB08B5FFF73FFA1B4A136843F481
:1008200080731360FFF7C6FE184A536B23F44033FE
:1008300043F482035363164BDA6842F08002DA60B5
:10084000DA685106FCD5FF221A611A6942F4FE02E9
:100850001A619A6822F040029A609A6822F44C5217
:100860009A60DA6822F08002DA60094BDA68920650
:10087000FCD5FF225A620122064B1A70FFF7C0FF17
:10088000054BC3E9000108BD00700040003802407C
:10089000002800402C4C0020304C002008B5094BAB
:1008A0001B7823B940F21F110748F3F767F9FFF7E8
:1008B00081FE064B9A6822F480729A60FF225A6287
:1008C00008BD00BF2C4C002021DF0108002800409B
:1008D00008B5144B1B7833B9134B144A40F2271157
:1008E000134806F00DFBFFF765FE124BDA6822F4A1
:1008F0008072DA60104A916841F4003191601168A9
:1009000041F400311160F0210C4A82F829134FF4B0
:10091000007151609A6842F488529A60FF225A62CC
:1009200008BD00BF2C4C0020A2DF01087BDF0108BE
:1009300021DF0108002800400004014000E100E040
:10094000F8B51E46194B17461B7833B9184B194A90
:100950004FF4A371184806F0D3FA184CFFF72AFE9B
:10096000A56825F48075A560E56825F48075E560C7
:10097000FFF716FE05460846FFF712FE000440EAA0
:1009800005613846FFF70CFE05463046FFF708FEC6
:10099000084340EA0520E368DB07FCD5FF23E0615C
:1009A0006362BDE8F840FFF793BF00BF2C4C002006
:1009B000A2DF010890DF010821DF010800280040C4
:1009C000037842788178C078FFF7BABF38B50D4612
:1009D0000446F2F797FE194A136823F001031360E7
:1009E000F2F7B0FE25B1164A536843F00603536090
:1009F00072B6BFF34F8FBFF36F8F124A0120136897
:100A000023F0030343F4007343F00103136000F089
:100A1000AFFD0D4B1A6942F004021A6130BF1A692A
:100A2000022022F004021A61FFF7FEF8034A13685D
:100A300043F00103136004B162B638BD10E000E07A
:100A4000002004E00070004000ED00E062B6704756
:100A500000220E4B10B51A700D4A0E4C138820461A
:100A600023F040031B041B0C13800D210222FFF70F
:100A7000B3FB204602220E21FFF7AEFB2046BDE865
:100A8000104002220F21FFF7A7BB00BF384C002007
:100A9000003800400004024038B50546274A28487F
:100AA000536A0C4643F4804353620D210522FFF73D
:100AB000D1FB05220E212248FFF7CCFB05220F2196
:100AC0001F48FFF7C7FBC5B101220D211C48FFF7E6
:100AD00025FB01220E211A48FFF720FB01220F21DE
:100AE0001748FFF71BFB012C21D144F4517401225C
:100AF000144B1C80144B1A7038BD2A460D21104827
:100B0000FFF70CFB2A460E210D48FFF707FB2A468C
:100B10000F210B48FFF702FB012C05D0022C03D05C
:100B2000032C14BF0024032444F45974DFE7022C7F
:100B3000DBD0032C0CBF03240024D6E7003802408E
:100B40000004024000380040384C0020064B074AA1
:100B5000988111781A461889C00701D40029FAD162
:100B60009089C0B2704700BF00380040384C002068
:100B7000284A38B5136A054643F4805313620522A8
:100B800025480C461146FFF765FB05220621224841
:100B9000FFF760FB052207211F48FFF75BFBC5B18C
:100BA000022205211C48FFF7B9FA022206211A4841
:100BB000FFF7B4FA022207211748FFF7AFFA012C1A
:100BC00021D144F451740122144B1C80144B1A702F
:100BD00038BD2A4605211048FFF7A0FA2A4606210B
:100BE0000D48FFF79BFA2A4607210B48FFF796FAB4
:100BF000012C05D0022C03D0032C14BF00240324A5
:100C000044F45974DFE7022CDBD0032C0CBF03241F
:100C10000024D6E7003802400000024000300140C6
:100C2000394C002000220E4B10B51A700D4A0E4CA4
:100C30001388204623F040031B041B0C138005215E
:100C40000222FFF7C9FA204602220621FFF7C4FA62
:100C50002046BDE8104002220721FFF7BDBA00BFC1
:100C6000394C00200030014000000240064B074A8A
:100C7000988111781A461889C00701D40029FAD141
:100C80009089C0B2704700BF00300140394C00204D
:100C9000054AD36823F4E0631B041B0C43F0BF63D5
:100CA00043F40033D360704700ED00E020220021C0
:100CB000114B10B5C3F88420104B114C1A6A204612
:100CC00042F480421A625A6942F480425A615A6977
:100CD00022F480425A610B4A91811A6A092122F456
:100CE00080421A620222FFF777FA2046BDE81040E0
:100CF00002220A21FFF770BA00E100E0003802404A
:100D0000000002400038014008B5064B024618605A
:100D100000B1012240F22551034800F018FE0120E5
:100D200008BD00BF3C4C00200038014010B50B4C02
:100D300040F22551204600F028FE48B1204600F040
:100D400002FE074BC0B21B6833B1BDE81040184724
:100D5000A388044ADBB2137010BD00BF0038014005
:100D60003C4C0020F450002010B504468021084877
:100D700000F005FE0028F9D02146054800F0DFFD0F
:100D8000034C4021204600F0FAFD0028F9D010BDA8
:100D90000038014010B5441E14F8010F00B910BD11
:100DA000FFF7E2FFF8E7000008B5024800F0CBFDCE
:100DB000C0B208BD003801402DE9F043884601214A
:100DC00089B08146084614461D4600F015FD0121F4
:100DD0004FF4804000F01CFD4FF4C0670223012255
:100DE000002602A93F488DF80C308DF80D308DF8A3
:100DF0000F2002978DF80E6000F060FC0722092199
:100E0000384800F09DFC07220A21364800F098FC83
:100E1000B8F1450FCDF810903CD14FF48063ADF898
:100E20001830072C42D10023ADF81430052D4ED1D7
:100E30004FF48053ADF816300023ADF81C300C236E
:100E400004A92948ADF81A3000F01EFD274B1A6896
:100E500002B1012240F22551234800F078FD012122
:100E6000214800F061FDFFF79FFF25238DF8043036
:100E70009DF840308DF8053000238DF806300123B1
:100E80008DF80730FFF704FF01A800F04BFA09B016
:100E9000BDE8F083B8F14F0F02D1ADF81870C0E78C
:100EA000072CADF818600DD1592107E0082C02D1AC
:100EB0004FF48053B8E7092CB8D154210C48F2F70D
:100EC0005DFEB3E7082CAED0092CAFD1F0E70F2DB3
:100ED00002D14FF44053ADE7022D0CBF4FF4005345
:100EE0000023A7E700000240003801403C4C0020EE
:100EF000ABDF01080E2307B5082200934E21012322
:100F0000FFF75AFF03B05DF804FB00004022002108
:100F10000D4B0E48C3F884200D4B5A6A42F4003240
:100F20005A629A6942F400329A619A6922F4003254
:100F30009A61084A91815A6A032122F400325A6266
:100F40000222FFF749B900BF00E100E000000240C3
:100F5000003802400044004008B5024800F0F3FCAD
:100F6000C0B208BD004400402DE9F04F4FF0000929
:100F70001F46262389B09DF848808A4614468DF87E
:100F8000043083469DF84C509DF850608DF80580E4
:100F90008DF806908DF80790FFF77AFE01A800F013
:100FA000C1F90121084600F027FC01214FF400306F
:100FB00000F03AFCB5B10823029302238DF80E909D
:100FC0008DF80C304FF00309012302A956488DF823
:100FD0000F308DF80D9000F071FB07224946524802
:100FE00000F0AEFBBEB10423029301238DF80F3055
:100FF00000234FF002098DF80E30032302A94A485E
:101000008DF80C908DF80D3000F058FB0722494602
:10101000454800F095FBBAF1450FCDF810B043D12B
:101020004FF48063072CADF818304BD10023ADF896
:101030001430052F57D14FF480530024ADF81630EB
:10104000ADF81C40002E59D1ADF81A6075B1BDF84D
:101050001A3043F00403ADF81A30344B1A6802B169
:10106000012240F22551324800F071FC04A93048B9
:1010700000F00AFC01212E4800F056FC0DB1FFF7EC
:101080006BFF26238DF8043000238DF806300123F2
:101090008DF805808DF80730FFF7FAFD01A800F004
:1010A00041F909B0BDE8F08FBAF14F0F02D14FF40A
:1010B000C063B7E70023072CADF818300ED14FF40A
:1010C000827107E0082C02D14FF48053AFE7092C5E
:1010D000AFD1FF211748F2F751FDAAE7082CA5D0A0
:1010E000092CA6D1F0E70F2F02D14FF44053A4E70B
:1010F000022F0CBF4FF4005300239EE70823224623
:1011000040F227710A48ADF81A3000F020FC40F296
:101110002661074800F058FC224640F22661044848
:1011200000F015FC92E700BF00000240404C002098
:1011300000440040ABDF0108F8B505460024134E1B
:10114000134F8021134800F01AFC68B1294611485A
:1011500000F0F5FB00240F4D0C4E0D4F40212846AA
:1011600000F00DFC48B1F8BD0134B442E9D94FF4A8
:10117000A4713846F2F702FDE3E70134B442EDD939
:1011800040F251113846F2F7F9FCE7E7FFFF0F0094
:10119000ABDF01080044004008B5064B024618606A
:1011A00000B1012240F22551034800F0D0FB01209C
:1011B00008BD00BF404C00200044004070B5134CF7
:1011C00040F22551204600F0E0FBC0B1104B1D68F5
:1011D00025B1204600F0B7FBC0B2A84740F2266117
:1011E0000A4800F0D2FB78B140F22661074800F0CF
:1011F000EBFB084B1B683BB1BDE870401847A38868
:10120000054ADBB21370E9E770BD00BF004400403F
:10121000404C0020444C0020F4500020BFF34F8F7E
:101220000449054BCA6802F4E0621343CB60BFF384
:101230004F8FFEE700ED00E00400FA0510B5441EF4
:10124000E3B2052B03D90E211148F2F797FCFEF704
:1012500041FD45F255520F4B1A60DA68D207FCD4B3
:10126000052C06D8DFE804F003090B0D0F1101224D
:101270005A604CF6CC421A6010BD0222F8E70322F5
:10128000F6E70422F4E70522F2E70622F0E700BFC2
:1012900084E001080030004010B5194C23683BB9C8
:1012A0005F2000F0D9FA28B1164B236000F0E4FA71
:1012B000206810BD5E2000F0CFFA08B1124BF4E7B1
:1012C0005D2000F0C9FA08B1104BEEE75C2000F099
:1012D000C3FA08B10E4BE8E75B2000F0BDFA08B195
:1012E0000C4BE2E75A2000F0B7FA08B10A4BDCE7F2
:1012F000592000F0B1FA08B1084BD6E7084BD4E703
:10130000484C0020FADF01080AE0010820E001084B
:101310003BE001084AE0010859E0010872E00108D9
:101320007CE0010830B5012403780A4D03F01F0268
:101330009440C278590952B1074A2B44D268427886
:101340001201D2B283F8002345F8214030BD20318C
:10135000FAE700BF00E100E000ED00E008B5084B4F
:1013600098420BD101214FF4007000F069FABDE8FA
:10137000084000214FF4007000F062BA08BD00BFC1
:101380000024014043680A7923F0407323F48073FA
:1013900043EA02230A6810B513434360D1E90323EB
:1013A00013438A6884681343084A224013434A79E6
:1013B00043EA420383600A7D036B013A23F0F8732A
:1013C000D2B243EA0253036310BD00BFFDF7FFC072
:1013D00000234FF040720360037143718360C0E9E2
:1013E0000323012303757047836819B143F0010398
:1013F0008360704723F00103FAE70000044B5A684A
:1014000018B142F400025A60704722F40002FAE771
:10141000002701401D2970B51BD90725A1F11E0623
:10142000C46D06EB4606B54024EA050403FA06F649
:101430002643C665062A38D81F24013A036C02EBFE
:101440008202944023EA040301FA02F21A4302647E
:1014500070BD13290DD90726A1F11405C46805EB49
:101460004505AE4024EA060403FA05F52543C560A8
:10147000E0E709290DD90726A1F10A04056904EB63
:101480004404A64025EA060503FA04F42C4304614B
:10149000D0E70726446901EB4105AE4024EA060483
:1014A00003FA05F626434661C4E70C2A0CD81F242C
:1014B000073AC36B02EB8202944023EA040301FA69
:1014C00002F21A43C263C3E7122A0CD81F240D3A52
:1014D000836B02EB8202944023EA040301FA02F2D6
:1014E0001A438263B4E7182A0CD81F24133A436BBB
:1014F00002EB8202944023EA040301FA02F21A4347
:101500004263A5E71F24193A036B02EB8202944061
:1015100023EA040391401943016399E7836843F088
:10152000804383607047806D80B2704703681942C2
:1015300014BF012000207047C943016070470000BC
:10154000044B1A6818B142F002021A60704722F088
:101550000202FAE7003C0240044B1A6818B142F05C
:1015600004021A60704722F00402FAE7003C0240CD
:10157000044B1A6818B142F008021A60704722F052
:101580000802FAE7003C0240044B5A68D20741BF08
:10159000034ADA60034ADA60704700BF003C024049
:1015A000EFCDAB8905040302024A536843F00103FF
:1015B00053607047003C0240014B9861704700BF88
:1015C000003C0240084B9A69D10709D49A69D205B8
:1015D00008D49B6913F4F05F14BF03200420704704
:1015E0000120704702207047003C0240042313B5DD
:1015F00004468DF80730FFF7E5FF8DF807009DF8EA
:101600000730012B0AD11CB905238DF8073007E0FC
:10161000FFF7D8FF013C8DF80700F0E7002CF3D06E
:101620009DF8070002B010BD10B504464FF400400D
:10163000FFF7DCFF042804BF0023236010BD000077
:1016400038B504464FF400400D46FFF7CFFF04289D
:101650000BD1064A4FF40040536823F48073536063
:101660002560BDE83840FFF7C1BF38BD003C0240EF
:1016700038B504464FF400400D46FFF7B7FF042885
:101680001BD135B125704FF40040BDE83840FFF75D
:10169000ADBFFF2324F0030504F003042968E40030
:1016A00003FA04F421EA04042846FFF7BDFF2146AB
:1016B0002846BDE83840FFF7C3BF38BD2DE9F043E9
:1016C0000022012703250E6807FA02F333EA060415
:1016D00031D14FEA420C05FA0CF4E44391F804E0EE
:1016E000D0F800900EFA0CF804EA09090EF1FF3E5A
:1016F00048EA0908BEF1010FC0F8008011D8D0F8FF
:1017000008E004EA0E0E4C7904FA0CF444EA0E04E4
:101710008460848824EA03048B7993409BB223433A
:101720008380C36805FA0CF423EA0404CB7903FA36
:101730000CF32343C3600132102AC5D1BDE8F08306
:1017400010B50F2401F00703C90800EB8100016AFE
:101750009B009C4021EA04010162016A9A400A430D
:10176000026210BD204B10B59A6802F00C020C2AE0
:1017700030D8DFE802F02F2F2F2F072F2F2F072F22
:101780002F2F2000194B184A036093681849C3F3A0
:101790000313CC5C0368E34043609468C4F3022401
:1017A0000C5D23FA04F484609268C2F3C2228A5C5E
:1017B000D340C36010BD99680E4CC1F383419A6851
:1017C000615C9B68094BC2F381524B430132B3FB0E
:1017D000F2F3D8E74FF400425B68C3F342330133BE
:1017E00002FA03F3CFE700BF003802400024F40000
:1017F000FC0100200C020020044BDA6911B11043F7
:10180000D861704722EA0000FAE700BF00380240C2
:10181000044B1A6A11B110431862704722EA0000A3
:10182000FAE700BF00380240044B5A6A11B1104376
:101830005862704722EA0000FAE700BF0038024011
:10184000044B5A6911B110435861704722EA0000F5
:10185000FAE700BF003802404309012B054B00F0B6
:101860001F000CBF1B685B6B23FA00F000F0010047
:10187000704700BF00380240024A536B43F0807348
:10188000536370470038024030B50D460446028A63
:10189000EB8892B222F440521A43898902828389EA
:1018A000288923F4B052AB8822F00C0203436889E4
:1018B00085B003431343A381A38A68469BB223F4F4
:1018C00040730B43A382FFF74DFFDDE90231154A58
:1018D000944218BF19461923A2894B432968100462
:1018E0004CBF49008900B3FBF1F16425B1FBF5F36E
:1018F000A2891801120405FB13130BD5DA0032324A
:10190000B2FBF5F202F0070242EA00039BB2238128
:1019100005B030BD1B013233B3FBF5F303F00F0309
:101920000343F3E700380140838919B143F40053BE
:101930008381704723F400531B041B0CF8E7C1F3A9
:101940000801818070478088C0F30800704701F06B
:101950001F0310B5C1F342140121012C01FA03F158
:1019600005D10C3003683AB11943016010BD022C57
:101970000CBF10301430F5E723EA0101F5E70388C6
:10198000194214BF0120002070470123C1F3421205
:1019900010B5012A01F01F0403FA04F30DD1828966
:1019A0001340028892B26BB10123090A03FA01F1D4
:1019B0000A4214BF1846002010BD022A0CBF028A3A
:1019C000828AEDE71846F7E70B0A01219940C943DF
:1019D00089B20180704700002DE9F3411F460023C2
:1019E00004460D46019316461AB9012002B0BDE81F
:1019F000F08140F6FF7301934FF40031204600F070
:101A00000EFD002852D10121204600F0D8FC4FF2F3
:101A1000FF71204600F0ECFC0121204600F0B9FCEB
:101A200040F6FF73DFF8B88101934146204600F08D
:101A3000EBFC002841D039460122204600F0CAFCC8
:101A400040F6FF73614F01933946204600F0E7FCF2
:101A5000002838D0012E42D10021204600F0AFFCF2
:101A6000F1F750FE31462046238B00F09DFCF1F744
:101A700069FE40F6FF73564E01933146204600F052
:101A8000CEFC30B3204600F0B0FC287040F6FF7367
:101A9000504D01932946204600F0C1FC0028A4D0F7
:101AA000019B5A1E0192002BF4D104E0019B5A1EA7
:101AB0000192002BA0D1002098E7019B5A1E0192B1
:101AC000002BB2D1F7E7019B5A1E0192002BBBD12C
:101AD000F1E7019B5A1E0192002BCED1EBE7022EBB
:101AE00025D1F1F70FFE4FF40061204600F080FC95
:101AF0000021204600F063FC238BF1F723FE40F623
:101B0000FF73354E01933146204600F088FC40B10A
:101B10000121204600F048FC238A2B70238A6B7039
:101B2000B4E7019B5A1E0192002BECD1C3E740F6AB
:101B3000FF77033E238BDFF8A0802E44B542019748
:101B40002CD1254E3146204600F069FC90B300218F
:101B5000204600F034FCF1F7D5FD204600F045FCAE
:101B600001212870204600F01FFCF1F7EBFD204614
:101B700000F03BFC40F6FF73184E6870019331464D
:101B8000204600F041FCD8B1204600F02EFCA870A1
:101B90007CE7019B5A1E0192002B8CD041462046C7
:101BA00000F03DFC0028F4D0204600F01EFC05F8B3
:101BB000010BC3E7019B5A1E0192002BC2D17AE7A9
:101BC000019B5A1E0192002BD9D174E7020000102C
:101BD000400000101000001004000010400003003E
:101BE000010003002DE9F3411E46002304460D4683
:101BF000019317461AB9012002B0BDE8F08140F602
